:1000000001000000000000A0000200000AB6BD1BB5
:100010001CF09FE51CF09FE51CF09FE51CF09FE5A0
:100020001CF09FE51CF09FE51CF09FE51CF09FE590
:100030000C1D0F0A5C120200A4110200B411020090
:100040000C1202001C1202002C1202003C120200D0
:1000500048120200000000EA488300EA28008FE20C
:10006000000C90E800A08AE000B08BE001704AE24A
:100070000B005AE14183000A0F00BAE814E04FE296
:10008000010013E303F0471013FF2FE11C160200D9
:100090005C1602000030A0E30040A0E30050A0E3A3
:1000A0000060A0E3102052E27800A128FCFFFF8A44
:1000B000822EB0E13000A128003081451EFF2FE1E3
:1000C00004309FE503308FE013FF2FE1750F02002E
:1000D0001D48802110B549F3DAEB1C48582149F33B
:1000E000D6EB1B4800210A0006C0202117485830D3
:1000F00049F3CCEB002010BDF0B50024144F0837B5
:10010000012609E0C519686801F04CFC69683000F7
:10011000884010498860641CE00039580029F1D1FA
:100120000B4F0024283709E0C519686801F03AFC34
:1001300069683000884008498860641CE0003958CC
:100140000029F1D10020F0BDD8160200F00F000404
:10015000400E0004009000A8009100A85E48042210
:100160000621027041700271417102724172704742
:10017000F8B505F0FCFA002803D002F0FFFC0028D7
:1001800079D1554800241838046000F02CFB05F0A4
:10019000BBFA52490D5C01F0B1FD290049F3BEECF8
:1001A0004F4E2300320049F338E9401C61410504F9
:1001B0002D0C05F0A9FA4B4940000F5A05F07DFBC4
:1001C000390049F3ACEC2300320049F326E9401C26
:1001D00061410004000C290000F014FB05F094FAC2
:1001E00041490D5C01F08AFD290049F398EC230098
:1001F000320049F312E9401C614105042D0C05F061
:1002000083FA3A490F5C01F079FD390020DD13C70C
:1002100001000000FC0100A000020000CE6362307B
:1002200049F386EC2300320049F300E9401C6141A8
:100230000004000C290000F006FB082000F0F2FA90
:1002400001F066FD310049F38EEC401C0004000C07
:1002500000F0F1FA01F05CFD052149F36AEC294A4E
:10026000230049F3E4E81922801861410006000EDA
:1002700000F0EFFA601E04F0D7F8FF24641C2000A1
:1002800004F0CCF8200004F0D5F804F0E5F804F010
:10029000F7F8402002F01AFC00F0ECFA00F0E1FA66
:1002A00019490120086004F017F904F02FF904F04F
:1002B00036F904F069F90C2001F01FFDC02001F0AF
:1002C0001CFD04F079F904F089F904F090F904F0C8
:1002D000A0F9302001F011FD0320000201F00DFD16
:1002E000FFF746FF00F090F9F8BD0000B05900B0EC
:1002F0002C00000440420F001600000442000004DD
:1003000037000004C0C62D00E85900B010402DE9A8
:100310005A8400EB78409FE5000094E5000050E32C
:100320000300000A6A0100FA000094E5000050E3AF
:100330005484001B080200FA0000A0E3E41500FB4F
:10034000950100FA0000A0E35B0100FB5B0100FAED
:10035000000094E5000050E34C01001BAF0100FBDE
:10036000DF0100FB000094E5000050E30100000AFB
:10037000AB0100FB431600FAA90100FA00000FE1EF
:10038000BF0000E200F021E13C1500FA0000A0E30C
:100390001080BDE8506600B010B500F0A3FC05F376
:1003A0009FF905F07BFB00F077FC002801D00120CD
:1003B00010BD05F073FF002010BD10B5FFF7E2FE81
:1003C00020F06AFE0400012003F0BCFF200020F0B2
:1003D00067FE05F0D6F9002805D002F0D9FB002809
:1003E00001D002F0C0FB002010BD10B502F044FDAA
:1003F00010BD9308002210B502E09400521C015178
:100400009A42FAD310BD064A0648002110B5FFF7FC
:10041000F0FF00F015FB00F09BF900200B414E0AA5
:1004200001000000F80300A0000200003A8BDC8D00
:1004300010BD000060530000B0910004F8B505F055
:1004400087F90500874801680222114301600168AD
:1004500008231943016083494031CB681343CB60C3
:10046000436813434360CA6840263243CA60CB687E
:1004700080221343CB60016831430160016811435E
:100480000160416831434160416811434160764CED
:1004900020681E2188432060744FF96A2020814320
:1004A000F96204F0A0FF022005F0EFF8000604D581
:1004B0004021272005F026F903E00321092005F05B
:1004C0002CF9A80703D4B86801210843B86068482C
:1004D000C16B0122D2059143C163C16B0322D204D7
:1004E0001143C1630721082005F017F903210720F4
:1004F00005F013F904F0A6FF2068E021884320608E
:1005000060691521884360616069B043606160691A
:1005100001218906884360616069052109078843D4
:100520006061E06953490840E061E06940084000CB
:10053000E061E0691027B843E06104F03FF84E4AFB
:1005400010682021084310604C4A10680421884339
:1005500010604B480D21006889014018016852065F
:1005600011430160A069B043A0616068454908403B
:1005700060606168444801406160A168434A11407D
:10058000A160A1680140A160E168414A1140E160B9
:10059000E1687A039143E160E1680140E160374A34
:1005A0001820C043C03A1168014039431160394AEC
:1005B000A906116803D501400820014301E001406C
:1005C00039431160344801690904090C016141692A
:1005D0000904090C416181690904090C8161E06920
:1005E000012189038843E061E06989008843E06173
:1005F000E06909118843E061E069052109060843C3
:10060000E06104F051F8F8BD10B500F008F8234897
:100610000068002801D0FFF711FF10BD7047124895
:100620000168032212029143016041699CD8E5BA36
:1006300001000000F40500A000020000237302FD89
:1006400042019143416141694200914341618169A5
:10065000C200914381610F480068016F012211437C
:100660000167016F022291430167C0300168D20621
:1006700011430160704700000023008000280080C3
:100680000029008000910090FBFBFFFF0027008005
:10069000403D0080045A00B0DFFFD5FD7FFF7FFFA3
:1006A000D5FDD5FDD5FDD7FDC03C008000220080E2
:1006B000506600B0084810B50168084B0A001031B8
:1006C00008001960111D5960242149F3FEE804490E
:1006D000022002F04DFC10BD34C800B0F85900B043
:1006E000B9380000F8B5002425001C48A7001426DE
:1006F0006643C5511A481421301849F3E6E81848F2
:1007000014211430301849F3E0E81548142128303A
:10071000301849F3DAE8114830222838C159104816
:1007200062433C301018C4608160456185610D49A9
:10073000C56101610C4901620C498562416206F3A1
:10074000EBF8641C012CD0DB0949082001F048F9C2
:100750000849FF20401C8860F8BD0000C86600B052
:1007600064FF00B0253B0000413D00006B3F0000EE
:100770004F410000009000A80F490E4810B50860D6
:100780000F490E48086010490E48086010490F488C
:10079000086011490F4808601048802149F394E827
:1007A0000E488021803049F390E80D48802149F3BC
:1007B0008CE810BD1D1602003CE50004DD4200007F
:1007C00040E500042143000044E500044054890052
:1007D00034E50004A086010038E50004DCCE00B05A
:1007E000DCCF00B010B5084C00206062DF200002B2
:1007F000E0620648A06201210548490249F364E825
:1008000001206062002010BDC09B00A800ADDEEF9B
:100810005CD000B026484068C168264A1143C160D8
:10082000704700B5FFF7F6FF214840684168012294
:100830005202114341604168D2001143C04DA55A94
:1008400001000000F00700A000020000D79BBC40A0
:10085000416000BD090401431A4840688161704746
:1008600018494968CA681204120C00040243CA609D
:100870007047144949684A69120C120402434A61DC
:100880007047090401430F484068C16370470D4930
:1008900049684A68120A120202434A6070470948CE
:1008A0004068FF30413041681D22914341607047EC
:1008B00004484068FF304130416802229143416062
:1008C00070470000005A00B08F0300008FC08FE215
:1008D0001CFF2FE101210920000701600021416078
:1008E00070476848012101600021416070476648F7
:1008F000016B80221143016370477047634800B564
:100900000068002801D0FFF7F2FFFFF7EAFF00BD03
:1009100010B55F4C20F0DAEDA04221D05D490840CF
:10092000040004F074FD262004F0C3FE0109200732
:100930000901000F08430106090E262004F0ABFE52
:1009400004F094FD200A4107534A490F042911700D
:1009500001DD04211170000702D5107840421070AB
:1009600010BDFF20C130202100B504F054FF00BDB0
:1009700010B54A4C207900280BD10120207104F0D9
:1009800060FF062004F095FEC006C00F607104F001
:100990004AFF607910BD70B50600FFF7E9FF404DD2
:1009A0002C0D002811D004F04CFF8021262004F0EB
:1009B000BDFE04F038FFA8682043A860394881686C
:1009C000220211438160002003E0A868A043A860D0
:1009D000300005F08FF870BD10B507F077FA04F01D
:1009E000ECFC02F0C3FE7D24E4010021200004F0B1
:1009F000ECFC0021200004F0EBFC0021200004F0BE
:100A0000EAFC0021200004F0E9FC274C0221200030
:100A100004F0DEFC0221200004F0E0FC234C6068BE
:100A2000234908406060E068172149020843E060FC
:100A300004F0A2FE2168C2061E4801D5014300E071
:100A400081436268626021602168014322E87D1B66
:100A500001000000EC0900A0000200001082BE1D91
:100A600021600F480068002802D0B520FFF79DFFE5
:100A700010BD7047704710B504F049FF0C4C0028BA
:100A800002D005F094F801E005F0A0F8E06010BD98
:100A90000F490E4808607047003000A8400C0090D5
:100AA000506600B0FFFF00003F0F0000005A00B08A
:100AB000C85A00B08028008040230080409C00007D
:100AC00000210080FF7FFF7F000000207F58000092
:100AD0004C5C00B0F8B5324800680002000F0828EE
:100AE00028D1304C6069E5042843606160694000AA
:100AF0004008606120680826304320602068EF12BB
:100B0000B84320604821452004F0CFFD042148204F
:100B100004F0CBFD2068304320602068384320601B
:100B2000322004F0E6FE60692843606160692105B7
:100B300008436061F8BD1C4810B5006800282DD03E
:100B400004F089FEFFF7C6FF2021192004F0F8FD0C
:100B50000221162004F0F4FD2F21332004F0A5FD1E
:100B60000321572004F0A1FD9221242004F09DFDD3
:100B70006221252004F099FD262004F0A4FD8008C0
:100B80008000022108430106090E262004F08DFD95
:100B90006621412004F089FD04F04FFE10BD0000E5
:100BA0000020008000280080506600B070B5444CE2
:100BB000444D2068444E002808D0E817306070602B
:100BC00004F0CEFF286A4000400828623D48C03843
:100BD000816A090C09048162816A8B2292001143A7
:100BE00081623A4900208860900639490122120446
:100BF000036880188842FBD3002001688018904267
:100C0000FBD30120800600682068002855D004F03E
:100C100022FE0F21622004F048FD1021332004F051
:100C20009AFD04F00AFE706B0121C902084370634B
:100C30003068632188433060F06826490840F060DE
:100C400004F0EFFB07210D2004F085FD07211B2098
:100C500004F081FD04211B2004F072FD859A84F9C3
:100C600001000000E80B00A000020000E46A00A000
:100C70004021252004F06EFD4021172004F06AFD7C
:100C8000022004F02AFD400603D540210B2004F089
:100C900061FD04F0FFFB04F083FD800604D4F068DE
:100CA000012189038843F0601048C168104A11404F
:100CB000C160C1680F4A1143C1602068002806D096
:100CC000012040046862801CA8620B48E862002092
:100CD00070BD0000506600B0C09000900021008000
:100CE00000230080000001B0C0FFFF7F802800804B
:100CF000F0F0FFFF0A0A00000202020000B50D49F1
:100D0000002087B00860020001001E2003AB07C36B
:100D100002000948FF21491C6B4607C3A838074A4F
:100D2000002307A103F3EEFB0006000E00D0012014
:100D300007B000BD9C0E0004EC16000443620000E6
:100D400049646C650000000010B5FFF7E9FC06F08F
:100D5000A6FD07F02FFA07F063FA10BD11483C21F9
:100D600010B548F3D0ED0F4800210160416081606B
:100D70008161016201630C4A4163C2620B4C816371
:100D80000B48EE22210048F31AED0948094B0422D2
:100D900021003EF3FEF810BD10B500F00DFB002061
:100DA00010BD00005CD6000477880000DC05000060
:100DB00068100004E3EE3300F8B5C54C20680C253C
:100DC000A8432060C348C168820C1143C160C16858
:100DD000072252021143C160C16801221206114369
:100DE000C160C16889098901C160C168C20D9143B0
:100DF000C160C168C20C9143C160C1685603B14370
:100E0000C160C1680722D2069143C160C168F21077
:100E10001143C1600168B04A114301607D20002187
:100E2000400204F0E6FA7D27FF010021380004F0BB
:100E3000E6FA0021380004F0DFFA0021380004F05F
:100E4000E1FAA649086A1022104308622068A84304
:100E50002060606851068843606004F00FFFA0685E
:100E6000B1000843A0602069A9058843EA2F2AB091
:100E700001000000E40D00A000020000FD92DED0A1
:100E800020612069304320619A4D686800206860C5
:100E9000686819210906084368609648803001682F
:100EA0004026B143016001680F22120291430160A4
:100EB0000168032252021143016001680F221203EC
:100EC00091430160016803225203114301600168EC
:100ED000090909010160016806273943016020689A
:100EE00030432060206830218843206004F052FCA9
:100EF0000528206802D910210843FFE720602868F0
:100F00000121084328602868B84328607648C168F2
:100F1000020D1143C160816A31438162012004F0F6
:100F200048FF012005F09AFAF8BD10B505F0DAFA8D
:100F30007149088071487249000C000408607249C8
:100F400070480860724971480860734971480860C8
:100F5000734972480860744972480860744973485C
:100F60000860754973480860754974480860764997
:100F70007448086076497548086077497548086084
:100F80007749764808607849764808607849774814
:100F900008607949774808607949784808607A4953
:100FA000784808607A49794808607B497948086040
:100FB0007B497A4808607C497A4808607C497B48CC
:100FC00008607C487C4908607D497C4808607E490F
:100FD0007C4808607E497D4808607F497D480860FC
:100FE0007F497E48086080497E48086080497F4884
:100FF000086081497F48086010BD0121080010B5D4
:1010000002F078FD04F0C6FB7C494000085A7C4998
:10101000086000F0FBF90221012002F06BFDFFF7F0
:10102000D5FE0321012002F065FD20F072EA0421C3
:10103000012002F05FFDFF22724919321C2005F3E6
:1010400089FD0521012002F055FD0621012002F055
:1010500051FDFFF76AFF0721012002F04BFD6A49AD
:10106000E1204002086020F058EA0821012002F047
:1010700041FD65490422072020F052EA167204A6B9
:1010800001000000E00F00A000020000097A606D7E
:101090000921012002F038FD614800210A0006C044
:1010A0005F4A60496048614B05F3CDFE0A2101208B
:1010B00002F02AFD00F0C2F90B21012002F024FD0C
:1010C00000F072F90C21012002F01EFD00F0B0F8D2
:1010D0000D21012002F018FD0E21012002F014FD67
:1010E000002010BD10B500F0B9F900F0F3F900F0E0
:1010F0005FF9002010BD0000002F0080002100805B
:1011000000081C200028008080260080C8E8000419
:101110003C7000B0BCEA0004F96200006CE5000419
:10112000458F00005CE500047B8F000060E5000453
:10113000958F000068E500048D8F000064E50004D1
:10114000C11200B098E600040D0F00B09CE6000448
:10115000651100B0A0E60004AB1100B0A4E60004E5
:10116000C71100B0A8E600045DE3000080EC0004B5
:101170006FE3000084EC000481E3000088EC0004CD
:10118000BF1200B0ACE60004AF1A00B0B0E6000435
:10119000591B00B0BCE600048F1B00B0C0E6000481
:1011A000931B00B0C4E6000497DE00008CE6000448
:1011B00067DF000090E60004B3630000F4F600046B
:1011C00015740000BCE5000497580000B4E6000464
:1011D00099580000B8E600049F740000B4E50004CC
:1011E00059740000B8E500048F6E0000B0E50004FB
:1011F000456E0000ACE500049763000084E600043F
:10120000A563000088E60004E763000094E600049C
:10121000000000047CE50004A833000494E5000409
:101220004C5B00B0B81B0000F0170004345900B04C
:101230000449034810B54860080005F08EF810BD59
:101240008B650000705B00B01149104808601249BE
:101250001048086012491148086013491148086095
:101260001349124808601449124808601449134889
:101270000860154913480860154914480860164964
:10128000144808601649154808607047C45C392442
:1012900001000000DC1100A0000200007761C7DD42
:1012A000E76A0000A0F50004E96A000090F5000478
:1012B0001F6B000094F50004256B000098F50004F6
:1012C0004D6B00009CF50004576B0000B0F5000466
:1012D0006F6B0000B4F500049D6B0000A4F50004E2
:1012E000B56B0000A8F50004816B0000B8F50004A0
:1012F0008F6B0000ACF5000410B50124A402204857
:10130000EE22210086B048F378EA11F0F7FE0DF0E6
:10131000DDF9012200210C2003AB07C302001848AD
:1013200002920090174A0019002317A1019403F3B9
:1013300007F900281DD1194815A101F393FE18489B
:101340001A4A4168174881601749016100214161CB
:101350008261174AC161026241621649816205F3E6
:1013600017FB002805D11449112000F075FB002857
:1013700002D0012006B010BD00F0CEFA0020F9E73F
:10138000683C0004B17A00004E66635461736B00E0
:101390004E6663466C6167730000000010410004F4
:1013A000F45B00B010EB00B0AD7A0000A97A000049
:1013B000957A00008B7A0000717A000006490020BF
:1013C00008807047064905480860074905480860D5
:1013D0000749064808607047C0ED00B0158000005E
:1013E00004FD0004EB7F000000FD0004E97F000025
:1013F000FCFC0004084804A1016008A141600C49FC
:101400000A480860704700006D6465765F61697521
:101410007265636F7264000018ED00046D64657698
:101420005F616975706C617900000000DD89000002
:101430009CF8000470B500240B4D04E0401940688E
:1014400000F00AFB641CE00029580029F6D170BDA9
:1014500006488168FF22521C114381608168102276
:1014600011438160704700007C5C00B0009000A8D0
:1014700010490F4810B5086010490F48086011491D
:101480000F480860114910480860FFF7E7FE20F098
:1014900060E800F053FA0F490D4808607F40A88DBE
:1014A00001000000D81300A00002000083897960C9
:1014B0000F490E48086006F3F3FD0F490D48086018
:1014C00010BD00007D64000024F600048564000067
:1014D0001CF600048D64000020F600044F2700B0C5
:1014E00024F50004671600B054F90004591A00B03E
:1014F00058F9000481310100C0FC000475497448AA
:1015000010B50860754974480860764974480860E9
:101510007649754808607749754808607749764884
:1015200008607849764808607849774808607949C2
:10153000774808607949784808607A487849416274
:101540007A4A4164784911607A4A794911607B4A44
:10155000794911607B4A7A4911607C4A7A49116065
:10156000C11D7B4AF9314A617B4A7A4911607C4945
:101570007A4A0A607B4A4A607C4A7B4911607D4A0C
:101580007B4911607D4A7C4911607E4A7C4911602B
:101590007D497E4A116001007D4A80310A61026501
:1015A0007C4A4A6142657C4ACA61C265C2667B4A1E
:1015B00002677B4A0A627B4A4A627C4A7A49116026
:1015C0007C4A7B4911607D4A7B4911607D4A7C4998
:1015D00011607E4A7C4911607E4A7D4911607F4AD4
:1015E0007D4911607F4A7E491160804A7E491160C1
:1015F0007F4901667F49814A41667F491160804980
:101600000162016480497F48086081497F48086021
:101610008149804808608249804808608249814841
:1016200008608349814808608249834802F004FFCA
:101630008349824808608449824808608449834815
:101640000860854983480860854984480860864960
:10165000844808608649854808608749854808604D
:1016600087498648086088498648086088498748CD
:1016700008608949874808608949884808608A491C
:10168000884808608A49894808608B498948086009
:101690008B498A4808608B49012008708B498A4829
:1016A00008608C498A4808608C498B48932A8B0CC7
:1016B00001000000D41500A0000200009A71A710DC
:1016C00008608D498B4808608D498C4808608E49B8
:1016D0008C4808608E498D4808608F498D48886124
:1016E00010BD00000D96000034FD00047B9000004A
:1016F00050F4000449900000C0FB0004B7950000BE
:1017000018F900040596000014F90004D9A8000097
:10171000C8F30004B99A000040FC000431A20000A4
:10172000BCFC000447A100003CFD00040FA4000025
:1017300054F70004BFA4000040EB000447A60000DB
:1017400018F6000441A70000C4FB0004B3A7000082
:10175000E4F60004F5A70000D8FC0004DB9B0000C1
:1017600048FC000413A800002DA8000034F7000472
:10177000DDA90000D8E8000403AA000029AA00009F
:1017800030F5000443AA000004F8000479AA000020
:1017900058F80004FFAA00002CFD0004CFAB0000A5
:1017A000DCFC000461AC00000DB300009FAD000044
:1017B000FBC1000047C20000B9C30000A5B3000090
:1017C0008CF70004BDB3000080F70004F1AD000009
:1017D0002CF7000469B300004CF80004C1C10000FC
:1017E0003CF80004F5B30000ECF400040BB5000075
:1017F0000CF80004D1B6000040F80004DDB600008B
:1018000014F80004F7B600003BB70000DFB9000091
:1018100060F80004C5B80000A5BB0000A4F70004F0
:1018200081BB000094F70004D1BB000098F70004CE
:10183000FDBB0000C0F7000421BC00005CFC0004FC
:1018400021C1000038F700040798017AC051320026
:1018500045C400002CF80004DDC4000098FB00041F
:1018600037C50000C0F600045FC5000030F4000476
:1018700085C50000B0F6000453C3000050F7000413
:1018800081C3000020F800044DC6000024F80004C5
:1018900089C6000044F800049FC60000D4F9000483
:1018A000F3C6000090F40004EFC70000ACF9000498
:1018B0000DC80000A0FB0004FDC70000DCBE9CF6C4
:1018C00001000000D01700A0000200006E9919ADC1
:1018D00058F6000471C800006CFB000493C80000B7
:1018E00048F60004DFC80000A4FC0004C5EA0004B8
:1018F0001DCA0000F8F70004CBCA000068FB000412
:10190000F1CA000078F60004FFCA000024E60004D3
:1019100073CB00008CFC000483CB000084FC00042B
:1019200093CB0000DCF60004EDCB000068E9000476
:10193000054810B50078102804D1044904484C2209
:1019400007F0D0FB10BD0000A50E0004B20E00048D
:10195000E20F00040548064910B50078097800F048
:1019600029F804480068804710BD0000004000AA24
:10197000004000AA74F000040749064808600849BE
:101980000648086008490748086009490748086090
:10199000704700002F8F0000CCF30004D931010004
:1019A000D4F70004E7310100D8F70004F531010055
:1019B000D0F70004064808B502680092054A0649B7
:1019C000130008000C386C3303F378FF08BD0000E7
:1019D000980E0004A02101B0006600B00449054A39
:1019E000497812780120914200D000207047000011
:1019F000000002A9000002A910B51FF0EEEC01F3EF
:101A000055FD002010BD10B50C0001F0DFF8844931
:101A10000860C10702D02100052015E0810702D52A
:101A20002100062010E0410702D5210007200BE02D
:101A3000010702D52100082006E0C00602D52100DA
:101A4000092001E0210000201FF03CED012010BD25
:101A5000F1B5002073490E68734F340005000AE0A9
:101A6000E10706D0A9007A58002A02D00099300078
:101A7000904764086D1C002CF2D1012803D0009916
:101A800000201FF020EDF8BD654910B5486001F059
:101A900024F910BD202800D3FEE7634A80001358C4
:101AA000002B00D0FEE71150002070475F4800680F
:101AB000002800D00120704702688368C1681000C8
:101AC000184770B55A4D6C6AE00703D0DFF01EAAC4
:101AD00001000000CC1900A000020000A9801BF04A
:101AE000FFF2ECEDA81768625748A10706D5202140
:101AF000C16042176A6282680A438260610703D547
:101B0000A96A04229143A96221070AD5A96A082279
:101B10009143A9628021C160D2436A6282680A430C
:101B20008260012070BDF8B5484D2C6BE00702D0F3
:101B3000A81728630440200606D58020C0432863E8
:101B40008020844301F043F8200709D50820C043D2
:101B500028630820844301F038FE082000F0B3FC1D
:101B6000600604D54020C043286340208443A0067B
:101B700006D52020C04328632020844300F06CFE5B
:101B8000600707D5042000F057FF0420C0432863F6
:101B900004208443200407D50126F603300001F019
:101BA00016F8F0432863B4436003400F06D00720C3
:101BB000000421000140C943296384430B2620000F
:101BC00036053040070005D0380000F09DFBF84393
:101BD0002863B443E000400F09D00727BF06260062
:101BE0003E40300000F0F9FAF0432863BC43002C7B
:101BF00006DA0120C00700F01AFB154828630440EC
:101C00001448044205D0200000F076F9200001F0CD
:101C100062FA0D4881680122D20411438160F8BD47
:101C2000094B0122D20410B5DA60FFF77CFF0120D6
:101C300010BD0000380E0004009100A8D816020064
:101C4000A8FD0004009400A8009000A88022008055
:101C5000FFFFFF7F0010000110B503F00AFE00280F
:101C600001D0AC48807D10BDF8B50027AA4D3C00DE
:101C7000E968A8683E0079407840084303D004F33F
:101C800077FF06000C00FFF7E7FF04F093FA1FF060
:101C90007EEB04F090FAE968A8687940084309D01F
:101CA00004F366FFAA68801BEB68A14180185941C4
:101CB000E960A860F8BD10B502F012FC002826D03B
:101CC00002F00DFC95490120C0048860001100F06D
:101CD00075FF93480088002801D102F07792018EA9
:101CE00001000000C81B00A0000200005D68A54DB7
:101CF00051FC02F0BAFC02F094FC02F05BFC01F033
:101D000024FEFFF7B3FF1FF04CEB01F029FE02F0B9
:101D100049FC02F0B3FC02F08DFC02F04CFC02F036
:101D2000E7FB10BDFEB50024250026001FF036FAA3
:101D3000019000F0D4FE002802D1FFF79FFF44E09D
:101D400000F091FC00F008FE00F0F7FE7748006814
:101D5000810702D5C10700D00124010702D5410740
:101D600000D50125810602D5C00600D5012604F064
:101D700097FC009001F09EF9070002D1012001F0CC
:101D8000ADF90120C007807804210840400702D443
:101D900000F04DFC05E0002CCFD0002DCDD0002E62
:101DA000CBD000980028C8D0002FC6D0604CA568C2
:101DB000E017E06001263603300000F012FFFFF765
:101DC00084FF300000F004FFA56001981FF0EAF9DD
:101DD000FEBD10B500F081FC00F00DFE00F0DEFE4F
:101DE000FFF7A0FF10BD10B51FF0D8F90400FEF7F3
:101DF00083FC01F02FFD20001FF0D4F910BD10B5B9
:101E000004001FF0CBF9494A1168214311601FF00B
:101E1000C9F910BD10B503F003FD47494000085A49
:101E2000464B47495843096A0B071B0F47F30CEF12
:101E3000080507060609090B0B06400810BD8008B7
:101E400010BDC00810BD000910BD10B504001FF082
:101E5000A5F9364A1168A14311601FF0A3F910BD1E
:101E6000324A010012680020914300D101207047DE
:101E7000F8B52E4C04F386FE22696369851A9941F0
:101E80000E00E1680091A0686422070047F3CEEEDF
:101E900033002A0047F34CEB009906000025380078
:101EA00069406840084309D10120E560A06004F35F
:101EB00069FE6A1E80185141616120613000F8BDE1
:101EC0001A4800218160C16001614161704710B50D
:101ED00002F022FB10BD70B5040002F01DFB041BD4
:101EE00003F077FD0500174900262000DEEEF3B170
:101EF00001000000C41D00A00002000044907B3DD2
:101F000047F3A2EE33002A0047F31CEB70BDC0007C
:101F100005D50B482C304068002800D0004770479A
:101F20000300012010B5FFF7A5FF002804D0D80159
:101F300002D5002000F0DBFA10BD0000A0020080F6
:101F4000985900B0009000A84A5B00B0000000045F
:101F5000A08601000028008040420F00022910B531
:101F600005D0032903D0042901D0052903D1C14B91
:101F7000FF21491C9960042A05D0052A03D0062AAE
:101F800001D0072A07D1002805D100210A22080024
:101F90000B0004F0DEFB10BD7047052803D2B649E4
:101FA0008000085C7047FF20704710B50C000020CF
:101FB000FFF7F3FFA04201D100F080FA0120FFF704
:101FC000ECFFA04201D100F051FC0220FFF7E5FF39
:101FD000A04201D100F03AFD10BD10B50C00002068
:101FE000FFF7DBFFA04201D100F07CFA0120FFF7F0
:101FF000D4FFA04201D100F03EFC0220FFF7CDFF4C
:10200000A04201D100F027FD10BD042910B507D072
:1020100004DC022904D0032906D101E0052903D1FB
:1020200000F01BFA002800D0012010BD022910B5D5
:1020300005D0032903D0042901D0052901D100F0DE
:10204000B5F910BD022910B505D0032903D0042924
:1020500001D0052901D100F068F910BDFF280BD08F
:10206000854A00218B00D35C834202D10806000E12
:102070007047491C0529F5D3FF207047FF280CD075
:102080007D4A00218B009B185B78834202D1880037
:10209000105C7047491C0529F4D3FF2070470528C0
:1020A00004D275498000401840787047FF2070477F
:1020B000FF280CD0704A00218B00D35C834203D1EF
:1020C0008800801840787047491C0529F4D3FF2008
:1020D0007047FF280CD0684A00218B00D35C8342F4
:1020E00003D18800801880787047491C0529F4D3F3
:1020F000FF207047F7B582B007000E00A6D95FC673
:1021000001000000C01F00A000020000B078C580E0
:102110000C2901D2092F02D3002005B0F0BD002503
:102120005A49A8000A5CBA421ED14418A278B242A9
:102130001AD02806000E3900019001F016FC002884
:1021400012D0A670E07804994007400FC9000843F8
:10215000E07001983200390001F009FC002808D035
:10216000E07802210843E0706D1C052DD8D30120D2
:10217000D3E74648AA00FF2110188170E078400795
:10218000400FE070C8E7F0B5060008003F4F00229E
:1021900004219300FC5CB44209D1DD19EC782300E2
:1021A0000B43002802D02300FB242340EB70521C79
:1021B000052AEED3F0BD354A00218B00D35C834263
:1021C00006D188008018C0784007C017401C7047AF
:1021D000491C0529F1D3002070470020704770B5D5
:1021E00005000C00100002F0B5F9200000F00DFD14
:1021F0002800FFF74DFF022805D0032803D004284C
:1022000001D0052803D1200000F09CF870BD20000B
:10221000FFF787FE70BD10B50400C00005D5012290
:10222000120311040C20FFF7DAFF200105D501226B
:10223000D20211040B20FFF7D2FF600105D5012265
:10224000920211040A20FFF7CAFF10BD0120C0034B
:1022500010B502F079F90120C00700F0CDFC0C4860
:10226000016A80221143016210BD0120C00310B534
:1022700002F070F90120C00700F0C7FC0449086AA9
:1022800080229043086210BD009000A8B05900B0B1
:1022900000280080F3B581B00F000198FFF7E8FE39
:1022A00004000198FFF70EFF06000198FFF71BFFDF
:1022B0000500002C03D0012C01D0022C19D1331FB2
:1022C0000126760547F3D4EC040309090E15102006
:1022D00002F040F90120000509E0202002F03AF95F
:1022E000300004E0802002F035F90120C00500F044
:1022F0009AFC002F1DD10198FFF75DFF002818D030
:102300002B1F47F3B6EC06161616160AD56B750F7B
:1023100001000000BC2100A000020000B8A7345D4D
:1023200004160198FFF763FF01000D2009E00198F2
:10233000FFF75DFF694AA1008918C978CA08010042
:10234000100000F0D2FFFF2201991000FFF741FEBC
:10235000FEBD08000021A7E710B50400C00203D5A8
:1023600001210220FFF7A0FFA00207D501210320D1
:10237000FFF79AFF01210420FFF796FF200203D503
:1023800001210520FFF790FF01200007844205D0BE
:102390004010844202D0401084421AD1FF208206AD
:1023A000A11808D0891804D0C206891804D10C20BD
:1023B00002E00B2000E00A20FFF774FE022805D09F
:1023C000032803D0042801D0052802D10121FFF7FA
:1023D0006BFF10BDF8B504000D0017000800FFF7F3
:1023E0008CFE0600002C03D0012C01D0022C22D13F
:1023F0003B1F01277F0547F346EC04030C0C141E1A
:10240000102002F0ABF8102002F0BAF8012000050D
:102410000FE0202002F0A2F8202002F0B1F83800EE
:1024200007E0802002F09AF8802002F0A9F801204D
:10243000C00500F0EBFB331F47F324EC061D1D1D08
:102440001D0E041D2800FFF7D2FE002801D1012136
:1024500000E000210D200CE02800FFF7C8FE002856
:1024600001D1012100E000211C4AA0008018C078A1
:10247000C00800F03AFFFF2229001000FFF7C1FD5D
:10248000F8BD70B504000020002C03D0012C01D051
:10249000022C20D1124D00222868462104F35FFB54
:1024A000002817D128680022082104F358FB0028CF
:1024B00010D1022C06D0012C04D01FF09EE8002879
:1024C0000AD007E005F0DEFA002803D105F0B6FCDB
:1024D000002801D1002070BD012070BDB05900B0AE
:1024E000800E0004022010B5FFF7CDFC02F01CF8AE
:1024F000002804D0012000F0B0F900F0C0F900215C
:10250000082208000B0004F038F910BD022010B5B5
:10251000FFF793FC10BD70B50020FFF791867E2D6C
:1025200001000000B82300A0000200004C4F8AE028
:1025300052FD04000020FFF7D0FD05000120FFF749
:10254000ACFC8549086A1022104308628349900355
:10255000886002F03FF8082000F06BFB2A002100A1
:102560000020FFF719FD70BD70B51EF03FFE05009D
:102570007B480068C00710D00020FFF7D6FF7D2001
:10258000C00003F038FA002036F3F7FF040002E041
:10259000002036F3F2FFA042FAD028001EF02AFEF7
:1025A00070BD002010B5FFF716FD04000020FFF7F6
:1025B00094FD020021000020FFF762FD10BD10B560
:1025C0001EF014FE040066480068800701D5FFF77E
:1025D000E8FF20001EF00EFE10BD002010B5FFF732
:1025E000FAFC04000020FFF778FD02002100002023
:1025F000FFF729FD002800D0012010BD38B501F0FB
:102600009DFF002826D1401E00905548554C00687B
:10261000C00711D06068401C18D0A068FFF783FC89
:10262000514947F34AEB00906168884201D300208A
:1026300000E0081A009009E0684603F0E4FF002873
:102640000CD000986060FFF76AFCA06021780098C9
:10265000884203D3FFF7C1FF002801D1002038BD15
:10266000012038BD3E4810B50068C00705D0FFF70F
:10267000C5FF002801D0012010BD002010BD0020A2
:1026800010B5FFF7A8FC04000020FFF726FD0200AC
:1026900021000020FFF7E8FC10BD10B5FFF79DFFFB
:1026A000002804D0002004F016F9002801D10020F1
:1026B00010BD012010BD2A4810B5006880070DD458
:1026C0002A480078022809D1FFF7CCFF002805D05E
:1026D000FFF7E3FF002801D0FFF7D1FF10BD70B571
:1026E0000020FFF778FC04000020FFF7F6FC2049EB
:1026F0000500096817204883082000F091FA01F0CE
:1027000061FF01F053FF154901208004C8602A00D1
:1027100021000020FFF75EFC0F48016A1022914360
:1027200001620120FFF793FB70BD0D487D3F30BF74
:1027300001000000B42500A00002000055B754902D
:1027400010B50068C0070FD1FFF762FF00280BD05B
:102750001EF056FD0400FFF75BFF002801D0FFF7D5
:10276000C8FF20001EF050FD10BD000000280080B2
:10277000009000A8985900B0DC5900B0E2040000B5
:102780006C5B00B084EA0004F8B51EF039FDBE4D64
:102790000700286800282ED103F0E9F8402118200E
:1027A00003F05AF803F0D5F8B84E30690221084317
:1027B00040084000306101F0E1FE040001F0DEFE5F
:1027C000A042FBD03069032108433061B04A9068D1
:1027D0000121490688439060AD4A803AD068884319
:1027E000D06003F0C4F80821332003F040F803F070
:1027F000B0F80120286038001EF006FDF8BDF8B5DD
:102800001EF0FEFCA04D00902868012835D103F091
:10281000AEF80821332003F01FF803F09AF89C4922
:102820008039C868012676063043C860984FB8687A
:10283000B043B8609549086902221043400840003F
:10284000086101F09BFE040001F098FEA042FBD05D
:102850000A2003F0DAF8B8683043B8608B49086999
:1028600080088000086103F082F84021182002F0FF
:10287000FEFF03F06EF80020286000981EF0C4FCF4
:10288000F8BD10B504000120FFF7AFFB002C05D107
:1028900080490968CA0705D0490603D5062801D032
:1028A000FFF7F2FC10BD012010B5FFF79EFB0628D4
:1028B00003D001F04DFE0028FBD110BD082010B55B
:1028C000FFF7F5FA10BD082010B5FFF7CAFA10BDE2
:1028D00038B5002000900120FFF787FB040001209D
:1028E000FFF705FC05000420FFF7E1FAFFF787FF7B
:1028F00001F0C0FE202000F0A6F901F08FFE68462E
:1029000005F0C4F80121644A4906002800D0009867
:1029100091602A0021000120FFF748FB38BD10B567
:102920001EF06EFC04005B480068400702D50020E2
:10293000FFF7CEFF20001EF067FC10BD8002761F5F
:1029400001000000B02700A000020000A15FEA2DF6
:10295000012010B5FFF753FB04000120FFF7D1FB66
:10296000020021000120FFF782FB002800D0012097
:1029700010BD08B5684605F08FF8002803D0FFF7B2
:10298000E7FF002801D1002008BD012008BD46480E
:1029900010B50068400705D5FFF7EBFF002801D010
:1029A000012010BD002010BD70B50120FFF727FBEE
:1029B00004000120FFF7A5FB05000020FFF71FFB27
:1029C000A04204D02A0021000120FFF761FB70BD66
:1029D000354810B50068000709D4FFF7D8FF002874
:1029E00005D0FFF7B5FF002801D0FFF7DDFF10BDD0
:1029F00010B501F01DFE03F020F810BD10B501F078
:102A000017FE03F01AF810BD38B500200090012021
:102A1000FFF7F5FA04000120FFF773FB0500202003
:102A200000F012F901F027FE204901204006C8609D
:102A3000684605F035F8002808D101F00BFE05F0D6
:102A400036F800280AD0FFF7A9FE07E00098002812
:102A500002D1FFF7CDFF01E0FFF7D0FF2A002100F0
:102A60000120FFF7CBFA0420FFF705FA38BD0E4826
:102A700010B5006840070FD4FFF77BFF00280BD08C
:102A80001EF0C8FB0400FFF774FF002801D0FFF719
:102A9000BBFF20001EF0C2FB10BD0000E85900B0D3
:102AA0000028008080210080985900B0009000A884
:102AB000202010B5FFF705FA10BD202010B5FFF754
:102AC000DAF910BD70B501F059FE01F073FE01286E
:102AD000FBD10220FFF793FA04000220FFF711FB5D
:102AE00005001020FFF7EDF95549012040048860EA
:102AF00001F032FE042000F0B0F801F01BFE2A00C5
:102B000021000220FFF75CFA4E480068800601D4DD
:102B100001F047FE70BD10B51EF07CFB0400494873
:102B20000068C00602D50020FFF7CCFF20001EF091
:102B300075FB10BD022010B5FFF761FA04000220FA
:102B4000FFF7DFFA020021000220FFF72FCB2C70E5
:102B500001000000AC2900A0000200006646E870F9
:102B600090FA002800D0012010BD10B505F08EF9B4
:102B7000002803D0FFF7E8FF002801D1002010BD96
:102B8000012010BD344810B50068C00605D5FFF718
:102B9000ECFF002801D0012010BD002010BD70B551
:102BA0000220FFF736FA04000220FFF7B4FA05000E
:102BB0000020FFF72EFAA04204D02A0021000220B4
:102BC000FFF770FA70BD244810B50068800609D47C
:102BD000FFF7D8FF002805D0FFF7B6FF002801D087
:102BE000FFF7DDFF10BD70B50220FFF712FA0400F9
:102BF0000220FFF790FA0500042000F02FF801F002
:102C0000ACFD01F0A1FD134901204004C8602A0079
:102C100021000220FFF7FCF91020FFF736F901F040
:102C2000AEFD01F0BEFD70BD0B4810B50068C006DA
:102C30000FD4FFF79AFF00280BD01EF0F5FA04001E
:102C4000FFF793FF002801D0FFF7CDFF20001EF013
:102C5000EFFA10BD009000A8985900B036494A6AB2
:102C600002434A62CA6A0243CA620120704732497B
:102C70004A6A82434A62CA6A8243CA620120704732
:102C80002D4940310868086070472B49C0430863EC
:102C900001207047284B80339969DA6909011209CC
:102CA00009091201002804D00520400701430A2029
:102CB00003E005200007014305200243D961DA61E2
:102CC00070471E48016B022291430163016B402251
:102CD00091430163016B04229143016370471748DC
:102CE000006B810701D500207047400601D5022006
:102CF00070470120704710B502F00BFE002804D089
:102D00000F498869CA0B9043886110BD10B502F065
:102D100000FE002803D00A488069C007C00F10BD1C
:102D200010B502F0F6FD002804D0054880690121A5
:102D30000904084010BD00008022008000210080AE
:102D4000C02A008070B5002402F0E3FD002808D0FE
:102D5000FFF7E6FF002803D1FFF7D8FFE6332396FD
:102D600001000000A82B00A00002000092AE56CD8A
:102D7000002800D001241EF061FA0500002C07D1C4
:102D800002201EF02FFD002802D014490120086007
:102D90000021012001F086FB28001EF053FA0020DC
:102DA00070BDF8B501200E4900F03AFF0B4E00242B
:102DB000361D0127FF0308E02104090C39430120D7
:102DC00000F02EFF70598047641CA5007059002840
:102DD000F2D103F041FF04F0B6FEF8BD506600B03A
:102DE0007F8B0000FF4841680068814201D10120CB
:102DF000704700207047FB4810B541680068012209
:102E000092070B00040093439443A34205D1114061
:102E10001040814201D0012010BD002010BDF249B8
:102E200000204861F14A5060EE4A1060C860704767
:102E3000EC48416801600168EB4841610021C160D4
:102E40007047F8B504000D0016001EF0F7F90700F2
:102E50000021032001F026FB002C0ED0002D0CD009
:102E600032002900200046F352ED032001F03CFB24
:102E700038001EF0E7F90020F8BD38001EF0E2F936
:102E8000FEE7D94810B58068342146F3DCED10BD6B
:102E9000F8B50C000700002600281CD0D24D287879
:102EA000012818D1012C02D11EF0C8F9060000211A
:102EB000032001F0F7FAFFF733FF00280DD0FFF7EA
:102EC000AEFF00202870032001F00EFB012C02D180
:102ED00030001EF0B7F90120F8BD1EF0AFF98446AE
:102EE000FFF789FF002804D060461EF0ABF90020F0
:102EF00013E0E868401CE860BA4800680C21000450
:102F0000000C4143BA480818002105000A000B00D4
:102F10000EC060461EF096F92800002800D1FEE79A
:102F2000FA78082A01D8121D00E00C22390046F375
:102F3000EEECAC4800F045F9AE49886B0122104335
:102F40008863032001F0D0FA012C02D130001EF07A
:102F500079F90020F8BD1CB50024E443A6480122FD
:102F6000032101AB009400F371F901989F3981F1BD
:102F700001000000A42D00A0000200008B5688BDB7
:102F80000028F5D00128F3D100F062F9F0E710B580
:102F90001EF05EF904000021032001F08DFA98482C
:102FA000001D00F018F99849C86BCA0D1043C8639A
:102FB000032001F0A3FA20001EF04EF910BD0028F6
:102FC00010B508D00078012805D1FFF73BFFFFF7C7
:102FD000DEFF002010BD012010BD10B501780429CE
:102FE00001D0012010BD85494A68521C4A60096918
:102FF000002901D0884701E0FFF7C9FF002010BD7C
:103000000EB504216B461970012159700221D97047
:10301000017819714078587178484168491C4160BD
:10302000FFF7B5FF01216846FFF73CFF00200EBD0A
:10303000F0B587B01EF00CF907007548FFF722FEC7
:1030400074490120C0048860C412200001F0C2FA53
:10305000200001F0CBFA6D486F49283001606F49BC
:1030600001616F494160654C0026266101220A20FA
:103070000592020003906B48012189026B46049679
:1030800007C300236148684AA83868A101F3E4FA3D
:10309000002802D0012007B0F0BD5C4865A100F314
:1030A0006DF800210320267001F006FAA068644D37
:1030B0000068A84207D1FFF73DFE00280AD0FFF7BD
:1030C00043FE002806D0FFF7E6FEA0680560FFF784
:1030D000B0FE0DE0FFF7B6FE4948466001206B46A2
:1030E0001874DE742070002104A8FFF7DBFE267040
:1030F000032001F003FA38001EF0AEF80020CAE702
:1031000000290CD005280AD2042802D13B480161CD
:1031100003E03E4A80002832115000207047012011
:10312000704770B5FFF706FE344C002802D000202F
:10313000207014E01EF08CF82F4D060008E0E168C6
:10314000002910D02D48491E1430E16000F043F8EA
:10315000606969688842F2D130001EF07DF83A4912
:103160003848086370BDFEE7234801684068814223
:1031700001D0012000E0002021494A68101BCF64E3
:1031800001000000A02F00A0000200007FBE36005A
:1031900009688A4201D0012100E000210843012191
:1031A0004840704701001E48002210B500F3F2F8B5
:1031B00010BD70B5040016480178012901D0012125
:1031C0000170E0010CD5254925480863CD0D280084
:1031D00001F010FA280001F007FA0120FFF7E2FFE2
:1031E000E00401D5FFF7A7FF70BD026801231104B9
:1031F000090C9B07491C1A4011430A009A43082AEC
:1032000001D359401940016070470000001300C00D
:103210002CC800B0801300C0081300C0802A0080B2
:10322000780401B000100001009000A8252E0000D5
:10323000FF2D0000E32D0000D0FF00B08F2D000017
:103240004963635461736B0049636351466C616702
:1032500073000000CDAB0000FFEFFFFF8022008075
:10326000FFFFFFFEF8B51DF0FDFF144C144E154D89
:1032700007001BE0FFF768FD002803D0124900207B
:10328000087017E070680C230004000C58434019C4
:103290000CD00178052905D28A00A258002A01D055
:1032A000002902D12168884700E0904770683168A2
:1032B0008842DFD138001DF0D9FFF8BDA00401B06D
:1032C000801300C0881300C02CC800B0F8B50400FB
:1032D0000D007648764A0168126801209047002860
:1032E00048D001202700734E0100103F0200A1408A
:1032F000BA40704B4036002D2ED00325082C07D243
:103300001E68620095409040AE4306431E6009E08F
:10331000102C0AD25E68083C620095409040AE4393
:1033200006435E60986888431AE0182C07D2F36958
:1033300079008D408840AB430343F36109E0202CC2
:1033400007D2336A183C61008D408840AB43034389
:103350003362706A904307E0102C03D298680843E8
:10336000986002E0706A1043706253490120096856
:1033700088470120F8BD70B504004C484C4A0D0048
:10338000016812680120904700281AD0A0DD321988
:10339000010000009C3100A00002000001A591B0D6
:1033A0000122102C08DA4849C868A2409043002D39
:1033B00000D01043C8600AE0434B4033986A103C89
:1033C000A24090430100002D00D0114399623F4973
:1033D00001200968884770BD10B504003848394A93
:1033E000016812680120904700281AD00122102C91
:1033F00006D235488168A24011438160006907E028
:1034000031484030416A103CA24011434162C06AD9
:10341000E0402E49C4070968E40F012088472000D6
:1034200010BDFF2010BDF8B52548264A0168126876
:1034300001209047002840D0254801210903C160A0
:103440002148016A20484030C06B0F043F0C000641
:10345000000A074300241F4801261EE04068E200DE
:103460008158002918D010184068320082403A4232
:1034700012D005008847102D06D21349086A320081
:10348000AA409043086207E00F494031C86B103DE5
:103490003200AA409043C863641C0E4801788C42F5
:1034A000DCD30B4881680122120311438160074974
:1034B0000120096888470020F8BD0120F8BD000000
:1034C00038E5000440E500040002009044E50004F3
:1034D000009000A8EC5900B0F8B50025FF4F387DEA
:1034E000012802D97D2000023860787DC00709D00C
:1034F00002F094FE3968884204D2787D400840008A
:1035000001257875787D400731D502F0A3FE7968F2
:103510000400FB26814220D8F868A0421DD805206F
:1035200002F031F8A04218D8052002F02FF8A0428E
:1035300013D8012002F027F8A0420ED8012002F093
:1035400025F8A04209D8022002F01DF8A04204D8B4
:10355000022002F01BF8A04201D9787D04E0787DBA
:10356000C10701D0810702D43040012578752800B9
:10357000F8BD70B51DF080FE0500FFF7ADFF002817
:10358000FBD1D64C607DC00706D002F01BFE0028A0
:1035900002D1012002F079FC607D80077C20F49E3E
:1035A00001000000983300A000020000F54D2F0D2F
:1035B00006D502F014FE002802D1012002F0F1FC31
:1035C000607D400709D502F0E8FD002802D1012006
:1035D00002F096FD607D400706D402F0DEFD002873
:1035E00002D0002002F08CFD607D800706D402F03E
:1035F000F6FD002802D0002002F0D3FC607DC00759
:1036000006D102F0E9FD002802D0002002F047FCBC
:103610006068002101F0B5FFA068002101F0B7FF4C
:10362000607DC00709D120687D210902884201D14F
:10363000012000E0002002F01BFEE068002101F004
:10364000A3FF2069002101F0A5FFAA49002008700E
:1036500028001DF01FFE002070BDF0B506000D0013
:1036600087B0A3490027182201A846F3E2E9A04C3D
:10367000607D000702D4012007B0F0BD002E02DA01
:103680007600760801273300042646F356EB0852ED
:1036900005142044512C385202F0CAFDA84204D22D
:1036A000607D40084000607503E0617D01200143BA
:1036B000617525603DE002F0D7FDA842607D02D231
:1036C000FB21084000E030436075656031E002F0A6
:1036D000CBFDA842607D02D2FB21084000E03043D0
:1036E0006075A56025E002F0BFFDA842607D02D2B2
:1036F000FB21084000E030436075E56019E002F00E
:10370000B3FDA842607D02D2FB21084000E03043B7
:10371000607525610DE0280002F0A2FD0028607DA3
:1037200002D1FD21084001E002210843607500E05C
:1037300025756F49182201A81DF0FAFB002802D058
:103740006C4901200870002F01D0FFF71CFF0020FA
:1037500092E7FEB500207D24E401270001250194B5
:10376000009011F32CFD8821694306000291405C12
:1037700002282FD12804000C1CF389FC0099491C55
:103780000906090E00910279012A02D181790129E5
:1037900004D0029989194B7D092B08D102997D200B
:1037A0008919C9788001002910D1401084CE057094
:1037B00001000000943500A000020000ECB5F17D8E
:1037C0000EE0052A05D18079052802D17D2000026E
:1037D00001E07D20C001C978002901D17D20800150
:1037E000844209D8040007E0012805D17D20C001EA
:1037F0008442F7D92000F5E76D1C082DBBD3009853
:10380000012805D97D200002844200D9200004004F
:103810003E48C06900280BD07D200002844200D9B8
:10382000200004007D20C001874200D93800070035
:103830003748807902280BD17D200002844200D9CC
:10384000200004007D20C001874200D93800070015
:1038500001990120FFF70BFF39000320FFF707FF55
:1038600021000220FFF703FF0020FEBD10B5254C0C
:10387000607D000734D502F0C2FC002802D101208F
:1038800002F019FC02F0B8FC002802D1012002F07D
:10389000D3FB02F0B7FC002802D1012002F08AFC21
:1038A0001C4801680420FFF7E2FEFFF75CFF7D2162
:1038B000490160680C008A00904201D9140011008F
:1038C0000720FFF7D4FE21000620FFF7D0FE0E48A8
:1038D0000078002804D001200021C007FFF7C7FEB0
:1038E00010BD084870B5407D000724D57D24E40153
:1038F000062001F05CFE050002F059FC002811D002
:103900000AE00000C4CE00B0F45900B008D70004AB
:10391000D0D1000494E5000402F0B0FCA04200D332
:1039200020000400A54206D20021200001F033FE51
:1039300007490120087070BD06480822417D1143E7
:10394000417570470348F722417D1140417570472A
:10395000F45900B0C4CE00B0002010B5FEF795FBBE
:1039600004000020FEF713FC0200002021000300E9
:1039700000F08CF80120FEF788FB04000120FEF720
:1039800006FC020021000120002300F07FF8022045
:10399000FEF77BFB04000220FEF7F9FB020021008A
:1039A0000220002300F072F810BDF8B5012633495B
:1039B000334F082A15D0092A43D1002B50C6243C86
:1039C00001000000903700A000020000185D4FC009
:1039D00041D108688C0C2043086001210D20FFF7BD
:1039E0009DFC00210D20FFF7EEFC7869A043786173
:1039F000B869A04322E0002B2DD18200264814187C
:103A0000E078C008192801D3002624E00B680125BE
:103A10002A00824013430B602900FFF77FFCE07807
:103A20000121C008FFF7CFFCE178C808102807D2B1
:103A300079698540A9437961B869A843B8610AE00A
:103A400014484030026B4906090F8D40AA430263B7
:103A5000416BA94341633000F8BD0123AFE7002368
:103A6000ADE70E4810B50068002804D00022110010
:103A7000032002F03DF810BD084810B5006800288A
:103A800004D000220121032002F032F810BD000012
:103A90004023008000020090B05900B048C800B038
:103AA0000A2A10B511D00B2A0FD00C2A0DD1002BE9
:103AB0000BD100210F20FFF731FC0448426981013E
:103AC0008A43426182698A43826110BD000200908C
:103AD0003EB50C2204006F4841686846FFF7EDF9D7
:103AE000A00702D5019805F066FAA00603D56B463B
:103AF000187A05F071FA3EBD10B54078FFF7E8FF7F
:103B0000FFF777FA002010BD3EB5040002E0012067
:103B100001F0D5FFFFF7A2F90028F8D002206B468C
:103B2000187000205C709870D87001216846FFF70B
:103B3000EBF93EBD574808B541680122891C68462B
:103B4000FFF7BBF96B46187808BD10B50400FFF706
:103B5000F1FF002802D12000FFF7D6FF10BD10B5FD
:103B60000C0001004B4824220068FFF7A6F9002C46
:103B700002D02000FFF7E9FF10BD464910B50968E3
:103B80002422FFF79AF910BD01B5424801220068CE
:103B900069460830FFF791F908BD01B53D4801229B
:103BA000006869460930FFF788F90820FFF7CDFF64
:103BB00008BD11B581B0374C0122216868460A3131
:103BC000FFF77BF96B46187819798842C01D0512FA
:103BD000010000008C3900A000020000DF444D9D70
:103BE00008D0206801220A3001A9FFF770F90820E7
:103BF000FFF7B5FF1CBD01B52B48012200686946DF
:103C00000B30FFF764F908BD01B5274801220068B1
:103C100069460C30FFF75BF908BD01B52248012267
:103C2000006869460D30FFF752F908BD13B504224C
:103C30001D4C694620681030FFF749F920680422BE
:103C4000143001A9FFF743F91CBD01B51648012244
:103C5000006869461D30FFF73AF908BD01B5124802
:103C60000122006869461E30FFF731F908BD01B531
:103C70000D480122006869462030FFF728F910201E
:103C8000FFF76DFF08BD084808B541680122684686
:103C9000FFF71DF96B46187808BD034910B5496850
:103CA0000C22FFF714F910BDF85900B0FB4A10B50B
:103CB0001068437804781802F94B2043984203D0E7
:103CC00010680170090A417010BDF4498000091F95
:103CD00008580221593002780A430270F14A507C98
:103CE000084350747047ED48F8B524300188EE4A17
:103CF00091421DD002001288012441889440EB4F6C
:103D0000012904D1FD68A5432C43260003E0FE6889
:103D1000A64334432500E6498088096846F320E835
:103D20008905800A0843FD6001D01DF0FAEBFE60B2
:103D3000F8BDDA4A8000121F105840308183D2E764
:103D400070B50500DB4C09D10022DB48110046F3B9
:103D500059F80028206001D020210181A8002158B5
:103D6000002908D00A898918CC4A121F12581167F5
:103D700020580821017370BD70B50400C068C74D9C
:103D8000012180002D1F285800264166E068800030
:103D900028584666E068800028580B23D83002680F
:103DA0009B021A430260E068800028580823D8303C
:103DB00002681A430260E068800028584B05D8303A
:103DC00002689A430260E06880002858D830026890
:103DD0000A430260E068FFF7B3FFE16865669BAFE6
:103DE00001000000883B00A0000200002BACF32083
:103DF0000720890069580866E068FFF770FFE068EF
:103E0000002802D1296817200866E0688000285839
:103E1000AA498666E068002804D1AB4A08321180BE
:103E200051809180A84A0B0A0E3211705370917024
:103E3000090AD17081000E3A5158002901D00D2194
:103E400000E00C21FFF77FFFE0689F498000091F19
:103E50000E50E0680521820095488258D170E168D3
:103E6000890041588E70E168890041580E71E168FF
:103E7000890040584671002070BDF8B50400142236
:103E8000914F62439248A5003F1F0026032911D19C
:103E9000002C0AD146F322F820213860018101006C
:103EA0002431002002F061FE14E0101846F316F8E9
:103EB00078510FE0052904D1002C08D0844814382B
:103EC000F3E7022901D0082904D1002C2ED146F3B2
:103ED00005F838607859002827D0002C25D138689B
:103EE000734C0189411848780B7802021A43241F49
:103EF0002068C030828248780A7803021343201D6C
:103F00000268D5780122AA40521E9A1803680068F8
:103F1000DB781A418270CA7820688030C2812268BA
:103F20003000D1660221FFF70EFFF8BD684814305B
:103F3000BBE7012270B5D2079378634C80000C3C3C
:103F400022588A422FD0002921500DD00020012272
:103F5000850065598D4204D0461C1500B5401D42B0
:103F600021D1401C0128F3D351480C3802788A42F1
:103F700019D00170514A3630002909D0C1788378B0
:103F80000802184390420ED001F0ADFD012008E078
:103F90004178037808021843904204D001F0A3FD51
:103FA0000020FEF7D1FE70BDFFB581B0040002987D
:103FB00000287BD0E068002878D1029D0498E88032
:103FC00020202881121D2035100A2A7068700020D8
:103FD0000126A8701DF082F90090E0680021FFF72B
:103FE000A8FFE068384F8000083F38589F5440DBF6
:103FF00001000000843D00A00002000032542D505A
:1040000000280ED00498032805D1291D002002F0B5
:10401000D0FD002805D100210B2208000B0002F082
:1040200038FC0498022874D0032821D005285BD0DE
:10403000082817D10320E870E0681421414329487B
:104040000818029945F37DFFE068244A8100121F99
:104050005258002A06D17958002903D10221FFF7CE
:1040600016FF002600981DF047F9300005B0F0BD9E
:10407000FE20E870291D002002F09BFD0028E0686A
:104080000BD01423584317494018029945F37BFF7E
:10409000E16800208900785006E01421414311486E
:1040A0000818029945F34DFFE0680C4A8100121F81
:1040B0005258002AD6D179580029D3D10321CEE70E
:1040C0002FE026E0A86600B0DCFE00008000008043
:1040D000FFFF00000002009044C800B0C46600B0BA
:1040E000B45B00B078FF00B00220E870E0681421F3
:1040F0004143FE480818029945F323FFE068FC4A53
:1041000081005258002AADD179580029AAD1052141
:10411000A5E70420E870E06814235843F3494018E9
:104120008FE70020A2E710B504001DF0E1F8F04A87
:10413000A1001C3AEF4B545863665258172313667C
:10414000EB4B00220C3B5A501DF0D6F810BDFEB5CB
:1041500084000600E64800251C3801590D66025906
:10416000012151660059E24F45663F1D385900282C
:1041700002D045F331FE3D51DC4914227243DC4F3D
:104180000B0014333859D31801930B00143BD31888
:1041900056180028009307D045F31EFE04E03000B7
:1041A00045F3A6FE3851F7E7300045F30AFF002833
:1041B000F5D105E0009845F39BFE385145F30CFE20
:1041C000009845F3FEFE0028F4D105E0019845F380
:1041D0008FFE385145F300FE019845F3F2FE0028AA
:1041E000F4D13D51FEBDF8B504001500C0481C389F
:1041F0000600083E15294DD010DCBD4FB963F853B9
:1042000001000000803F00A000020000C6BC93ED4A
:10421000091F00223F1D0B0045F3CAED11DEDFDF51
:10422000DFCA98DFA3DFAEAEDFDFDFDFAA2ADF0061
:10423000B44812301C293ED009DC17295ED0192958
:104240007ED01A292FD11DF05DF8756129E01D2956
:1042500040D01E294DD0202973D04629F2D1E068E4
:104260000028EFD1A7480068002800D00120F8BD41
:104270001DF048F80500E0688100795800290FD149
:10428000FFF77CFDE06881007958002903D1280000
:104290001DF03CF8EAE7002802D10121FFF767FD95
:1042A00028001DF033F898E0E168890040580221A9
:1042B00080680840F8BD69782A78090211430170C6
:1042C000090A4170E978AA78090211438170090A44
:1042D000C17082E041780278090211432970090A0D
:1042E0006970C178827808021043A870000AE870EB
:1042F00073E0E0680121FFF730FE6EE0814E834AF3
:104300000C3630880F2801D99042AFD1E0680028E0
:1043100063D1A8883080E98871802B899042B3806E
:104320005BD0FFF778F87A4B1A683088012181401A
:104330000A431A600006000E0121FFF717F84CE04F
:1043400000E043E0E068002847D107E0E06800288B
:1043500043D16C490C39096800293ED0FFF7EDFEC6
:104360003BE0E168002938D100681721016634E09C
:10437000E068FFF7F6FE30E0E16800290FD17178C0
:1043800000290CD0634900685E4BC0308182E06830
:104390008000183B18580170090A41707270E0687B
:1043A00081007958002918D00121FFF7E0FC14E0C2
:1043B000E068002811D152481438816814308068B0
:1043C00009184F48143080680818F8BDE0684D4956
:1043D000800008310D5000E035610020F8BDF8B5CF
:1043E0000025A80047491C390A581023566EF2438D
:1043F0001A430B585A6608584030007E002D7ED173
:104400000024F1073FD040073DD43E4910A5D7977F
:10441000010000007C4100A00002000023EBCEEA76
:104420000022091D08680389C418637827781B02D5
:104430003B433E4FBB4204D901212800FFF7A1FCBA
:104440002AE00223037334480021001D0768072275
:1044500008000B0002F031FA0020FFF799FC2E480B
:10446000001D0068002803D001212800FFF789FC07
:104470003889001D3881E078FE2801D10120E070E4
:10448000E078F8802348244928307861E3780831BF
:104490000C6800223900A0470124B00754D51E4FF4
:1044A00000213868002816D001894118091D002014
:1044B00002F089FB002802D00120391F086016484D
:1044C000243801693868002901D0884701E045F3A4
:1044D00097FC00203860230400211B0C06220800F2
:1044E00002F0EBF90B4C200045F37FFD002809D1C9
:1044F000200045F37AFD002804D1200045F375FD26
:10450000002821D00449091F0968002916D00B2270
:104510000EE02DE078FF00B0C06600B0EFFEFFFFB8
:10452000FFFF000040230080DCFE000005040000C7
:10453000002108000B0002F0C0F905E0C088010668
:10454000090E2800FFF7B7FC0C490868006EC0068A
:104550000ED5F0060CD50A00012010321060096853
:10456000072008660021092208000B0002F0A5F9C7
:104570006D1C012D00DA3EE70120F8BDA46600B0F5
:1045800070B505000C0009D102E0012001F0C9FA64
:1045900028001DF095F90028F7D011E0641E2800CE
:1045A0001DF08EF900280BD1012001F0BAFA002C81
:1045B000F4D11249A8000A58521C0A50002070BDBC
:1045C000012070BD0E4B30B501215A6881400A4070
:1045D0008000002A05D1094980310A58521C0A502E
:1045E000FEE7064C803C2258012A02D15D688D43CB
:1045F0005D60521E2250012030BD00005CCF00B033
:10460000C02A008030B500240D4B2200D5005D5932
:10461000002D0ED1D40018510A4B9200B2CA3C9A18
:1046200001000000784300A000020000D70370578B
:10463000D318D96000030321000B890740180749EC
:104640005118086030BD521C042AE9DB012CF9D056
:10465000FEE700005CD000B0C09B00A8009800A856
:10466000FF484068016F1022114301677047FC4802
:104670004068016F10229143016770470020704726
:1046800070477047F6484068816B090C01D00020E4
:104690007047816B490504D5816B0904090FFBD173
:1046A00000E0806B01207047ED484068406B704728
:1046B000EB4949684A6E82434A667047E84949684F
:1046C0004A6E02434A667047E5494968CA6E02432A
:1046D000CA667047E24949688A6E02438A66704733
:1046E000DF484068806B8007C00F7047DC48406837
:1046F000C030416837229143416041680122114333
:1047000041607047D6484068C030416808229143F4
:1047100041607047D2484068C03041680822114368
:1047200041607047CE484068C030016801221143A3
:1047300001607047CA484068C030016849084900B4
:104740000160704770477047C54840684168012262
:104750009204114341608168121191438160FF30DE
:10476000401C41684908490041607047BC484068A6
:10477000C11DF9314A6801231A434A6041689A040D
:104780009143416081681211114381607047B448C0
:104790004068FF30401C41680222914341607047ED
:1047A000AF484068FF30401C41680222114341601D
:1047B0007047AB484068FF30401C0168012211433C
:1047C00001607047A6484068FF30401C01684908F6
:1047D000490001607047A2484068FF30401C0168F2
:1047E00008221143016070479D484068FF30401C1B
:1047F0000168082291430160704799484068C030C1
:1048000001680122D2071143016070479448406853
:10481000C03001684900490801607047904840680D
:10482000FF30401C01680122D2071143FF31EB0128
:1048300001000000744500A000020000CEFBAE277E
:10484000016070478B48406880680003C00F704764
:104850008848406881680122D20411438160704712
:1048600084484068FF304130416A890889004162CC
:10487000704780484068FF304130416A04229143CC
:10488000416270477B484068FF304130416A0422F2
:1048900011434162704777484068FF304130016AF8
:1048A000012211430162704772484068FF30413075
:1048B000016A49084900016270476E484068FF304C
:1048C0004130016A0122D2071143016270476948F1
:1048D0004068FF304130016A490049080162704771
:1048E00064484068FF304130806A0005C00F70475F
:1048F00060484168092080010818C16901229203BB
:104900001143C161C16952001143C161C1695200C3
:104910001143C16170475748416809208001081858
:10492000C169012292031143C161C169520011435F
:10493000C161C16952009143C16170474D484068EF
:10494000816810221143816070474A4841680920FC
:1049500080010818C169012252041143C161C16973
:10496000D2001143C1617047424905224968D20112
:104970008918CA69382340079A43800E0243CA61E6
:10498000C86901221043C86170473A4A0023D356D0
:104990001F21C0181F2800DA01000806000E70470A
:1049A0000D2804D8334900228A56002A00DBECE7A0
:1049B0007047F0B593B0304C2068030960681B0164
:1049C0000109A06809010209E0681201000900015B
:1049D000C01C12902069491C050960692D0100095D
:1049E0000001401D1190A069921C00090001801D6A
:1049F0001090E0692D1D0609206A360100090001AA
:104A000008300F90606AF61D0009000109300E9011
:104A1000A06A000900010A300D90E06A0009000157
:104A20000B300C90206B000900010C300B90606B78
:104A30000709A06B3F01000900010D3072B29A9482
:104A400001000000704700A0000200003A13109A15
:104A50000A90E06B0D37000900010D308646F0200A
:104A60008143103109911299854340350895119D74
:104A70008243814320323031854350350795109D64
:104A800083438543944603E0005A00B05CD200B0F3
:104A9000503506950F9D0C9A8543503505950E9D12
:104AA00082438543503504950D9D503285435035E2
:104AB00003950B9D02928543503501950A9D7246E0
:104AC000854382438643874350351F20000200956B
:104AD000132583432D025B192360099B8143834384
:104AE0005B196360634683435B194919A360E16006
:104AF000089D50320B218543490296466A1822616F
:104B0000079D503685436A186261069D864385433A
:104B10006918A1610321C9027218E261059D50372D
:104B200085436A182262049D874385436A1862623E
:104B3000039D85436A18A262029A82435218E26278
:104B4000019D85436A1822637A186263009D85433C
:104B50006A18A26372468243511800250700E16378
:104B6000AE00A059C004C00EFFF719FFA159C0063E
:104B7000C00CB9436D1C01432D062D0E102DA15103
:104B8000EED313B0F0BDF0B588B0FF490A6A120643
:104B9000130F4A6A1206120F120113438A6A120691
:104BA000120F12021343CA6A1206120F12031343A2
:104BB0000A6B1206120F120413434A6B1206120FED
:104BC000120513438A6BC96B1206120F09061206EF
:104BD000090F134309070B43EC494A68D11DFF3104
:104BE000FA310C690B610C6B0B630924A4011219D7
:104BF000D468D360E44BDC682406260F04969C68D6
:104C000035012406240F03942C431D692D062E0F15
:104C1000350237032C43059700962600A6465C69AB
:104C20003E432406240F0194240426430694019C49
:104C300027059C693E432406240F2506DC692E4384
:104C40002406240F2407264302960796798E1F59BF
:104C5000010000006C4900A000020000FD0A12C71C
:104C60005B68BC461B061F0F039B1E013B003343C2
:104C7000049E059F36023343009E3B4336041E4389
:104C800067463E432E432643072803D0062801D01B
:104C90000A2809D1906802989060C8680798C8608F
:104CA000C86ACE6208B0F0BD0528FBD19068019EAD
:104CB000704636033043069E3043664630432843F1
:104CC00020439060CA68C860C86A0698034360467B
:104CD00003432B432343CB62E4E7F0B5AF480168BD
:104CE000426809071207090F120E11438268036B0D
:104CF0001207120D1143C2681207120C1143026908
:104D00001207120B114342691207120A11438269FA
:104D1000120712091143C2699446120711439646BD
:104D2000026A1407426A240F1207120E1443826AA1
:104D30001207120D1443C26A1207120C14431A0709
:104D4000120F15042C43456B26002D072D0A2E4308
:104D5000856BC06B2D072D092E4300070643904835
:104D60004568E81DFF30FA30476841608768866013
:104D700016053443120614431A07144309229201FC
:104D8000AA18136811605368546062461207120F24
:104D90001301134314022343140323431404234332
:104DA000140523431206134372461343426A4162B9
:104DB000816A8362F0BDF0B5784908684A69C00429
:104DC000C50E4868D204C004C00E4001054388687F
:104DD000D20EC004C00E80020543C8685206C0044B
:104DE000C00EC00305430869CB69C004C00E0405AA
:104DF000254315438A69DB04D204DB0ED20E5B0126
:104E00001A430B6AAC46DB04DB0E9B021A434B6A67
:104E10004D6BDB04DB0EDB031A438B6AED04DB0412
:104E2000DB0E1B051A43CB6AED0EDB04DB0E5B06C3
:104E30001A430B6B6D01DB04DB0E2B438D6BC96BCF
:104E4000ED04ED0EAD022B43C904C90E4701060067
:104E50003E4387023E43C7033E4326431B396C0E45
:104E600001000000684B00A00002000009E2AC7ADB
:104E70004006064348010C000443880204434D48A1
:104E8000CD0340682B430100FF302C43FF30801CD2
:104E900045696546456187698261C769C361436B3E
:104EA00033004663866B8363C66BC36308000921C6
:104EB0008901401801690561416942618169846124
:104EC000F0BD10B50400FFF712FF2000FFF76FFEE2
:104ED000FFF77BFF10BD37494968FF31FF31891C5F
:104EE0000A6A000712091201000F02430A62086AE7
:104EF0000F2212039043086270472E494968FF3120
:104F0000FF31891C0A6AF02300079A43000E02430E
:104F10000A62086A1A0390430862704730B50400B9
:104F2000244D04280CD21120FFF758FD696809228E
:104F300092018918C9698904C90E884200D20424E3
:104F40006868FF30FF30801C016A0F221202914313
:104F50002207120D1143016230BD164A10B5536885
:104F60000522D2019A1813691F246406C006A343C0
:104F700080080343136110696311C9069843C90986
:104F80000843106110BD0B4A10B553680522D201C9
:104F90009A1813691F24E403C006A343000B0343BC
:104FA000136110696311C9069843490C084303E073
:104FB0005CD200B0005A00B0106110BDF94A10B5C3
:104FC00052680523DB01D21813691F246401C0064F
:104FD000A343800D034313611069C90640094001D2
:104FE000C90E0843106110BDEE4A10B55268052382
:104FF000DB01D21853691F246401C006A343800D4E
:10500000034353615069C90640094001C90E084372
:10501000506110BD0C2010B5FFF7D5FC0400112025
:10502000FFF7D1FC2100FFF7DFFF1220FFF7CBFCD9
:1050300004001320FFF7C7FC2100FFF78EFF1420A8
:10504000FFF7C1FC04001620FFF7BDFC2100FFF7AD
:105050009AFF1720FFF7B7FC04001920FFF7B3FCF5
:105060002100FFF7ABFF10BDCE49052277A994DCE4
:1050700001000000644D00A000020000101A720A36
:105080004968D20189180A699205D20E824206D374
:105090000A69D206D20E824201D8082070470A69F6
:1050A0001203D20E824206D30A695204D20E824201
:1050B00001D8042070470A699200D20E824206D3BA
:1050C0000A69D201D20E824201D8022070474A6991
:1050D0009205D20E824206D34969C906C90E8142A1
:1050E00001D80120704700207047B34949688031DA
:1050F000CA6AFF23E13300079A43C00D0243CA6224
:105100007047AD4900B549688031CA6AC306520983
:105110005201DB0E1A43CA62FFF7B0FF0006000E11
:10512000FFF7E3FF00BDA4494968C0314A69FF2386
:10513000E13300079A43C00D02434A6170479E491C
:1051400000B54968C0314A69C30652095201DB0EF5
:105150001A434A61FFF792FF0006000EFFF7E3FFD4
:1051600000BD95494968FF3141314A6BFF23E13366
:1051700000079A43C00D02434A6370478E4900B549
:105180004968FF3141314A6BC30652095201DB0EB7
:105190001A434A63FFF772FF0006000EFFF7E1FFB4
:1051A00000BD85494968FF31491C4A69FF23E13345
:1051B00000079A43C00D02434A6170477E4900B51B
:1051C0004968FF31491C4A69C30652095201DB0E86
:1051D0001A434A61FFF752FF0006000EFFF7E1FF96
:1051E00000BD75494968FF31FF31891C0A6A0F23E8
:1051F0005B0600079A43C00802430A6270476E4983
:1052000000B54968FF31FF31891C0A6A1F231B055D
:105210009A43C306DB091A430A62FFF72FFF000611
:10522000000EFFF7DEFF00BD70B505000D20FFF793
:10523000DFFB61494E68092189017118CA6992042E
:10524000D20E904201D2012200E000225A480024EE
:10525000401C035DAB4204D0641C2406240E022CC7
:10526000F7D3086A18255543534A000C0004083246
:10527000535B18430862486A000C0004D91C8687F7
:1052800001000000604F00A000020000E4F2CCB773
:10529000AA18538818434862886A9388000C00044F
:1052A00018438862C86AD388000C00041843C86297
:1052B000086B1389000C000418430863486B53897A
:1052C000000C000418434863886B9389000C0004A9
:1052D00018438863C86BD389000C00041843C86363
:1052E0000520C00130180368168A1B0C1B043343C9
:1052F00003604368568A1B0C1B0433434360836876
:10530000968A1B0C1B0433438360C368D28A1B0C30
:105310001B041343C36030232C4A634338329A186A
:10532000535B0C6A1B042404240C23430B625219A4
:1053300053884C6A1B042404240C23434B62938837
:105340008C6A1B042404240C23438B62D388CC6A0C
:105350001B042404240C2343CB6213890C6B1B0411
:105360002404240C23430B6353894C6B1B04240437
:10537000240C23434B6393898C6B1B042404240C5F
:1053800023438B63D389CC6B1B042404240C234359
:10539000CB63118A036809041B041B0C19430160C9
:1053A000518A436809041B041B0C19434160918A0C
:1053B000836809041B041B0C19438160D18AC268ED
:1053C00009041204120C1143C16070BD005A00B0F0
:1053D00055494A68092189015118CA691F235B028E
:1053E000C0069A43800C0243CA61C8690122920434
:1053F0009043C86170474C494968C0314A690F23DE
:105400009B0300079A43800B02434A617047464959
:1054100000B54968C0314A691F235B029A43C3063D
:105420009B0C1A434A61FFF733FE0006000EFFF79C
:10543000E2FF00BD3C494A68092189015118CA6947
:10544000FF23E13300079A43C00D0243CA6170474E
:10545000354900B54A68092189015118CA69C3064E
:1054600052095201DB0E1A43CA61FFF711FE000612
:10547000000EFFF7DFFF00BD10B504000D20FFF7A1
:10548000C1FAFFF7A5FF1620FFF7B1FA13C8512E96
:10549000010000005C5100A0000200009AE96B07C7
:1054A000FFF7C1FEE00614D50120C007C07CC1078C
:1054B0000FD00007400F02282AD0032809D1162058
:1054C000FFF7AAFAFFF78EFF1620FFF79AFAFFF709
:1054D000AAFE1620FFF795FAFFF7C4FF1620FFF784
:1054E00090FAFFF79EFF1820FFF78BFAFFF71DFEDB
:1054F0001620FFF786FAFFF736FE1620FFF781FA2F
:10550000FFF750FE1620FFF77CFAFFF76BFE10BD89
:105510001120FFF781FAFFF765FFDAE70848816895
:1055200001221207914381608168C2059143816025
:10553000816852109143816070470000005A00B0AA
:10554000802A008070B506000C0015001BF034FFA7
:10555000604A31018918002D03D0002C06D1091DA5
:1055600004E0002C01D0083100E00C310C681BF085
:1055700027FF200070BDFFB585B014000D001E0090
:105580001BF01AFF01905348290108180100083147
:105590000F1D002E049105D0002C01D0010006E063
:1055A000011D04E0002C01D0049900E03900494BB2
:1055B00009681A0060329646121D0392121D944625
:1055C000121D002E029204D0002C724605D1039ABF
:1055D00003E0002C624600D1029A059B1268150078
:1055E000002E03D0002C06D1001D04E0002C01D0B9
:1055F000049800E0380003600598904202D9059DA8
:10560000012727E0914244D10598814241D9314B8D
:10561000012700252800002E08D0002C02D001010F
:10562000C9180CE00101C918091D08E0002C03D0BD
:105630000101C918083102E00101C9180C310968DB
:10564000A94200D90D00401C0628E4DB954220D079
:10565000002F1ED0002E04D0002C704605D10398D8
:1056600003E0002C604600D10298002F056010D0A6
:10567000002C09D0002E03D0280000F078FA08E0B2
:10568000280002F0F8FD04E0002E02D0280002F00D
:10569000D9FD01981BF094FE280009B05DF1027855
:1056A00001000000585300A0000200006E01D5BAAE
:1056B000F0BD0E4810B50068002801D0FFF738FF94
:1056C00010BD0122130060E7012200235DE70022E4
:1056D00001235AE70022130057E7012211003BE79C
:1056E0000022012138E700009CD200B0506600B0D3
:1056F00010B502F0BDFE10BDF949FF22C832888BFB
:105700001042FCD17047F8B5F64C6069002802D011
:105710001BF05CFEFEE71BF059FE606100210120DA
:10572000FEF788FF002810D0EF4EB48801208002D9
:105730000440B088EC4D3527A0433F012035B842E6
:1057400004D1287D012108432875F8BD022000F00E
:105750001CFB0028F9D03C43B480297D0120014383
:105760002975F8BDDF4810B5446900214161FF216A
:105770000170DD482030017D490849000175012094
:10578000FEF77AFF20001BF025FE10BD70B5D54C4A
:105790006069002802D01BF019FEFEE71BF016FE20
:1057A000606100210120FEF745FF00280DD0CE4D9D
:1057B000AC88012080020440A888A04305D00120C5
:1057C00000F0E3FA002800D0AC8070BDC54810B5E9
:1057D000446900214161FF2101700120FEF74CFF67
:1057E00020001BF0F7FD10BD70B5BE4E706900289B
:1057F00002D01BF0EBFDFEE71BF0E8FD706100211D
:105800000120FEF717FF002814D0B74DAC88012007
:1058100080020440A888A04382280BD02888F0800A
:10582000002000F0B2FA002804D0A888308182203D
:105830000443AC8070BDAB4810B5AB4902894469E4
:105840008A80C2880A8000214161FF210170012005
:10585000FEF712FF20001BF0BDFD10BD70B5A14D7D
:105860006869002802D01BF0B1FDFEE71BF0AEFD19
:10587000686100210120FEF7DDFE00281BD09A4E52
:10588000B488012080020440B088A043022812D0CE
:10589000FDF7F7FA002803D0012803D13F2002E0EA
:1058A0001A2000E07F203188E98030809AB47D7E24
:1058B00001000000545500A00002000077F90BCA57
:1058C000B088288102200443B48070BD8A4810B596
:1058D0008A49028944698A80C2880A80002141611C
:1058E000FF2101700120FEF7D1FE20001BF07CFD9E
:1058F00010BD70B5804C6069002802D01BF070FDAF
:10590000FEE71BF06DFD7B4D6061AC8801208002DD
:105910000440A8887A4EA043B04206D0042000F08C
:105920003EFA002801D03443AC8070BD724910B5F6
:10593000486900224A61FF220A701BF055FD10BD24
:1059400070B56D4C6069002802D01BF049FDFEE780
:105950001BF046FD606100210120FEF775FE002866
:1059600010D0644DAC88012080020440A888654EA8
:10597000A043B04206D0042000F011FA002801D064
:105980003443AC8070BD5C4810B54469002141616E
:10599000FF2101700120FEF779FE20001BF024FD9D
:1059A00010BD70B505000E0002F06CFD534C2034A4
:1059B000258102F067FDA68002F064FD70BD70B520
:1059C000050002F05FFD4D4C2034258102F05AFDA8
:1059D000207970BD30B505000C00FFF797FE454BF0
:1059E00020331D81FFF792FE9C80FFF78FFE30BDB4
:1059F00030B505000C00FFF789FE3E4B20331D81BA
:105A0000FFF784FE9C80FFF781FE30BD10B50400D7
:105A1000FFF77CFE374B20331C81FFF777FE988819
:105A200010BD10B50400FFF771FE324B20331C810E
:105A3000FFF76CFE187910BD70B504000D00FFF77C
:105A4000BEFF284301002000FFF7ABFF70BD70B51B
:105A500004000D00FFF7B3FFA84301002000FFF78B
:105A6000A0FF70BD24484178002909D12649096862
:105A7000012209024270090F02002032515C81703C
:105A8000807870471C4910B5C878002815D1086186
:105A90001D4840680A008007800F1032102301243F
:105AA000002807D0012803D0022803D0032803D1FF
:105AB000136001E030201060CC700869E7758759E9
:105AC00001000000505700A0000200008311B577CC
:105AD00010BD1248803000880006000E704700B5E7
:105AE000FFF7F7FF022805D10C4840688007800FB8
:105AF000012800D0002000BD094B5968382291438D
:105B00001040084358607047003800A8C85A00B0D9
:105B10000008009050530000501300000020008047
:105B200000290080A84B59680F2292019143104030
:105B300008435860E7E710B50C00FFF7F3FF2000BB
:105B4000FFF7DAFF10BDA14810B54469002141619B
:105B5000FF2101700120FEF7A3FD20001BF04EFC89
:105B600010BD70B5994C6069002802D01BF042FC52
:105B7000FEE71BF03FFC606100210120FEF76EFD97
:105B8000002811D0924DAC88012080020440A888E2
:105B9000B526A0433601B04206D0022000F009F934
:105BA000002801D03443AC8070BD10B502F043FB37
:105BB00010BD8848C16889008908C160C168032296
:105BC00092071143C160810C7F4880304161824956
:105BD0000161824941610521016194E7804800B576
:105BE0000068002801D0FFF7E4FF7E491620C86056
:105BF00048607D488168C2051143816000BD7B49D2
:105C000010B5096844F342E98905800A084301D0C8
:105C10001BF01CED10BD76E775E7754800680007BE
:105C200001D501206FE700206DE76848C0686AE78A
:105C3000F7B586B004000D001BF0DCFB00900021DE
:105C40000120FEF70BFD002854D00321620008005C
:105C5000904004902000083840000E0086400390D9
:105C600020001038059242000B009340029222005F
:105C7000183A520091408E4601210F00874001934F
:105C80005C480B00A34094465A4A4030002D39D05E
:105C9000082C04D21568049EB543156012E0102C40
:105CA00003D25568B54355600CE0182C04D2C56981
:105CB000019EB543C56105E0202C03D2056A7646F6
:105CC000B5430562089D002D15D0102CF5B1CB927F
:105CD000010000004C5900A0000200004408B72A4F
:105CE00003D294681C43946002E0426A3A434262E1
:105CF000826802231A4382603F4A80325068DB0583
:105D0000184350603E48416055E03B4A803210687D
:105D10000821884310604EE0082C09D21668059DC2
:105D2000AC46049DAE436546A9400E43166021E093
:105D3000102C0AD25568AC46039DAE466546B54365
:105D40007646B1400D43556014E0182C09D2C6695F
:105D5000029DAC46019DAE436546A9400E43C66117
:105D600008E0202C06D2056A7646B5436646B14067
:105D70000D4305620899002917D0102C03D29168B1
:105D80009943916002E0416AB9434162816802220D
:105D900091438160184A8032506801210906884386
:105DA000506017490020486005E0134980310868B9
:105DB0000822104308600120FEF77CFC00981BF0CD
:105DC00027FB09B0F0BD10210A2803D20449400086
:105DD0003031095A0348018001209EE600290080E5
:105DE000C85A00B000080090002A0080170000FF89
:105DF00010200000506600B0C0220080009100A872
:105E000044C800B00020008000020090044903480C
:105E100008600449001F007808707047085B00B0F4
:105E2000F05900B0EC5900B070B505002924FFF717
:105E3000A2FE2000FFF7D7FD29002000FFF7C5FDD7
:105E4000FFF78BFE70BD704710B50400FFF793FE9F
:105E5000002C0AD0FFF72AFE000706D42C211920B7
:105E6000FFF7B3FDFFF779FE10BDEE211920FFF714
:105E7000ACFD60211A20FFF7A8FD6C212820EFE778
:105E800010B5FFF703FE052806D0062806D00A281D
:105E900006D17D21090205E0324903E0324901E0E3
:105EA0000121C903314A93681B041B0C09041943DF
:105EB0009160916802231943916091680424214301
:105EC0009160072802D190689843906010BD01202E
:105ED00010B5FFF7B9FF26480168C20BFBCDBF30F4
:105EE00001000000485B00A000020000B0E009973C
:105EF000114301600168490849000160000C10BDB0
:105F000070B5FAF7D9FE1F49CA0B0028086805D0FA
:105F10001043086008680122104304E01043086041
:105F200008684008400008600020FFF797FF144C05
:105F3000403CA06B21050843A063A06BC910084337
:105F4000A063A56BFFF7ACFD052805D0062805D09A
:105F50000A2805D10C4804E00C4802E00C4800E097
:105F60000C48290E09060143A1630B490868022267
:105F700010430860080C70BD143B0000AB7A0000B1
:105F800040210080002800808509040020DF0300F4
:105F9000705E040068310400002C008070B5FFF7CB
:105FA0007FFDFC4BC1005A58FB4814010DD4C46856
:105FB000FA4D2C40C4604468A400C46802D5012591
:105FC0002C4301E064086400C46044683D25AD06CC
:105FD0002C40AA43144344608268CB185B68920E3D
:105FE00092069B019B091A43826043680122920634
:105FF00013434360836813438360E648E84A843070
:106000004358D36008184068906070BD10B5FFF722
:1060100047FDE44AD16AE44B80001940DD4B583318
:106020001858E14BDB4318400143D16210BDFEB567
:106030000400002001901BF0F1F9DC4E0090B068E4
:10604000844237D0F069002804D0002C02D101200E
:1060500001902FE0D64F3D6A1020054007D1386AE5
:106060001021084338627D20C000FFF7DCFDFFF7F8
:1060700095FFC948012241685207002C07D01143FF
:106080004160C16801221143C160B2600CE09143DC
:106090004160C16849084900C16041680122920617
:1060A000914341600020B060002D03D1386A102177
:1060B0008843386200981BF0B5F90198FEBDFEB523
:1060C0000500002001901BF0A9F9B84F0090F86876
:1060D000854229D0F869002804D0002D02D1012082
:1060E000019021E0B34C266A012000068BEC4C4F56
:1060F00001000000445D00A000020000A918D7E7DD
:10610000064008D1206A01210906084320627D204B
:10611000C000FFF792FD216A0820002D03D0014343
:106120002162012002E0814321620020002EF860FC
:1061300004D1216A012000068143216200981BF0EE
:106140007BF90198FEBDF8B5002506001BF070F93B
:106150009B4C00902069864231D0E16996489B4F64
:10616000002903D0002E03D1012528E0002E19D0EC
:10617000416A012631434162FFF79CFC944940008B
:10618000085A642358430009F8627D21C90043F38B
:10619000B6EE3100002800D001003963A6616661C7
:1061A00026610CE0416A4908490041627D20800176
:1061B000F862082038630020A061606120610098C7
:1061C0001BF03AF92800F8BDF8B5040000251BF0D3
:1061D0002FF97B4E07007069844223D0F0690028B4
:1061E00001D0002C07D0B369734802214022002B54
:1061F00003D1002C1BD0012514E0002C17D0040083
:10620000806A0843A062A06A1043A062FFF752FCB4
:10621000062805D9A06A3C2188431C210843A062B6
:106220000120706138001BF007F92800F8BD836A6F
:1062300093438362826A04239A438262826A8A4316
:1062400082620020EDE7F8B5040000251BF0F0F8AD
:106250005B4E0700B06984421FD0F069002801D06E
:10626000002C04D07069002803D0002C01D1012536
:1062700013E0FFF7D5FE5048816AC20C002C04D011
:10628000114381620120B06107E0914381620021E6
:10629000B161C16A04229143C16238001BF0CCF89D
:1062A0002800F8BDF8B5040000261BF0C1F8444FE3
:1062B0000090F86984423DD0B8683F4D00280BD06B
:1062C000F868002808D03869002805D078690028C7
:1062D00002D0B869002803D1002C13D0012629E090
:1062E000002C0FD0A8690F2109040322884352040F
:1062F0008018A861286A884380182862B436B8C616
:1063000001000000405F00A0000200005DF0695A3B
:10631000FEF732FA01200CE0FEF735FAA869000911
:106320000001801CA861286A00090001C01C2862C5
:106330000020F8610620FFF70CFA01F0A4FF062008
:10634000FFF70AFA01F0DDFF00981BF07FF830003C
:10635000F8BD2048C069704770B5040000251BF0E7
:1063600071F80600FEF7F0FA002801D0002C0AD1DF
:10637000FEF7EAFA204306D01648C06901E0FEF7AE
:106380003BFA0028FBD030001BF060F8280070BDFD
:106390001048806870470F48006970470D48406991
:1063A00070470C488069704710B50024FEF7CCFA9E
:1063B000002800D00124200010BD0000500000047F
:1063C000002F00800300FCFF802600800021008059
:1063D000F9FF0000285B00B000280080403D0080ED
:1063E000009400A80000000470B51D4C206800282F
:1063F00011D1FFF769FB0500FFF766FB1949400063
:10640000085A194AE900515864235843C90F491CD6
:1064100043F37EED206070BD114901204860704754
:1064200010B501F087FFC7E770B5040000251BF029
:1064300009F80B49896800290DD10C490C220B6819
:10644000002C06D093430B600A6804231A430A60A9
:1064500001E093430B601AF0F9FF280070BD0000C3
:10646000285B00B00000000450000004002F0080F2
:1064700070477047F8B58A48017801297ED001211C
:1064800001701AF0DFFF00908648422143F3DEEBF3
:106490000121844AC90700200B781354491C401C71
:1064A0000A28F9DB804900200B781418491C401C8D
:1064B0000B28A372F8DB7C4890380178517501797C
:1064C00091754179D175017A1176417A5176017BC6
:1064D0009176407B7449D076803900200B7814186F
:1064E000491C401C0A282377F8DB6F4950390A7E83
:1064F0006C48203082710A7FC271497F01726A49FB
:1065000030390A7842724A7882728A784EA30FD85C
:10651000010000003C6100A000020000552F988798
:10652000C2720A7902734A7942738A7982730A7A4B
:10653000C2734A7A02748A7A42740A7B82744A7BF2
:10654000C2748A7B0275CA7B42750A7C82754A7C5A
:10655000C2758A7C0276C97C4176584930310A7806
:1065600082764A78C2760A7902774A794277544A23
:10657000137C8377927CC2770A7F20300270497F38
:1065800041704E4E042010368446B078EE2800E06C
:106590003EE0FAD16046F070FF20B07000222FE09C
:1065A000B078EE28FCD10C245443464B1959F170B5
:1065B000080A3071080C7071080EB071FF20B070BD
:1065C000002903D1B078FE28FCD11BE03B4FE51831
:1065D00069681A37B078EE28FCD1384813300B7848
:1065E0000370491C401CB842F9D9364B68681B59E6
:1065F000C01888420DD8287AB070521C1206120EAC
:106600006245CDD300981AF02BFF2A480021017073
:10661000F8BDFF20B070DDE7284810308078EE2804
:1066200000D131E7704770B5FBF73BFD26480022EB
:1066300000680D2100F3D3FB0120FDF7E0FB234DA3
:106640002C6804E06068002800D080472468002C93
:10665000F8D1FFF7E1FFFBF71AFDF1E71C4810B591
:10666000FEF2C6FA10BD10B5134C203C6360E26028
:10667000A16020601BF0A4E820611BF0B2E860611B
:106680001BF0BEE8A0611BF0CCE8E061FEE710B5AE
:1066900004001AF0E1FE0D4B19680A0000E00968D9
:1066A000002902D0A142FAD101E022601C601AF058
:1066B000D7FE10BD485B00B02CD300B09002008024
:1066C000800000802C010004800E00049C0E000459
:1066D00044160004004870470C1D0F0A704770B53F
:1066E0007D240500010024022000FFF730F8290076
:1066F0002000FFF72FF829002000FFF72EF82900CF
:106700002000FFF72DF870BD10B504000100002037
:10671000FFF71DF821000020FFF71CF8F2C50F8ECF
:1067200001000000386300A000020000A1C7263A63
:1067300021000020FFF71BF821000020FFF71AF8C6
:1067400010BD0120D5E70120E8E7414A002010B53F
:1067500004000C21414389180B7A002B03D04968AF
:10676000A14200D90C00401C0228F2DB05212000C8
:10677000FEF7F7FF05212000FEF7F6FF05212000B8
:10678000FEF7F5FF05212000FEF7F4FF10BD0C23F6
:1067900058432F4A012180180172D6E70C23584331
:1067A0002B4A002180180172CFE72A4909784172EB
:1067B000294909784181704770B50124002800D02B
:1067C000264C274DA868A043A8600220FFF753FA83
:1067D000A8682043A8602348FFF74DFA70BDF8B5BC
:1067E0000125AD05204C214E214F012815D16068AF
:1067F0006900884360606068284360603068018C8D
:10680000E20D1143018400F35BFC3868C18A220C5D
:106810001143C18200F360FCF8BD00F351FC3868FD
:10682000C18A4904490CC18200F356FC3068018CCE
:10683000FF22521C914301846068A8436060F8BD48
:1068400010B5FFF751FF7321000E0902401810BD6B
:10685000545B00B0A1E50004A0E5000401000004C1
:1068600080210080DC0500004023008064EA0004F1
:1068700034EA000410B537F3A5FB10BD10B537F3AB
:1068800064FB10BD704710B504000020C0432060B9
:1068900046488079042805D003281AD1002024F323
:1068A00045F9206042480068401C0BD0012024F3C9
:1068B0003DF92168884203D2012024F337F900E032
:1068C000080020603B488178002904D00079002826
:1068D00001D1002010BD012010BD704710B50A780D
:1068E000012A0BD0022A09D0032A1BD1012819D171
:1068F00031480078012813D0022202E0012804D197
:106900000122002108000B0008E003280AD1887842
:106910004B780002034300210122080000F077F8C1
:10692000012010BD002010BD38B500248D9EFD9DB6
:1069300001000000346500A000020000B83FF84AE2
:106940000878F12807D0F22805D103200090012013
:106950006946FFF7CDFF200038BD70B5050038F35C
:10696000A8F9002803D104F052FB002801D001242B
:1069700000E00024002D02D038F38DF900E0002063
:10698000204370BD10B506F09DFE10BD102010B55F
:1069900004F042FB10BD10B50C4C6078002803D009
:1069A00001F3F2FD002060700120FBF7CBFB002813
:1069B00001D102F0DCFB02F06EFAFDF747F810BDE2
:1069C000D0D10004E0E900046CE600046C5B00B088
:1069D000F8B50D00060000200090180017001C00FC
:1069E0000D3000F393FA0028009018D0002D04D049
:1069F000FC4901600572466004E0FA49491E0160E5
:106A0000FF2101724472220039000A3043F3A0E8EA
:106A1000F5480168684600F388FA0020F8BD0120B7
:106A2000F8BD38B50D0011001A061C00120E012D1C
:106A30006B4604D119705A7000216A4604E01A703E
:106A4000220A6B465A706A460223FFF7C1FF38BD1F
:106A5000F8B5002406000F001AF012FD0500E34807
:106A600031010818037B43F362EA050E0E0E04059C
:106A70000E0001240021017341700800FBF7F5FBB3
:106A80000021FBF7DEFC28001AF0FEFC002C07D0EA
:106A9000002F05D02022012130000223FFF7C1FF83
:106AA000F8BDF1B50020FBF7E0FB05000098D04EE3
:106AB0000101CE480C182079FF2828D160790028E0
:106AC00019D0FF2817D0A068FBF777FB6179FE2962
:106AD00001D1C84902E07D23DB00594388420AD234
:106AE0000D1A012D07D9FBF764FB07003800FBF7EF
:106AF00064FBA842FAD9306800220B2100F383F925
:106B000000980121FFF7A4FF00206070F8BD280065
:106B1000FBF7C1FC01002079FCF73BFD6079FF2801
:106B20001DD000280BD0FBF744FB06003000FBF71C
:106B300044FB61797D23DB00594388423BC1BE277A
:106B400001000000306700A0000200004CD746F7AB
:106B5000F6D92800FBF7A9FC002801D1012100E0AB
:106B600000212079FCF71FFD00980121FFF77AFF33
:106B7000F8BD306800220B2100F34FF9F8BD70B565
:106B800006009F4900014418085C257B002817D0A7
:106B9000E088002808D0A068FBF719FBE1887D2376
:106BA000DB00594381420BD8002D03D0032D07D1C0
:106BB000012070BD0021042230000B00FFF73BFFD5
:106BC000002070BD10B50400FBF74DFE8C4821017C
:106BD0000818017B002909D0032906D14078002834
:106BE00003D100212000FFF73DFF10BDC078002831
:106BF000FBD00021042220000B00FFF71CFF10BD7A
:106C0000F7B500200C0082B0FBF739FB02997C4AF3
:106C10000700230009017B4D002601208C1843F357
:106C200090E90C0A070C0E13373A3E54640A790AAD
:106C300050540498E08005B0F0BD5654FBE7A178AD
:106C40000029F8D0E070F6E707002073E07800280C
:106C500017D002985A2201210023FFF7ECFE67703B
:106C6000E67028681D216A4600F3D7F86B46D8887D
:106C70000128E0D00020FBF702FB0121FBF7EBFB32
:106C8000D9E70121029820220B00FFF7D4FED2E7BA
:106C900002202073CFE7029800F0CDF8CBE7207BED
:106CA000022801D1042020730020FBF7E8FA00211C
:106CB000FBF7D1FB607800282AD100210298FFF76A
:106CC000D1FEFBF780FAA060B5E76078002802D01B
:106CD0002079FF28AFD128680022192100F39DF800
:106CE00002980121FFF7BEFEA5E7286800220921CE
:106CF00000F393F82079FF280AD03800FBF7D5FB82
:106D0000002801D1012100E000212079FCF74BFC93
:106D10000121D3E7607800288DD00298FFF7CBFEE1
:106D200089E70B788A78FF2B01D15A2A04D0202AD0
:106D300006D1C978012903D1052200210B007AE68A
:106D400070470878FF2804D188785A2878D32F22F2
:106D5000010000002C6900A0000200008BCE44AAB4
:106D600001D101207047002070478878202804D185
:106D7000C878022801D101207047002070472549BA
:106D8000000140184078002800D001207047F8B575
:106D900015000600022945D12878FF2818D11E4881
:106DA000006800283ED01E49096888423AD1006830
:106DB000002807D0012807D0022807D0032831D1A6
:106DC00007240AE0042408E0052406E0062404E081
:106DD0000D2801D1092400E008240020FBF759FA0E
:106DE0002A7807002100FBF701FB00281AD0094888
:106DF000320101211018817029780171697841717F
:106E000000213800FBF731FB0120F8BDEC13000036
:106E1000E0A6340070D300B0880E000440420F009A
:106E2000800E00040020F0E702001301234A10B591
:106E30009A1893780120002B06D01279FF2A03D0EC
:106E40001000FCF7BAFB002010BD70B50500002053
:106E5000FBF71FFA0600194829010C18207B0228AD
:106E600023D1032020737D20C000FEF722FF60782D
:106E7000002819D02079FF280BD03000FBF71FFB2A
:106E8000002801D1012100E000212079FCF795FBC9
:106E900002E0FBF7A2F9A060002D05D1084800220E
:106EA00000681E21FFF2C3FF70BD00212800FFF71C
:106EB000E3FDFBF792F9A06070BD000070D300B055
:106EC000880E000438B58D21564D4901280042F343
:106ED0001AEF5549554842F316EF554C564922686A
:106EE00008000092534A514B0C38FEF281FE524981
:106EF00022681C3908000092504B514A3430FEF28F
:106F000077FE22684C4900924D4A143908002B0044
:106F100020323830FEF26CFE38BD704710B5FAF7FB
:106F20005FFF002801D0002201E00022D243424846
:106F30000021243043F356F8002806D13E49243975
:106F40000868401C0860002010BD282101812830FD
:106F500010BD3C490968084737480022C3086A2A1F
:106F600001000000286B00A0000200007F26FA1735
:106F70001100183010B543F33FF8002806D133490B
:106F800024394868401C4860002010BD2821018138
:106F9000283010BD283810B543F304F810BD2F2356
:106FA0001B0158432D494018817B491C81732021C6
:106FB0000181203070472F231B0158432749401877
:106FC000817B491E817370472F231B01584323493E
:106FD0004018203070472F231B0158432049401888
:106FE000203070472F231B0158431D494018817BD7
:106FF000491C817320210181203070472F231B0100
:10700000584317494018817B491E817370472F23CD
:107010001B0158431249401870470C4900201C3985
:107020000968002902D088680006000E70470D48E4
:1070300000090001704700008CB600B0F057000056
:107040003C7000B0980E000420E500B09C5B00B0DE
:107050002C9500B038E600B078FB000480D300B077
:1070600050DC00B00CDF00B070B501253A4C2D07A4
:10707000E560FCF744FD39480021006843F316F849
:10708000A0682843A060012070BD10B500F03DF855
:1070900006F039F800F013F8314801681322114363
:1070A000016030491C20FAF799FE2B4881680122C3
:1070B00012071143816006F05FFB002010BD00B590
:1070C0002948142187B042F3FEED274814211430DB
:1070D00042F3F8ED01220021042003AB07C30200B4
:1070E0002248FF2191316B4607C3A838204A00236C
:1070F00020A1FDF2E7FB0004000C04D11A4820A1F6
:107100002830FCF271F907B000BD38B5204D1F489A
:10711000204C2860226800921F4A291D0800130095
:1071200018304033FEF26EFD226800921B4A29009F
:107130000C31080013001C304033FEF263FD22685E
:1071400029000092084A143108002B68203A2030A8
:10715000FEF258FD38BD0000009000A8845D00B02C
:1071600000F003A9216C0000502101B09972BFFB0F
:1071700001000000246D00A00002000066DE24670C
:10718000600501B077D20000426C654D62785461B1
:10719000736B0000426C654D6278466C61677300EA
:1071A000DC6600B04CC800B0980E0004F00601B0D8
:1071B000300E01B0F8B5F9480569681C3DD01020C3
:1071C000FFF2CCFE0028009037D0F549002402C021
:1071D000FF220A2142F3DCEC24E0E80720D0601E05
:1071E0000D281DD8A0000019083800D50020010086
:1071F0001A314F2903DD4F210E2C00D03520009A83
:10720000091A121D41188C4608E04607C108760F7E
:107210000127535CB740BB43401C53548445F4D80A
:107220006D08641C002DD8D10098001D07F04EFA9F
:10723000DC4801686846FFF2A0FEF8BDD74901208E
:1072400010B50870FFF7B6FF01F34BFB012007F004
:107250001BFA10BDF8B505000600D04F0C003878B9
:107260001C3E00280AD0D0480079C0070BD000206F
:10727000FFF799FD002806D0032C04D03000F480DD
:107280001AF03AEBF8BD0020FFF7BAFC1AF038EB21
:107290006A7AF868921C2300310042F305FFF8BDBA
:1072A00010B501F396FCBD490400C86849688842DE
:1072B00003D100221421FFF2CEFD02212000FFF7AE
:1072C000C9FF10BDF1B50098C17A857A047A40688B
:1072D000090206060D43360E6846FFF242FE2A00FA
:1072E00021003000FFF7AAFCF8BDF1B50027009897
:1072F000AB4A01688588C6880C32914203D10521CA
:1073000007F065F9F8BD806824210400283C21813C
:10731000001F290A05704170310A8670C170A248A9
:107320000079C0072CD00020FFF73DFD002827D0B2
:1073300000988068C27881781202114342790379FB
:1073400012024778134302783F023A43964F921E47
:107350003F881206120E8F420DD1934F79889942C1
:1073600009D17B793900934205D1801D891D19F01F
:1073700001FF002803D06846FFF2F3FD14F5B64B79
:1073800001000000206F00A00002000092369ADA8F
:1073900029E001270020FFF73DFC00982A0B2D056E
:1073A00081682D0D2800012306F027FF6846FFF2B3
:1073B000E2FD7F480078002805D10520E08020000C
:1073C0001AF0A4EAF8BD7E480168002903D0200025
:1073D00088470028F6D11AF09EEA012F09D1774894
:1073E0000079800705D5774920000968283088474B
:1073F000F8BD75480078002809D074490888401EF7
:1074000008807349E80040184188491C4180684859
:10741000321DC0682100052342F350FEF8BD1CB5A3
:10742000C188022935D02423421C052918D00829F7
:1074300013D103819A5CC15C120211430905090D45
:10744000644A8B005918535C002B06D0891801221E
:107450008A56002A01DD521E4A7042F3B7FD1CBD58
:10746000048903819A5CC15C120211430905090D6C
:1074700080393F29F1D958490481097828300129F8
:1074800001D0504900E055490968884701F3C0FB25
:107490001CBD01001C310191097A3E29DDD005296E
:1074A0000BD10420FFF264FD42490090783901605D
:1074B0004B4801686846FFF26AFD01A8FFF25BFDD8
:1074C0001CBD10B580884749884202D1FBF799FB63
:1074D00010BD4449491C884202D1FBF784FC10BD11
:1074E000FBF7BEF910BDF8B504000F000578407831
:1074F0000026000205432805000D8038402817D3D8
:107500001420FFF235FDFF21FF31009001608580DE
:10751000E278A17812021143C1800021C181241DAB
:10752000477384602E4801686846FFF230FD04E02E
:107530003900200000F0C9FB06003000F8BDF8B5A6
:107540000D001B4E3178002901D16869F06028894F
:107550004419E888082806D01DDC012850D00228EC
:1075600042D0032874D10C20FFF202FD00280090C5
:107570006ED0FBF775F90F490098183901606278F1
:1075800021781202114381808560154877DB49C755
:10759000010000001C7100A000020000EC2D3D6AFB
:1075A00001686846FFF2FDFC64E0092832D00A2831
:1075B00024D0112856D1FBF75DF901212000FFF7F7
:1075C0009CFF57E07C0E000401140000E4A6340088
:1075D000A05C00B078E6000494F500049BE500048C
:1075E000A8E50004489D0004109E000498E50004EE
:1075F0009CF50004E0A6340080FE0000FBF73AF999
:1076000000212000FFF779FF002833D0280042F343
:10761000E7FC2FE0002901D1FFF724FE7168F06834
:10762000884227D1A0780930FFF2ACFCFF490090D6
:10763000016062782178120211438180A178817102
:10764000A278E11CC01D42F3C0EA0098FFF743FF97
:10765000009807F0F4F8002804D1F548016868465E
:10766000FFF29FFC280042F3BBFCF06800221421CB
:10767000FFF205FC0020F8BDFEB500220500FF2149
:10768000EC48D243193142F3D5FC07005BD0A888FF
:107690000005000D00900020FFF7C6FA0320F880D7
:1076A00024203C183881A8882070A8881C23000A50
:1076B0006070E888A070009881000918DE480E18F4
:1076C0007078DE49401C707000985843401840792B
:1076D000FFF7BBFC0189DA4A08180190A968401A33
:1076E00080180290EA88824201D8E01C0AE0029ADF
:1076F000E01C42F36AEAE8880299421A029801996A
:107700002018C01C42F360EACE480078022803D15A
:107710007078401E707010E000981AF00AE9002896
:1077200012D07078401E7070009801F334F9207008
:10773000009801F330F9000A6070EA8839000020EF
:107740000323FFF706FFFEBDBF480168002903D0F1
:10775000380088470028F6D100981AF0EEE8002893
:1077600006D07078401E7070380042F339FCFEBDC0
:10777000A278B648D21CC0683900082342F3A8FC9E
:10778000FEBD71B581B0019AB04E908894680B2807
:1077900039D2A94983001B1859188B78FE99318C6E
:1077A00001000000187300A00002000018C583D774
:1077B000002B32D0FF23F73300921360009A238905
:1077C000D3800A79521C0A71A3490978012905D08E
:1077D000A44801686846FFF2EEFB1BE021891C23E8
:1077E0000D1958439A4940189F49407909688847BC
:1077F000009AA978D180AA78E91C42F3F0E90098B0
:1078000001F3BAFD200042F3F5FBF06800221421D9
:10781000FFF23FFB002001907CBD200042F3EAFB19
:10782000F06800221421FFF234FB01980028F3D005
:1078300001A8FFF2B4FB7CBDF1B500998A884E7BAC
:107840001005000D05000B2822D2920B00D000205D
:10785000864AC3009C182279002A19D0E5808A88BC
:107860008968120B002306F0DCFC002E02D160793F
:10787000401C607178480078012805D0794801687B
:107880006846FFF298FBF8BD009801F358FCF8BD7C
:1078900088687749096888476846FFF280FB002EB0
:1078A000F5D101212800FFF719FDF8BD31B5009889
:1078B000664D80880005000D84002418295D00298C
:1078C00012D06849096801F3BFF9654801780029B9
:1078D0000AD0611901228A56032A05DA4078002865
:1078E00002D10098FFF7D2FE6846FFF258FB38BD80
:1078F00001B55948007802281CD0009881888A0B6D
:1079000001D0002101E00905090DCA0057495118AD
:107910000A79002A0BD08279002A08D14A79521EAE
:107920004A71808801210005000DFFF7D7FC6846E9
:10793000FFF235FB08BD31B500984C4A8188090536
:10794000490C525C4449002A097817D0022912D008
:1079500048490978002903D047490988002902D0FD
:10796000FFF7E1FC38BD454A454C11788B00491CB6
:10797000E050117038BD01F310FC38BD806801295A
:1079800001D0404900E03A49096888476846FFF25B
:1079900006FB01F351F938BD01B500988068002855
:1079A00007D042F327FB2E480022C06800EE867DF8
:1079B00001000000147500A000020000013D5DA759
:1079C0001421FFF270FA0098808819F0C6EF0028A1
:1079D00003D06846FFF2EDFA08BD009801F3B6F94E
:1079E00008BD10B5234CE068002817D100212BA05A
:1079F000FFF20DFA6060A2681A21FFF254FA294AD8
:107A000060682021FFF24FFA274A60680421FFF2E4
:107A10004AFA60682549E0602348086010BDF0B567
:107A2000002185B022A0FFF2F2F9124DA860FFF705
:107A3000D8FF214F0421388801F3C9F801F3D8F8A1
:107A4000114E0024FFF2EEFA024B0390026812334B
:107A5000D11A33E092130000E4A63400905B00B02A
:107A6000109E0004B4B40004D202000098E50004A3
:107A70007CE600047C0E0004FCA93400ACF5000494
:107A8000489D00049CF500049BE50004A8E5000463
:107A90009CE50004E09D000494F5000462745F73AB
:107AA00064696F00CF700000AF6F0000B0EC00049D
:107AB00062745F6863690000A4E500049A426FD0B5
:107AC00024DCAC49531A8A427CD017DCAA4BD11A69
:107AD0009A4267D009DCFF3AF63A70D0032A6FD099
:107AE000092A54D1FFF7B2FE35E00129F1D0062969
:107AF00067D009294BD101F3CAF82CE0133B42F3BC
:107B000066EA084D73787F8446469C4648294AD0E9
:107B100023DC342965D015DC01296FD002296ED011
:107B2000032934D10820FFF241FA924902903631FC
:107B300001609249097801719148016802A8FFF239
:107B400044FA24E0452971D0462970D047291ED136
:107B50000321FFF7A7FB039474E7692968D009DCC8
:107B60004F2976D05C2975D0682910D1022106F002
:107B700056FDF0E76A2919D0722908D1EB686968C7
:107B80008B4204D1020017211800FFF28CF90398F0
:107B90000028E1D003A8FFF20CFA53E70221D8E74E
:107BA0004EE00FE063E0FFF7B5FBD4E7826941697F
:107BB000001D019200910FC819F0D6EE1787469D5F
:107BC00001000000107700A000020000F5D5E31AC4
:107BD000E7E750E052E057E030780028E1D06E4807
:107BE00000880028DDD068497D2000224F31C00088
:107BF00030F37AFBD5E701F348F9D2E706F06BFDE5
:107C000001F345FA55E08179808801F3C3F9C8E7AB
:107C10002BE018E08179808801F391F9C1E7808831
:107C2000010080393F2902D806F047FDB9E701F38A
:107C3000F3F9039900228888891D19F0A4EEB0E7B2
:107C400016E024E038E0007901F344F8A9E7007970
:107C50003070A6E7514A018911808088042138805C
:107C600000F3BFFF9DE716E01BE001F3C8F898E7BB
:107C7000FFF7A5FD79E7FFF7A3FE76E7FFF72AFEFA
:107C800073E7FFF749FE70E7FFF769FE6DE74449C8
:107C90000079087085E706F0BEFA03A8FFF293F9B1
:107CA0007FE740682969884292D0286128780028B7
:107CB0008ED0FFF7B1FA74E706F0E9FC55E7010052
:107CC00000200B2906D2374AC900891809790029F2
:107CD00000D001207047344810B541693348344A18
:107CE00081600021016141618161C1610262416283
:107CF000FFF24CF806F0B2FD10BD01000020002993
:107D00000AD1294AD168002906D01378002B03D064
:107D10005268914200D101207047F3B5012406005A
:107D200081B08578C078000205432002854200D8E2
:107D30000024002C25D11C48C1684068814203D131
:107D40000298002800D10124002C15D000221948E7
:107D5000110042F38DF9002803D1212000F326FF02
:107D60000FE00221C1802421471801812A1D310022
:107D7000380041F348EF00E037000299380006F080
:107D80003FFC2000FEBD000089130000FF01000041
:107D900098E50004E4A63400AAE50004A8E5000480
:107DA0009FE50004489D00047C0E000468E600B0D6
:107DB000CF70000074C800B000210160012070473E
:107DC000002101600848006B8001C00F1C6C5CB78B
:107DD000010000000C7900A00002000032CCE14755
:107DE0007047064840300079C00701D10120704734
:107DF0000020704702484068C07A704770DA00047B
:107E000070DC000470B50124394D6406EC6039481B
:107E10000021406842F390F9AC603748807EC0078B
:107E200004D136498888621390438880012070BD50
:107E3000012B10B50BD1324842F3AFF9314800683D
:107E40008047002803D13049012009688847002075
:107E500010BD2E4808B502680092264A2C4B1032FD
:107E60001100083908001030FDF212FF08BD244847
:107E7000142110B541F36CEF06F056FD25480021A2
:107E80004068C1721B48026823488260234A02612D
:107E9000234A81614261234AC161026241622249EF
:107EA00009688162002121A0FEF2C5FF22491A4A19
:107EB00008601A21FFF20BF8204B174801211B68BC
:107EC0000D228902303098471348FEF269FF0028DE
:107ED00001D0012010BD1A491920F9F7C5FF00286B
:107EE000F8D10349012040068860002010BD000041
:107EF000009000A8D05B00B090DA0004C02800A871
:107F000078DC00045CEF000468F00004980E0004C4
:107F10008CCC00B070DC0004E0E600B0451034000A
:107F2000491034005D7900002CF000046863695F3B
:107F30006D75785F666D00003CED000464F0000430
:107F40003179000070B501248A4D6404EC608A48E0
:107F50000021406942F3F0F8AC60012070BD10B51B
:107F60000AF0FCFD002010BD08001100012B10B527
:107F700002D1824A12689047002010BD002070474D
:107F800000207047FEB50020010001907CA0FEF2A9
:107F900052FF794C606109F057FF002179A0FEF291
:107FA0004AFFA06162691A21FEF291FF2600784F14
:107FB0001C3600F03DF9774C774D01E02068804792
:107FC000386880470028F9D1286880470028F5D113
:107FD000421E009271480122072101AB54834F14C5
:107FE00001000000087B00A000020000C6245FFA28
:107FF000FBF2BCFA00240CE0E00085196A680A4232
:1080000006D0325820009047696801988843019053
:10801000641C01990029EFD1D5E71C3010B5417AD5
:10802000092901D0082917D162490024447209683E
:10803000884761480068804754488168491E8160CC
:108040000178002905D00470806900221421FEF215
:1080500048FF55480068804710BD70B505004B4E7D
:108060000C00B06900280ED029682200022342F3D8
:1080700061F8002803D0F068844200D9F4604D49CB
:1080800028000968884770BD01004948002210B5E2
:10809000FBF2FCFA10BD1CB500200200019000901C
:1080A0004348072101ABFBF261FA002804D1019893
:1080B000400700D001201CBD00201CBD38B50500C4
:1080C0000C00FCF20DFD0022D24300923848230040
:1080D00001222900FBF24AFA38BDF8B50125060055
:1080E000364CAD0219F03AFA284F00213A69AA1A23
:1080F00004E02378EE2B03D1641C491C8A42F8D893
:10810000691A002E396101D0691A316019F02AFA12
:108110003869F8BD10B504002748006880471B483F
:1081200021494278944202D10868804710BD4470CA
:1081300008688047002CF9D0012C04D17D24E4018B
:10814000FBF758FD03E07D242402FBF759FD0321D2
:108150002000FDF77EFB03212000FDF780FB0321BB
:108160002000FDF779FB03212000FDF77BFB10BD0C
:1081700010B509F09BFE012010BD08B56846FFF759
:10818000ACFF012008BD0000009000A8F45B00B027
:108190007CF000046E6663006863695F6D75785FEC
:1081A0006E666300C4F20004D0F20004C8F200045A
:1081B00010410004BCF10004CCF20004683C00044F
:1081C000254810B50068C00604D5FFF764FF0028F5
:1081D00036D007E0FFF75FFF002803D11F48C07CBF
:1081E000002801D0002010BD06F0A1FED646604652
:1081F00001000000047D00A000020000DFDC818A95
:108200000028FAD006F05BFE0028F5D106F052FEF9
:108210000028F1D119F0D8EB0028EDD107F0EEFFDE
:108220000028EAD006F0EBFD0028E6D00AF0D4FEE4
:108230000028E2D00F4800780028DDD106F0DFFDED
:10824000012803D10AF0ACF8002803D006F0D7FDCE
:108250000228D1D1012010BD10B5FFF7BBFF0028C7
:1082600001D009F089FC10BD70470000985900B09A
:108270008CF200B02D5E00B0F8B5150006000A4C77
:10828000302021781A004843084B069FC018491C2B
:108290003060217000922B003A00611CF9F2FEFC64
:1082A0000006000EF8BD0000940E000440EB00B084
:1082B00070B50500824A834E1178C807000F335805
:1082C000AB4201D1801907E0491CC807040F1170A7
:1082D0003059A84202D1A019406870BD642128001D
:1082E00041F3ACEE7849020000204300CB5A9342A0
:1082F00002D2401C0928F8D3A1193551486070BD3D
:1083000070B505006E4A6F4E51781036C807000FE1
:108310003358AB4201D1801907E0491CC807040F4C
:1083200051703059A84202D1A019406870BD642133
:10833000280041F384EE64490200002032314300FA
:10834000CB5A934202D2401C0C28F8D3A1193551C4
:10835000486070BD5E485D4A4168114341605D4AB6
:10836000C1681143C16070475B4870B50068002860
:108370001ED0FDF73FFC0500FDF74CFC0400FCF7A8
:10838000E2FBFCF7FAFBFCF72CFC2800FCF793FE61
:108390002800FFF7DFFFFCF737FF2000FDF752F959
:1083A0002800FDF731F80520FCF7F6FBFCF7B8FBD9
:1083B00070BD70B5040019F0DBF805002000FFF770
:1083C00077FF41496A310C5C2000FCF77EFE3E4994
:1083D00060001231085A642444437D21A002C90080
:1083E00041F32CEE401E052141F328EE3B49401C91
:1083F0000860280019F0C0F8200070BD5B51050B23
:1084000001000000007F00A0000200002B343F3775
:1084100070B5040019F0B6F805002000FFF752FF10
:108420002E496A310C5C2000FCF76BFE2B49600082
:108430001231085A64244443280019F0A7F8200098
:1084400070BD70B5040019F09DF805002000FFF71D
:1084500061FF22497A310C5C2000FCF763FE1F4962
:1084600060004A31085A64244443280019F08EF809
:10847000200070BD70B5174CA068002829D1606835
:10848000002816D1FDF7C0FB05280DD0062808D01E
:1084900012498B3107280BD00A2809D10800203057
:1084A00004E00E489B3001E00C48BB30606000E007
:1084B000616060680949407A08390D5CFDF7A4FBEA
:1084C0000C494000085A64235843290041F3C0ED89
:1084D000A06070BD405C00B0A0ED00B038020004A8
:1084E000103254760027008022436577506600B032
:1084F00044C800B0000000047047002811D088076D
:10850000800F0ED001280CD0022801D0032808D1FA
:108510003B488168090104D5816801229206114314
:10852000816070471123374A1B02002910D00129AE
:1085300017D0022915D0032912D1510D00289068B7
:108540001FD033231B02984390609068084306E0D5
:108550000028906802D0FF21491CF7E798439060FB
:1085600070470028906809D0984390609068012176
:1085700049020843906090680901E7E71121490228
:10858000FFE78843EBE7F0B50D00C10701D10C28E8
:1085900001D91220F0BD0024400884462BE0297840
:1085A0006D1C2A786D1CFF2A03D10020FFF7BAFF4B
:1085B0001EE00023180009E04700BE19B7788F427B
:1085C00001D10123F270401C0006000E0E4E3788C8
:1085D0008742F1D8002B0BD1300003885B001B18B9
:1085E0009970018849000918CA700188491C0180E6
:1085F000641C2406240EA445D1D80020F0BD000040
:10860000002F008040230080C0ED00B09982D89CEC
:1086100001000000FC8000A000020000ACE4E44483
:10862000FF2212020240010612021143FF2212042D
:108630000240120A1143000E084370470349FF220B
:10864000C432888B1042FCD17047000000080090B3
:10865000F8B5002425000F4E0F4F1049A0003550EB
:10866000095830206043C019C46081600C49016121
:108670000C4941610C4981610C49C1610C4901629D
:108680000C4941620C498162FEF2B2FB641C022C6F
:10869000E3DBF8BDF0EC00044CD8000400ED00046E
:1086A0005FFB330093FB3300D5FB3300F3FB330058
:1086B0000BFC330075FC330055FC33000C480021E3
:1086C00010B501600B4802680B488260C1600B491D
:1086D00001610B4941610B4981610B49C1610B4942
:1086E00001620B4941620B498162FEF281FB10BDC0
:1086F000E4EC0004E8EC00041CD80004F5F93300B5
:108700001BFA330035FA330043FA330061FA3300C1
:1087100099FA33007FFA33000278FA49401C0A7054
:108720000278401C4A7002784078000202430A81B5
:10873000704710B5F34C0020210062784B6909891D
:10874000012A07D0022A0BD0032A08D18B4206D374
:10875000606103E05A06520E8A4200D2012010BD29
:10876000E94BA2695A43E94BD218A2611A408A42E6
:10877000F4D810BD10B537F3ABFE10BD10B537F30C
:10878000CEFE10BD10B537F3EEFE10BD70B5E04D56
:108790002878002833D10021DEA0FEF274FBE04CE3
:1087A00000212061DFA0FEF26EFB60610021E0A0ED
:1087B000FEF269FBE0600020A06120690022202118
:1087C000FEF2ADFB206901222B21FEF2A8FB6069BD
:1087D00000222021FEF2A3FB606901222B21FEF280
:1087E0009EFBD64AE0682021FEF299FBD448442142
:1087F00041F300EB0120D4492870D24808600020E2
:1088000070BDF0B585B0D1480078002878D137F335
:10881000C5FE0024E443CE4822000021622B5B0603
:1088200001000000F88200A000020000580C5AF974
:1088300041F35AFCCC4F22003860CA48002141F372
:1088400053FCCA49BB4E086038686A46018908185B
:10885000000C009030692521FEF26BFBC3486A468C
:10886000006801890818000C009070692521FEF24B
:1088700060FBBF481A210180A9490024091D84809A
:108880000181C480012144814180B94A3069262197
:10889000FEF24FFBB74D3A20E880B54A70692621B9
:1088A000FEF247FBB4483A21C1803968F0230A89B7
:1088B0002A815F006B810122AF812A80AB4A6C80E4
:1088C000126815890581438187810480448010895D
:1088D00082180889411801A837F393FF6B4618796D
:1088E000F7210840A54901AA0978C909C900084328
:1088F0001871F0682521FEF21CFBA14B00221B68B9
:108900000221100098479F48006801880322D20284
:1089100091430180002005B0F0BD70B59A4D954C93
:108920002868002812D1421E98485C2141F3DCFBE4
:1089300003212860C1802030C17028682421018172
:108940000021618029210028A1800ED02868A188FB
:10895000018185490122096804230860754800697E
:1089600041F310FC6088401C6080002070BDF8B5A9
:10897000012204236F487C4900690968FEF2CDFAA0
:108980007C484188002948D07F4D24212C68624BC7
:1089900021814188C088EF274143891CA1806D490E
:1089A00024340A7922704979E01C0907090F6170A3
:1089B00029688988A1700121E17021790A091201D1
:1089C0000832DF210A409978CE07B60E3243960668
:1089D000F60F3A40360132438E075206F60F520E1A
:1089E000F6013243D609BF27B6013A403243491C4B
:1089F00042708807800F9870601D37F3CBFD2868A0
:108A000000268088A41C0655296861488A88006869
:108A1000D21C032341F3B6FB2E600020F8BDF8B54D
:108A200000263D49009608695B4F401CD3CBEEFC05
:108A300001000000F48400A00002000041F48489D9
:108A40000861594835000068002821D1380041F3F9
:108A5000B7FB554C2060396800290AD05449096891
:108A60008847380041F3ACFB2060304800210125E5
:108A70000171206800284AD0444A002151800189B0
:108A800001260B189B78C91C8380918001813EE0F0
:108A90003E4980884A88C9885118891C814235D945
:108AA000424841F38DFB0400386800280BD0404950
:108AB0002000096888473D4841F382FB04001B48B9
:108AC000002101250171002C21D0208901260019E7
:108AD00082782E48A280808820810119324800685F
:108AE00087880389BA181204DB19120C1B188280BC
:108AF000FF203130824200D9FEE7A288180041F3FE
:108B0000C8E82B4920000968884700E0012626486C
:108B10001E4A0068D28881880024891A891E0F04A1
:108B20003F0C002E7DD001890E187EE0505C00B015
:108B30000D661900FF7F000098EC00046D646576F7
:108B40005F736263456E630008D700046D646576E9
:108B50005F736263446563006D6465765F62745F32
:108B600070636D0055310100C4D6000451820000CD
:108B70007CE60004B4EC0004B45B00B0A0EC00049C
:108B8000A4EC0004B8D60004FCD700040CD8000400
:108B9000E7E90004A4F800046CEA0004ACEC00046B
:108BA000905B00B0840E0004A8EC000498D600048A
:108BB000B0EC00043019FFF7F5FD002834D030196F
:108BC000407837F319FEC24A1179002906D1401CBA
:108BD0008007800FD0700120107116E0D17881429B
:108BE00003D1491C8807800F0EE0491C8907890FB3
:108BF000814206D1401C8007800F00270125D070DC
:108C000020E0401C8007800FD070A41C30190600A3
:108C1000FFF7CCFD002805D0300037F3A9FCAD4F9D
:108C20000BE018E0012505E0641CAB484088001902
:108C3000B842BFD9A748874204D1FFF71A20D345CD
:108C400001000000F08600A000020000B51C3A34CC
:108C50008EFD002800D0A64FA449488800194880FE
:108C600089880818A349096808819F48A24C87424F
:108C70000ED1002D0CD19B480121C180C168491C37
:108C8000C1609C482168006808600120009023E0D2
:108C90009748874201D0002D02D00120009003E0C8
:108CA00096490868401C08608E480021C18094489D
:108CB0004A1E41F32DFA934E306001890D18392177
:108CC00081800A009049280040F3ECEF280037F338
:108CD00059FC2168306808608C4E21687069012257
:108CE000052341F363FA7F4DE888002809D18848BD
:108CF000406B002805D18748FDF264FC844920318F
:108D0000C88182482168406901220523FEF219F9D1
:108D10000098002813D07549764E4888CA88801874
:108D200048808A8812183068028149888288914276
:108D300005D17949096888470020306018E06D48FE
:108D40000268002A14D0694E93887088F188401810
:108D5000801C98420CD910898118B08810817788BE
:108D60008018DB1B938000237380928840F39AEF76
:108D70006A48664F6A494289F86809680823FEF222
:108D8000E0F8FFF7DEFD206801890E186869401CD5
:108D900068612878002813D0E888012805D15D484B
:108DA00032003100FDF211FE0AE05648006800284A
:108DB00001D041F383F9574832003100FDF29FFDA5
:108DC0004A4821684289F868082341F3EFF9FFF720
:108DD000E2FD0020F8BD10B504000020E20702D03B
:108DE0000800FFF7F1FC4F490978012914D1210748
:108DF00001D5FFF724FD610601D500F02BF821060F
:108E000001D500F043F8A10501D5FFF71CFE61076D
:108E1000890F01D000F001F810BD70B50025414E5A
:108E20003078012812D14048384C05702069FEF294
:108E300078F86069FEF275F8E068FEF272F8256174
:108E40006561E560E561357037F3C6FB2AC2BC3267
:108E500001000000EC8800A00002000072053869E3
:108E600037480560002070BD70B50024334E224D98
:108E70003078002808D12A480022C0682821FEF254
:108E800076F8AC70EC702C710120307020480460D2
:108E90002C4804602448FDF293FB00206C6170BDF7
:108EA00070B5264D287801280FD11D4C0022E068AE
:108EB0002921FEF25CF8206900222A21FEF257F8EF
:108EC000606900222A21FEF252F800242C701E4D07
:108ED0002868002802D041F3FBF82C60134C0A4D9F
:108EE0002868002801D021688847184841F37CF998
:108EF00000282860F4D170BD505C00B0FFFF000076
:108F00000CD80004FF070000A8EC0004A4EC000447
:108F1000BCEC0004B45B00B0A00E000490A43400CC
:108F200008D70004F843000438410004B0EC000402
:108F3000FCD70004A0EC000498EC0004B4EC00049E
:108F40007CE60004B8EC0004ACEC000498D6000405
:108F500010B536F392FD00210800FFF715FB002045
:108F600010BD000070B5012500201AF395FC040027
:108F700003201DF3EDFA002804D105201DF3E8FAC3
:108F800000283BD0012138224A43A05C800705D548
:108F90001019C079002801D1002504E0491C0904FA
:108FA000090C0829EFD32800FAF79DFFFF4E30681F
:108FB0000088C50AFEF7C7F80400FAF77FFFE90743
:108FC000FB48FC4D09D00078844210D90020FAF704
:108FD0007EFF30680188A94308E04078844206D8C3
:108FE0000120FAF774FF3068018829430180082CBA
:108FF00004D2F149A0000A58521C0A5070BDF0B5C5
:10900000002595B0ED4F2E000CA80295FAF74FFF02
:1090100024220CA903A840F3BAEE00216B46D973B1
:1090200008ABE748E74AD97200781278024302D0C9
:1090300001226B46DA73002802D0012008ABD872F7
:10904000E1486B4699730079002801D0012098739C
:1090500000206B46187358739874D8745842472C84
:1090600001000000E88A00A00002000086ED86D41E
:10907000D876987608AB012418711C206043D84933
:10908000085C032801D005285ED1082C25D32000D8
:1090900008380104090C01910EF30AFA01991E2304
:1090A0005943091848797F2801D26B469874487A49
:1090B0002C2805D03D2803D00D2801D00C2801D143
:1090C000062004E06B46D87C002802D102206B46C3
:1090D000D87401206B46587336E026F369FF64218B
:1090E00061436D1C09183420405C2D062D0E0328A9
:1090F00001D0012807D1761C403188883606360E0B
:10910000B84200D20700200005F0F1F9002803D092
:109110006B46987E401C987601206B4618732000A1
:1091200017F32EFC002804D120002BF345FD002866
:1091300002D001206B46D876200002F014FC0028F3
:1091400002D0012008AB1871641C2404240C0B2CE1
:1091500093D300206B461874002D587406D0B54286
:1091600004D10120102F187400D2587408AB0120CC
:109170005D71FDF7B0FC08ABD871FDF7C5FC08AB1D
:10918000040018729748984B00787D215843C90015
:1091900040F39AEF0006000E08AB98716B46197BFE
:1091A00008AB1A7C914227D16B46597B08AB5A7C9D
:1091B000914221D16B46D97B08ABDA7C91421BD11D
:1091C000197910AB1A7A914216D1997A884213D143
:1091D0006B46187C08AB197D88420DD16B46587CD4
:1091E00008AB597D884207D1D87910ABD97A88422B
:1091F00002D1187B844201D00420029024220CA9C1
:1092000003A818F04DF8002803D0029903A8FAF734
:109210004AFE15B0F0BDF1B501242700694E2100CA
:10922000F07841F359FB002814D0442060436F4983
:1092300000254018C16B0098401A002801DB050486
:109240002D0C7079210041F347FB002808D070896C
:1092500085420DD838007179A0408143717107E0D3
:109260003089854204D338007179A04069DE8BE9EA
:1092700001000000E48C00A0000200009F1558A42B
:1092800008437071641C2404240C082CD1D3F8BD4D
:10929000514910B5C968401A802802DD0020FAF74C
:1092A0004EFE10BD10B530F3F8FC0400FFF7BDFF13
:1092B0002000FFF7EDFF10BD10B5FDF758FF464940
:1092C0008A78904202D94879002800D00120FAF724
:1092D00048FE10BD424810B500240C38FAF781FE54
:1092E0003F480C380178002906D0417A002903D084
:1092F0004078002800D001244248047010BD10B509
:10930000FFF7E8FFFFF742FEFFF7CCFFFFF7D4FFC0
:1093100010BD38B504000820FDF2C0FE0028009002
:1093200007D00521890212C0374801686846FDF25E
:10933000C4FE38BD38B50028274C01D1012002E019
:10934000012801D10020A0710820FDF2A7FE00280D
:10935000009008D02D490160A17901712C48016865
:109360006846FDF2AAFE38BD1B48002901D0022143
:1093700000E003218170704770B504001500FAF712
:1093800026FE002810D01C2068431A494018007996
:10939000002800D001201F49C969002900D00121FF
:1093A000012C01D1FFF7E0FF70BD70B506000D0084
:1093B0000120FAF7C4FD0020FAF7CAFD064C01208F
:1093C000A840E178002E41D0014348226A43E17071
:1093D000114923E064EA00046C5C00B0000800005E
:1093E000DCED00B0FFFF0000D7EA0004D8EA00047B
:1093F0006CD20004B4B40004BC5C00B0E204000011
:1094000058D30004C35C00B0E0A63400141400007C
:10941000E4A6340008D7000470CA00045118897EFD
:10942000002903D121790843207102E02179814389
:109430002171E078002800D00120FAF7AAFD2079F8
:10944000002800D00120FAF7ADFD70BD8143E17026
:10945000ECE70B001100012830B408D00D4A0120C0
:10946000D47888408443D470547984435471002B59
:1094700008D0012B04D0022B04D10120D449D4837D
:1094800001000000E08E00A0000200006BFDE61964
:1094900030BC94E70020FBE730BC704710B530F3D8
:1094A00006FC0149C86010BD6C5C00B070B50125B8
:1094B0000E4CAD04E5600E480078002802D004F0A0
:1094C0005FFC07E00120FDF7E4FAFAF7CCFB00208F
:1094D00021F393FCA0682843A060012070BD0348DD
:1094E000816801229204114381607047009000A8B6
:1094F000C95D00B010B50400F8F730FD1C3421043C
:10950000090C002801D0002201E00022D2430F48BC
:1095100040F326FE002805D10D490868401C08606C
:10952000002010BD0189081810BD10B504000068A6
:109530001C3840F3EBFD0020206010BD11681C3981
:10954000488170471C38408970470000905B00B02C
:10955000B85C00B0002310B508E09C000C5B8442AE
:1095600003D11C489A00885210BD5B1C9342F4D36F
:1095700010BD30B5002409E0A500555B854204D13B
:10958000A00080188170012030BD641C9C42F3D380
:10959000002030BDF7B59446040000260D4F12E0C0
:1095A00029194988B94204D101996246FFF7D2FFCF
:1095B00007E00906019A090E6346FFF7DAFF002863
:1095C00000D06753761C0349B500605B491C884294
:1095D000E6D1FEBDFE0F00000100897E01200029BA
:1095E00000D00020704701218140FA48014201D09B
:1095F0000120704700207047F8B5F74C658BF6489E
:1096000020308688E78B0020FDF7B2F9F348006828
:1096100080471FF395FBF2490020C87308746583E7
:10962000ED4820308680E783F8BDFEB507000BF3D8
:1096300092FF3C680600A588E01D01AA02A921F35B
:1096400025FD6B461889242819D1A0888823584302
:109650008019C078E34E0028207A03D1C007C00FDC
:1096600020D104E0C006800F1BD001281AD1FAF7E0
:10967000B8FC002815D13078012812D812E0DA4958
:1096800088420FD10820FDF213FDD8495A3A289A92
:1096900001000000DC9000A00002000015E641A9D6
:1096A00000900160A1888180617A8171D54801684C
:1096B0006846FDF216FDFEBD38000AF3B6FE6B46A5
:1096C0001889D1498842F6D1CA4A0120917BA84025
:1096D00081439173FEBDF8B500210600CB483EF3EF
:1096E0004FFA0700C94801213EF34AFA0400C7486F
:1096F00002213EF345FA050002203900C0433EF343
:1097000007FA2E60266069680020C0430860696817
:10971000062E48601BD16A68410091606968C86084
:1097200069680861696848616168B948086061688A
:10973000B84848606168B84888606168B748C860E0
:109740006168B74808616168B648486125E06968A2
:1097500088606A680021D1606A6811616A68516135
:109760006A68012191616968C8616168AE480860F2
:109770006168AE4848606168AD4888606168AD481E
:10978000C8606168AC4808616168AC48486161685C
:10979000AB4888616168AB48C8612A002100380085
:1097A00000233EF333FCF8BDF7B582B00398403098
:1097B0000778202F00D92027A348BC080068816EB5
:1097C0000968A14203D1C06E0068A04202D0200007
:1097D000FFF781FF8D4802213EF3D2F900909B48AC
:1097E00000213EF3FFFB01900298019940683EF38F
:1097F000E0FD864800213EF3C3F90460050040689F
:1098000003993A0040F380EA804801213EF3B8F919
:1098100004600399060040683A00203140F374EA7E
:10982000019B0022310028003EF376FC0406240E42
:1098300028D02868002824DB834829000068C06EEF
:109840003EF30CFB00281CDD3068002819DB7E4845
:1098500031000068C06E3EF301FB002811DD029864
:10986000019A806801993EF316FE009A00990198CA
:109870003EF394FC00983A004168049840F344EAAF
:1098800000E00024200005B0F0BD70B50400082001
:109890002060200014308821050040F3F5EAE165DE
:1098A00001000000D89200A000020000E10EFF14A9
:1098B000D2EA20009C306C21060040F3CCEA002163
:1098C00028003EF367F9A060012128003EF362F909
:1098D000E060022128003EF35DF9206100213000A4
:1098E0003EF38AFB60604E4800213EF353F90600C8
:1098F0004B4801213EF34EF905000220A168C04308
:109900003EF310F9206830602168296071680020FA
:10991000C04308607168002348607168886072689D
:109920000021D16072681161726851617268012111
:10993000916171683200C861686840490160686877
:109940003F49416068683F49816068683E49C1603D
:1099500068683E49016168683D49416168683D4900
:10996000816168683C49C161A06829003EF358FBE9
:109970002B4800213EF30EF90500294801213EF352
:1099800009F901002068086028606A68354810609D
:109990006A68354850606A68344890606A6834483C
:1099A000D0606A68334810616A68334850616A68F9
:1099B000324890616A683248D0614A683148106024
:1099C0004A68314850604A68304890604A68304878
:1099D000D0604A682F4810614A682F4850614A6831
:1099E0002E4890614A682E48D061636800222800A2
:1099F0003EF39CFB2000FEF299FB70BD18CF0000E7
:109A0000000A00A9C8F70004BC5C00B0D0EA00045A
:109A10007F200000C60C000004AA34007F10000064
:109A2000549C0004B1B946C1ECDEB8FE4930247242
:109A3000ABE9A70FE7809CE5190521644B60D227AD
:109A40003E3CCE3BF6B053CCB0061D65BC86987646
:109A500055BDEBB3E7933AAAD835C65AF8EE0004E1
:109A6000DC9C000496C298D84539A1F4A033EB2DB4
:109A7000817D0377F240A463E5E6BCF847422CE120
:109A8000F2D1176BF551BF376840B6CBCE5E316B64
:109A90005733CE2B169E0F7C4AEBE78E9B7F1AFE28
:109AA000E242E34F38B50500FB4C200026E97EF585
:109AB00001000000D49400A000020000F8F6216428
:109AC000FFF7F7FE4C20FDF211FBF9490090016011
:109AD000E16820224968083040F394E92069202297
:109AE00041680098283040F38EE92800FDF2DFFB42
:109AF00001006846FDF209FB38BD38B50400282096
:109B0000FDF2F4FA821D0090E848A11DFFF760FE07
:109B100001000098E74A026003D0002120308171E3
:109B200007E0122226210A54FF222021801D40F343
:109B3000F8E82000FDF2BBFB01006846FDF2E5FA03
:109B400038BD38B5040018F307F94620005D202819
:109B500001D1D94D00E0D94D2820FDF2C7FA821D70
:109B60000090A11D2800FFF733FED14A0099D21EB4
:109B70000A60A2888A8001220028D149A08804D0E6
:109B80008240087A9043087203E08240087A0243D8
:109B90000A722000FDF28BFB01006846FDF2B5FA67
:109BA00038BD31B50024FCF7C6FE0098C54A0168EF
:109BB00089181AD003290DD005290ED0072912D1F2
:109BC000BE48FEF2BDFABC48FEF2BAFABC4900201B
:109BD000C87204E0FFF770FF01E0FFF78EFF012479
:109BE0006846FDF286FA200038BDFFF7AAFFF6E7C7
:109BF00010B5FCF7A2FE10BD10B50400FFF2F7F996
:109C0000200004F01CFC10BD8079AF49002801D071
:109C1000FF2801D1002000E0012048727047F8B50C
:109C200026F3F8F90700012464256543785D0028D0
:109C300021D01C206043A5494618307900281AD04D
:109C4000A3492000096888470090B078A1490C23F7
:109C50005843096840188088009940F368EA411C1D
:109C600000989D4A414312680904090C200090475E
:109C7000E91960310880641C2404240C072CD3D912
:109C8000964900200870F8BD48214143944A10B518
:109C90008C1832F3FFFE00281DD020002FF344FF64
:109CA00004214020015500202FF3A1FEC01C80019B
:109CB000800930F300F88B4B01221B682BEFC39A0D
:109CC00001000000D09600A0000200000C1E9FD9E9
:109CD0000100200098470200210002202FF39BFF83
:109CE000864A0221002021F301F810BD70B504005E
:109CF0002FF324FF00202FF384FE2FF3E6FF010053
:109D0000052220002FF3A9FF7D48804D03787D4870
:109D10002D6802787C4801782000A8473120005D3A
:109D2000A0857EE648214143F8B57248784F0D186A
:109D30000124482060436F494618B54218D044209A
:109D4000805D052801D0092812D1F878210040F360
:109D5000FFFD00280CD06F48005D012808D13100BC
:109D6000280034F321FBB08D082CA88508D304E02B
:109D7000641C2404240C082CDBD32800FFF7B6FF56
:109D8000288A26F37AF92876288A26F37CF96876D9
:109D9000F8BD10B5040026F347F9642161430818A3
:109DA000407810BDF8B5050048235843514A584C37
:109DB0008618584801274155E078AF40B8430B005A
:109DC000E07040F3AEE906041904042828182800BE
:109DD000FFF7DFFF01280ED1B07E00280BD14D48E0
:109DE00003214155A078290040F3B2FD002802D19B
:109DF000E0783843E070F8BD4420805D052803D04A
:109E0000092801D00628F6D1B07E0028F3D1280019
:109E1000FFF788FFECE738432E49E0700020887197
:109E2000F8BDF7B54821050010004143314A01272C
:109E300089180E008E463F21490151184A7A8B78C5
:109E40009446344A2036145C3A008240002D1CD0DF
:109E500013438B701C233D004343214FDB199F7834
:109E60002D4B1B681B88BD402B4202D16346134318
:109E70004B722849012C1AD0019A022A01D10522DD
:109E800000E004220A5400210BE093438B706346E8
:109E90009343204A042C4B7201D0052C07D100219A
:109EA0001154724691850B4A31755171917119495E
:109EB000095CFFF777FF194800688047FEBD000086
:109EC0009CEE00B0A60F0000A80F0000BD16D5172D
:109ED00001000000CC9800A000020000CB079D8488
:109EE0004C9B0004449A0004BC5C00B05EF0FFFF91
:109EF000C0BD0004B4B400044CF7000498EA0004A8
:109F00002CFC000427E9000470CA000458F800047F
:109F1000D7E733001CEB000404EB00040CEB000457
:109F2000A0F7000450D2000424EB00041CEA000453
:109F3000BCF70004F8B5060000202FF36CFD050007
:109F40000024FF4FF969884203D0FE4805631AF3E5
:109F5000C1F9082EFD610CD0102E06D01AF3BAF903
:109F600004061AF3B7F9000404431AF3B3F9000224
:109F700004431AF3AFF92043F8BDF3B5040083B0EE
:109F8000F14D687901283FD1F04B00201A68C100DB
:109F9000565A3607360F0A2E04D1565A360936015C
:109FA000761C5652401C0004000C0E28EED3AE89DD
:109FB00001204002864201D9060002E0402E00D274
:109FC000402600202FF327FD07001020FFF7B2FFE7
:109FD000310040F3C0E878188601DD48B609EE6428
:109FE0000068008FC107DB4800D001210174017CAB
:109FF0000172AA89E989019200912B7CD64D012238
:10A000002D6831000C20A847D4480078002813D0D0
:10A010000820FDF27FF8FF215C3102900160217879
:10A02000017161784171A17881710499C171CC4845
:10A03000016802A8FDF27DF84DE40121C04A81408B
:10A04000507B884350737047BD4930B51023C548D5
:10A050008A780068002A2BD0C34AC54C557AC34A77
:10A06000247812782243002D0DD0002A03D1C14A52
:10A070001278012A03D930224A700B7011E03C2279
:10A080004A7004220CE02024002A01D04C7001E028
:10A090002D224A70CA79D20701D00C7001E00C223F
:10A0A0000A708979002902D1C18E1943C18630BD59
:10A0B000C28E9A43C28600204871887130BD01214A
:10A0C00081409F48427B114341737047F1B50024A2
:10A0D0000098858825F3B2FF060000985A9CE08816
:10A0E00001000000C89A00A0000200003FEF2339E1
:10A0F000A64B01680027CA1A99427ED01FDCA44BE8
:10A10000CA1A994268D013DCA24A891837D04E295E
:10A110006BD1A14AA14B5188994266D08079012820
:10A1200063D15078002828D10800FFF7D2FF5CE007
:10A13000072A20D0412A58D1FFF784FD55E01C2A78
:10A1400056D009DC0F2A44D0142A4ED1072141569B
:10A15000001DFFF71CFF37E0232A2ED0572A44D1D9
:10A160008288017A8079FFF770FE00988188C07933
:10A1700030F34DFB28E08088D7E708001AE0642020
:10A18000684380192030007D01280AD11C206843D3
:10A19000834940180079002803D182480178491C7E
:10A1A00001706C4A01219078A94088439070FFF7B4
:10A1B00055FF2800FFF74BFF17E025F37EFF0098BF
:10A1C000642380885843375401246846FCF2AFFF6B
:10A1D0000BE0FFF742FDF7E7017D002905D072494A
:10A1E0004A8B6E498A4200D107752000F8BD04E011
:10A1F00081798088FFF7EAFDE6E78088FFF762FD56
:10A20000E2E7FFB50020A3B000210A000F9005A8E7
:10A210001C0006C025F31CFF019024981C23007825
:10A220001D90A1881C91E188A2891B92627A5943F2
:10A2300052081A92A27A1992E27B52081692584A50
:10A24000891809791890259815910290FF22082104
:10A2500003A83FF384ED16F32AF9002801D1012069
:10A2600001E016F324F9040016F324F96100081A3A
:10A27000C10F0818C003000C0D900120109018ABFE
:10A28000197D4A4B259A1B6805A89847012425008B
:10A2900002E0641C2404240C642060430199085CDF
:10A2A000002801D10B2CF4D30B2C52D1002010909C
:10A2B000D9E13F4920000968884700287AD01C98D6
:10A2C0008442FBD01C206043354940180079159921
:10A2D00088426FD164206043019940182290C07C6D
:10A2E000012810D11A9925983FF36AEEA213C8B538
:10A2F00001000000C49C00A0000200002617FD49D8
:10A3000022980E0040691A993FF364EE8E42EAD11A
:10A310006B46987D401C9875AAE122981A9980692D
:10A32000884201DB1A9801E00006000E1B99179085
:10A33000012010290BD01B99202908D01B99CA1F76
:10A34000F93A04D01B99CA1FFF3AFA3A00D1032008
:10A350001699229A41180E06928B360E0121102A68
:10A360003AD0202A31E080E1BC5C00B000E8000473
:10A370006CD2000428EA000484EA0004ACD2000491
:10A38000A4F70004C0E80004F4E7000464EA000451
:10A3900050D20004D7EA0004D8EA0004D0EA00044E
:10A3A000BB0C00004F0C000009F4FFFF48E900045B
:10A3B000FFFF0000B4B4000470EC0004A0AD000482
:10A3C00034FC000468FC00046BE005D0D31FF93BAB
:10A3D00002D0FF3B5B1E00D10321229A20329278EB
:10A3E00052181206120E431813920DE0139A8A4265
:10A3F00005D9139A521E1206120E139204E08642D9
:10A400004AD9761E3606360E179A934244D8139AC6
:10A41000179FB218BA42E9D83EE0139833E0259866
:10A420002190801920901799401E3FF3D4ED229877
:10A430000F0041691298401E1F90081817993FF3AA
:10A44000CAED8F421CD16B46987D0025401C987543
:10A4500021990298884204D122981F994069401896
:10A4600001E02098401E0121490688421A99259052
:10A4700003DB7F2252068018FFE73FF3ACED1D910E
:10A480001F980006000E012D129002D1129801288B
:10A49000C5D2761E3606360E012D02D1012EBCD253
:10A4A00003E0002D7ED0012D7DD164206043019911
:10A4B00046183420805D002875D00428FCD0200088
:10A4C000FF4A0D99126890470C901C206043FD498B
:10A4D00047183879002803D1FB4800780028E3D1D9
:10A4E0004036B0881A99884201D31A9801E00006D4
:10A4F000000E1790012014901B981028BBA717EF8F
:10A5000001000000C09E00A000020000D2FF43F442
:10A510000BD01B98202808D01B98C11FF93904D0F4
:10A520001B98C11FFF39FA3901D103201490EC495F
:10A5300020000968884711901598002804D13879BF
:10A54000002801D002200C90E6490120097800295A
:10A5500000D070890C990818401E0004000C0B9064
:10A560000020089001200A9061E0002009902599C0
:10A570000A98012608181E904DE01E981799401E53
:10A580003FF332ED11980F0080191799401E3FF3E9
:10A590002CED8F4237D108986B46401C0004000C0C
:10A5A0000890187D0025401C1875CF4801680029C7
:10A5B00008D02000884701E064E03BE0002801D09B
:10A5C000012000E000206B46997D401898750A999B
:10A5D00014980C9A401A0B990006000E891B10184B
:10A5E000814206DB1998F82807D10C98864215D9C4
:10A5F00003E00C990998884210D36B46587D0125D9
:10A60000401C58750AE00998401C0004000C761C98
:10A610003604360C09900B988642AED90A98401C35
:10A620000006000E0A900898002803D10A98149991
:10A6300088429AD90B2C03D0002D01D1AB48457824
:10A64000012D1FD1641C2404240C64206043019953
:10A65000085C002801D10B2CF4D30B2C0FD1A3489C
:10A660004078002808D0A24A0021126805A8904727
:10A67000002801D0012000E00020109005E0012D0D
:10A6800000D12AE60B2C27D11098002824D1159848
:10A69000002821D11B99012010290BD01B992029BA
:10A6A00008D01B99CA1FF93A04D01B99CA1FFF3A58
:10A6B000FA3A00D10320259918AB0E911A7D8D4BE3
:10A6C0001A991D680EABA847002800D00120012868
:10A6D00010900F9000D10124874A03A9126805A8A1
:10A6E0009047109801281DD1259818AB401C259043
:10A6F000197D1A9A491C0906090E91421D9101D132
:10A7000000211D9118AB197D189A91429E04056095
:10A7100001000000BCA000A000020000DA20B22965
:10A7200001D1002110911A9A02998918814203DD02
:10A730001098012800D1C0E50F9800287048407893
:10A7400015D0002802D10B2C27D006E06D4A00213D
:10A75000126805A8904700281FD06D4B01201B6888
:10A7600025AA1DA99847012817D10B2415E0002818
:10A7700013D0644D00212A6805A8904700280CD00A
:10A780002A6807A903A89047002806D06B46187FBF
:10A79000002802D1D87B1D90E7E7239818AB0480EE
:10A7A0002498197D017027B0F0BDF7B584B005007D
:10A7B0000AF32BFF5749040068000F5A88266E439E
:10A7C0008821A05D794303910290605C022805D046
:10A7D00051488189A943818107B0F0BD0220A0556D
:10A7E000069A05992800FCF277FF0298A055039875
:10A7F0000019007D0028EFD1380001A91BF395FD59
:10A800000028E9D0444801780029E5D04349096887
:10A810008A686B4619798B001B18DB69D21A920182
:10A82000192392095B019A42D6D98089E840C00772
:10A83000C00FFCF227FFCFE7F8B5820006003848CA
:10A840000D001018012282560021AA4201DB0024CB
:10A8500004E002228256AA421BDC0124C278A242F2
:10A8600000D001210029C47013D0300006F3D3FDBD
:10A8700000280ED00820FCF275FCFF2182310090E8
:10A88000016086808471C571264801686846FCF2C3
:10A8900078FCC9E4F3B5002083B001902FF3E3F80E
:10A8A00000900AF3B2FE01251C246C430F48015DA1
:10A8B00000297ED0201887781B490C20784309682E
:10A8C000085A1A4900040968001688470600074814
:10A8D000005D03282CD1280002A91BF326FD0028C7
:10A8E00026D0012025E0000064FC0004B4B400047C
:10A8F000D1EA000448F7000420E9000490E60004CF
:10A9000020E9000438FC00049CF3000430FC00043F
:10A91000ACF30004E8B5000450990004C6A874859F
:10A9200001000000B8A200A0000200002EC80C9494
:10A9300078EA0004FCB50004F4E7000498EA000497
:10A94000D8F50004002000280CD06B46187AF9498D
:10A950000C2358430968085AF7490004096800168F
:10A9600088470600F548C419A07D012803D00328B4
:10A9700001D0042858D10AF352FE882169430818EF
:10A9800016303B2120F3CEF902000120EC49019062
:10A99000A800085C002847D1E849B8004018816C3D
:10A9A0004B1C0BD0009B591AE44B890140339B8808
:10A9B0008909994202D30021C943816404998E42D6
:10A9C0001BDAA17D00E043E0032916D00221A17526
:10A9D000009B002A83640ED039200257D7481823E1
:10A9E0002030C356921B9A4200DC0121D54A280030
:10A9F0001268904716E0012111E003998E4211DDA3
:10AA0000A17D04290ED0816C491C0BD10221A175B6
:10AA10000099002A816401D00021E7E70021280085
:10AA20000AF375FB39200655C74B31001B68A27D20
:10AA300038009847280006F3F8FC002808D0C049E1
:10AA4000A800085C002803D031002800FFF7FEFEB4
:10AA50006D1C2D042D0C082D00D22FE70198002825
:10AA600003D0FCF2EDFD022803D1FCF2E9FD012840
:10AA700007D1B648006880470022B54913002DF37E
:10AA8000D7FC05B0F0BD70B50C21B248B24C817254
:10AA90000B2141710A2141740921C17100256571A1
:10AAA0002D20A571607020202070A561A57031F364
:10AAB00089FEAA4840213FF31EEAA94820213FF31E
:10AAC0001AEAA8480068018CC908C9000184018CF1
:10AAD000022211430184C18E10229143C1869F48F6
:10AAE0006021403065823FF306EA9F491920887251
:10AAF0006573E57170BD70B50D001400012A07D9AA
:10AB0000401B0019401E21003FF356EB44436019DF
:10AB100070BDF8B50C00070015001E0025F3C0FA43
:10AB200064217943081840308188218074D7B1436B
:10AB300001000000B4A400A0000200003730D2E4FD
:10AB400041892980C0893080B7E6F3B583B0039886
:10AB5000874F0468258A002C65D0200030F3D3FB92
:10AB6000E16940180499081A5DD4002620002FF3EB
:10AB70002BF8ED00785D00283BD0ED196868E1699D
:10AB800001AA471A208A02A96B46FFF7CCFF002FC3
:10AB900012DC6F686B461A8904983900FFF7B5FF1D
:10ABA00068600C2201206282A0850020E082049867
:10ABB0003900FFF7AAFF0FE00C2F09DA68686B462F
:10ABC000E061188960829888A0851888E08204E096
:10ABD000049920002FF3FDF8E06120002EF3F4FF2C
:10ABE0000020E0764420025DE16920002FF37BF82D
:10ABF00008E0634B049A1B68039821009847E069BA
:10AC0000E9194860A07E002804D020002030867B0F
:10AC10000121817320002FF341FAA07E002801D08A
:10AC20002034A67337E7E07E0128FBD1E800385CCA
:10AC30000128F7D00020E0762DE7FFB583B0482348
:10AC40000F0003984F4958430C9E40180D9D0290E9
:10AC50002EF3BAFF0398C40045480C2E14D90121E5
:10AC600001553800484F06D006982FF374F8404934
:10AC70006118486002E00598002809D10C260125DA
:10AC800000200E90B86905E00021002F015504D185
:10AC90000298C0692FF35CF806900E9A3B4C009224
:10ACA00024682B00069903983200A047A8E510B548
:10ACB00014001A00002C05D1354B1C5C042C01D06B
:10ACC000052C03D1334B1B68984710BD33F33AFA78
:10ACD00010BDF7B584B004000F0025F3EBF90500B3
:10ACE00000202EF3D4FE48216143264A2A4B8918BE
:10ACF0001C226243D2186423634312795B19342502
:10AD0000ED5C002D12D0012D48D0022D54D0042D21
:10AD100006D19D885A78010020002B00FFF7C7FF5D
:10AD2000069A3900200024F363FB69E5496800298D
:10AD3000F6D0002AF4D19D885A7801002F4D25E2E3
:10AD400001000000B0A600A000020000C3D86C59AA
:10AD500020002B00FFF7B5FF5CE5000098EA000437
:10AD6000D8F50004B4C70004FCB5000430F40004B6
:10AD70003CFD0004E0F60004470C00002CEB00044E
:10AD8000BC5C00B0FCED00B038D3000464EA000401
:10AD900030D2000460F8000470CA0004B0D100048E
:10ADA000ACF7000424EB00048CF70004B4B40004F6
:10ADB00018004030C289418980886D4607C5390036
:10ADC0009B6B069A2000FFF742FF23E50020E50079
:10ADD000FF4E7055986B2EF3C8FFA9194860A9E77C
:10ADE00031B584B00499FB4A08680024801810D05B
:10ADF00045282BD18879012828D1083101A81BF3D7
:10AE000064FCF5480C22006801A910301BF3B8FA65
:10AE10001CE00AF318FC0499F04D89880122130004
:10AE2000AD7B8B402B4211D088234B4318186030E8
:10AE3000C277EB4A0023126800920A00808BE9492E
:10AE40002DF3FEFA012404A8FCF2ADF9200005B0B0
:10AE500030BD10B501680022FF397E3900290BD0C2
:10AE6000DC4BD533C91812D18188DF4B8900595C7E
:10AE700001290CD182720AE08179002907D08188EA
:10AE80001C235943D94BC9188B78D9495A542CF3F0
:10AE900040FF10BDD74910B509680A8880239A433E
:10AEA000D54B1B78DB09DB011A430A802DF307FC25
:10AEB00010BD70B5D24AD14C527A2578002A01D003
:10AEC0000122227031F3DCFA257070BDFFB581B02C
:10AED000482300250198CB4F5843C419A17E0298FE
:10AEE000814219D12E20005D002815D10398012838
:10AEF00001D1012601E00026F643019822F3CBFBA5
:10AF0000C149884208D048235843C419206A80198F
:10AF10002062E0698019E06140342079042802D180
:10AF200004250220207101A80FC831F37AFD042DF9
:10AF300001D104202071B8E5C100B44A09184901C3
:10AF400089188031C97C002914D01C23471C2CFD92
:10AF500001000000ACA800A00002000004C16E04C3
:10AF60005843A749142340188078AE4958430968CC
:10AF70000A5A002A08D140184188002904D1808843
:10AF8000002801D10120704700207047F8B50D005E
:10AF90001E040700360C0AF360FBAC88022F4AD16E
:10AFA0000127032E2AD1002018F316FD0600287A67
:10AFB0004006400E11283ED18F4821005B302DF312
:10AFC00064FA2878C107C90F200028F37DFE20000D
:10AFD000FFF7BCFF00280FD0382060438019006ABB
:10AFE000002809D01C20604385491423401880782C
:10AFF0008C49584309680F52012072E4132E12D174
:10B00000882161430818007D002814D18648007803
:10B01000012810D9E8791322C107C90F2000212384
:10B0200020F33EF9E8E78148864204D17048A74002
:10B03000817B0F438773002053E4F8B504000D00B3
:10B040007B484079012810D17A4B00201A68C10052
:10B05000565A3607360F0A2E04D1565A360936018B
:10B06000761C5652401C0E28F0D30820FCF2A2F8A1
:10B070007149009001602178017161784171A17876
:10B080008171C5716D4801686846FCF2A2F828E438
:10B0900056481CB56946006810301BF3A6FB68488B
:10B0A00001680D200856674909688847010068460D
:10B0B000FFF7C3FF1CBD4D481CB5694600681C3036
:10B0C0001BF393FB5E4801680D2008565D49096833
:10B0D000884701006846FFF7B0FF1CBD10B5019816
:10B0E00059494008884202D11BF31DF910BD1020B8
:10B0F000FEF770FF10BD10B52FF3CEF9454820388C
:10B100004188912901D99121418010BD70B502007B
:10B11000548A0800012C08D9D5692100401B001968
:10B12000401E3EF394EF4443281970BDF7B584B038
:10B1300004001700066B456B008A19F31EFA3843AA
:10B1400000D001200690069A059920002FF308FFF1
:10B150004020005D032827D1200020308EB11490BC
:10B1600001000000A8AA00A000020000F029D0B948
:10B170000390C77F0297608A019047430598390082
:10B18000401BC0193EF36CEF78434719676306987C
:10B19000002811D00398857F0198009545430598B4
:10B1A0002900801B40193EF35CEF6843801920633F
:10B1B000009A0299914200D8380095E5059920003F
:10B1C000FFF7AEFF90E5F8B506002EF35DFB0A2110
:10B1D000714305000C18603C207C012856D1607D2D
:10B1E000002853D03000FDF2F8FC070001003000C9
:10B1F00016F0D4EC002833E0FCED00B039F4FFFF8A
:10B2000088EA0004BC5C00B0F8A93400BD0B000063
:10B21000FCB50004B4B40004CAC7000470EA00041A
:10B22000E7E90004D1EA000450D2000470CA000427
:10B23000FFFF0000E0BD000460EA0004D0EA000463
:10B240007F1000006CD2000428EA0004CF0C00003C
:10B2500000AA34008CEA0004D8F50004AF8119007C
:10B2600010D0390030002EF33EFB0A207843002135
:10B270004019603821740174617541753800FDF220
:10B280008CFC06E0300016F08EEC02E03000FDF29F
:10B29000BCFC002076E438B50C001100049A009242
:10B2A0000A0021002DF314FBFD4861010068091814
:10B2B0008888FC4A1278002A04D05622562800D9E1
:10B2C000020010008880488138BDF7480088400798
:10B2D000C00F7047F44930B50400098800201422DB
:10B2E000114001D0012030BDF04D0A224A435219CD
:10B2F000137A022B02D15288A242F3D3491C0904CB
:10B30000090C0229F1D330BD0C235843E8494018F9
:10B310000089704700B5008AFFF7F6FF904201D917
:10B32000012000BD002000BDFFB583B00C000D0062
:10B330002035C8690290287D0190C87E002637001C
:10B34000002828D1218ADB4A505410003B388179EB
:10B35000002920D0218A80783FF35EFB00281AD094
:10B36000D44A01203B3A518A4003A37E94729757F6
:10B3700001000000A4AC00A000020000E9D10EC949
:10B3800081430120002B00D00020400301434804EA
:10B390000121400CC903401850825079297D814217
:10B3A00000D30800012637005071069B059A0398C8
:10B3B000210030F3A4FB0090208AC3490A5C521C90
:10B3C0000A54208A19F3E1F8002804D0A0898008E3
:10B3D0008000401CA0810298002E00D1E069002F5F
:10B3E000E06105D001982875002801D0401E28751D
:10B3F000B54E218A3B3EB0783FF318FB00283AD087
:10B400007079002801D0401E7071208AAF49095C14
:10B41000052905D1707900282DD00320E0762AE097
:10B42000B179012927D1A37E01221100002B00D080
:10B430000921A54B1B5C8B420DD91C235843A44901
:10B440000A2340188078A34958430968085A80079E
:10B4500001D5A2850FE0059906222000FFF764FFC1
:10B46000002808D0287D401C2875A08D401CA08590
:10B470007079401C7071009840E4FEB50D00160014
:10B48000847E099A0899002C09D1078A8F4CE45DC3
:10B49000042C01D0052C02D103200870FEBD0192BE
:10B4A00000913200290030F349FFFEBD10B50400C1
:10B4B00024F328FE64216143425C002A04D008186A
:10B4C0002030007D012800D0002010BDF0B587B0ED
:10B4D00000217D48804C3B38817001206E46482118
:10B4E000414342001218091920314D7C6B469D548E
:10B4F000D2180D7C401C00045570897C000C072874
:10B500009170ECD92FF3D9F8744F01253E00A03685
:10B510004821694370480C18280024F3FBFD0028DB
:10B520003AD06A48405D042801D0052853D124F35D
:10B530004DFD002822D164493B39C879C0071DD090
:10B540000120A84006908A7810438870F07829007E
:10B550003FF36CFA002805D1F07806990843F070A3
:10B56000B869E061680040196A46115C20348018AF
:10B570006174417821748078A0742CE0F8CB45B1D7
:10B5800001000000A0AE00A0000200001D39B07450
:10B59000F07829003FF354FA002826D00120F178F2
:10B5A000A8408143F170B869E0611EE0280024F3EF
:10B5B000CDFD002804D12800FFF782FF002814D019
:10B5C0001C20684347494018007900280DD14420C9
:10B5D000005D042806D0208A3F49C0004039085C3D
:10B5E000012802D10120207660766D1C2D042D0CDF
:10B5F000072D97D9FEF796FD0FE43849F1B50025E0
:10B600003B3901264D71354F31003B3FB8783FF350
:10B6100017FA00283CD048207043344944182000D1
:10B620002EF304FB38008079012831D030483100F6
:10B63000A030407A3FF304FA218A294A515C052957
:10B6400017D03337002800D1083F19F34BFE2821CB
:10B6500071434018407821002031385C0A00087599
:10B66000A17E00290BD00A210A2800D901001175FA
:10B6700005E03C21002800D12D2134200155342043
:10B68000015D16483B384279891841714078A085A0
:10B69000761C3604360C072EB5D9104F3B3FB879CF
:10B6A000012806D078793900401E0006000E787116
:10B6B00020D13878801C06060098360E8019B861B3
:10B6C0000220B87119E0000074EA0004CEE800041A
:10B6D0007AEC000448D600043CEE00B0F75C00B001
:10B6E00024EB0004B4B4000490EA000470CA00041F
:10B6F000B0D100040026012088710124B87821000F
:10B700003FF39EF900281BD048216143FF480818E9
:10B710000021C176BA79012A07D1002D00D1050098
:10B72000FB4A1219203AD17703E001213422115447
:10B730008185A84204D00099052289192EF305FBC2
:10B74000641C2404240C072CD8D9002D04D00099A3
:10B75000052228002EF3F9FA6DE4F0B518231C2613
:10B76000EC4A002552785A43E84BD2180B23DB01F0
:10B77000D218146A028AE84B5643F3189E789C4606
:10B780000C237343E54E36689B199B88E2CB1EEF72
:10B79000010000009CB000A000020000632217C45A
:10B7A000E44E7688B34204D9836BCB1AB34200D9F6
:10B7B0000125002C0BD0E38E934204D1C2698A1A72
:10B7C000B24200DB0125628A012A00D100256246CF
:10B7D0001279002A0BD09122002C03D0638A032B0C
:10B7E00000D82822FFF7B4FD002800D0012528004A
:10B7F000F0BDF7B582B004000020019019F37CFD84
:10B80000218A282359434018CB4940780978884237
:10B8100008D3039919222000FFF79AFD002801D0D0
:10B82000012000E000200090BE48218A2438807862
:10B830003FF310F9002804D103992000FFF797FF88
:10B840000190BC4D218A2035A8783FF303F9070009
:10B85000218AE8783FF3FEF82500060040350028ED
:10B8600009D0208AB549085C012811D0032802D1EB
:10B87000287909280CD0AB48218A243880783FF3F6
:10B88000E9F8012804D0002F04D02879092801D133
:10B89000012000E0002001990027002923D0002E7C
:10B8A00004D0218AA54A515C01291CD020002EF326
:10B8B000C7F9E776A07E00280FD1A148417800297A
:10B8C0000BD18078002808D1208A18F37EFE00284A
:10B8D00003D1618A0398081803903520297901550E
:10B8E0000399062252E0E17E019A009B0A4303433A
:10B8F0001A433AD0A28DE069039B82189A1A50D459
:10B9000020002EF39DF9002E31D08648218A24385C
:10B9100080783FF39FF8012803D10398FFF777FE63
:10B9200006E0884BE7761B68049A03992000984745
:10B930002879052819D1208A8049085C032814D168
:10B94000794818234079764958437F4E40180B2197
:10B95000C9014018056A06E0A54203D032682900F3
:10B96000200090472D68002DF6D105B0F0BD774836
:10B97000016800290ED0208A884700280AD0E7767F
:10B98000039920002EF361FA049A010020002EF39F
:10B99000E6F9EAE76E4B049A1B680399D0320A99DC
:10B9A0000100000098B200A00002000097CAA97927
:10B9B00020009847E3E70029E1D0A17E002918D1B3
:10B9C000002E16D0218A624A515C012911D106004D
:10B9D00020002EF33FF9E7762879052802D1E169A6
:10B9E000049ADDE7049A039920002EF3C2F9E66178
:10B9F000C5E7514D243DA8790128C0D1218AA878F6
:10BA00003FF332F80128BAD120002EF323F96879E8
:10BA1000002803D10398FFF704FEB0E7E776E16959
:10BA20000522BDE7F3B581B006000768027A0299E6
:10BA30003800FFF7E8FE0124482161433D480D1816
:10BA40004420405D317A884214D1AF4212D0298A15
:10BA50003F48405C04280DD005280BD03A482030E0
:10BA6000C0783FF301F8002804D0327A0299280008
:10BA700030F332FB641C2404240C082CDCD3FEBD00
:10BA800070B50025384C25602EF3FAF92A4924397F
:10BA90004879002803D1488A4004400C48822A484B
:10BAA00017238038C069498A8288DB029A4319408B
:10BAB0000A4382802D482060012070BD70B50400CB
:10BAC0002348055D200032F36AFA29002000FEF7C2
:10BAD000F5F970BD70B50400254D002028602000E8
:10BAE00032F376FB234828601948015D2000FEF7F9
:10BAF000E5F9012070BD012181400F48243880788C
:10BB0000014201D0012070470020704770B50D0040
:10BB10001949060040000C5A2900300018F33EFE77
:10BB2000002E35D0154968062BD50C2060430A5CE1
:10BB3000521C25E070CA0004E05C00B02CEB00044D
:10BB4000B4B4000498EA000430D20004A2E5000472
:10BB500024EB000478D5000418F7000478F70004FB
:10BB600090E600040CF800044CF8000469B30000EF
:10BB700080F70004BDB30000E8B500043CEE00B05F
:10BB80000A54280604D50C2060430A5C521C0A544F
:10BB900070BDF8B52EF33FF9FD4905000A6A9042E1
:10BBA0003ED0FC4F01240D62200017F3C7E2C5E12F
:10BBB0000100000094B400A0000200008E3277095A
:10BBC00047FF0078002830D01C206043F749F84A2E
:10BBD00040188078126801018918F64AC00012687E
:10BBE0008018C088002801D1012000E00020C0009A
:10BBF0000818C688200018F3FCFC00280CD00C2183
:10BC00006143C8194278795C8A4205D14188B142C2
:10BC100002D14168691A07E00C206043395CC01901
:10BC200041704560002146800181641C2404240C7D
:10BC3000072CC3D9AEE5F7B588B00400C669008A01
:10BC4000DD4A0490126809999047DC4A0390126813
:10BC50000999049890470290049844235843D8497E
:10BC600040180190D748049980783EF307FF079069
:10BC7000049818F3BEFCD44D002803D1287902990A
:10BC8000884201D9012000E000202A79039B01218C
:10BC90009A4200D800210843059101D0012700E015
:10BCA0000027049818F3A5FC002809D00199403119
:10BCB00088780978884200D308000299884208D31E
:10BCC0000598002807D001984030417803988142B8
:10BCD00001D2012000E000200690A07E00286ED155
:10BCE000E27E002A03D1E18A0998461AE6610798A4
:10BCF00000282BD0617E237E0320C91849084B1CE5
:10BD0000032B01D30800401C002F009007D0012A0C
:10BD100005D1AE4B029A1B6803992000984700207A
:10BD2000002FE07621D00199403108784978884287
:10BD300000D30800079AE979002A00D1A979009A6E
:10BD40005143814206D9099E00251AE0607E217E7A
:10BD50004018D8E73421095D002901D00091F2E7AD
:10BD6000618A81420CD808000AE00820FEF76EF9CB
:10BD70008107608A890F411A0D042D0CA84200D258
:10BD80000500069901200F4300D00098E082079932
:10BD900005200927002900D00700092F27D18C484A
:10BDA000218A00783EF36AFE002806D18948218A5C
:10BDB00000783EF363FE002819D00527A559B94F36
:10BDC0000100000090B600A0000200007ADAC9B4B9
:10BDD00017E0002F05D0824B029A1B6803992000C0
:10BDE000984700200500E0760798099E002805D0B6
:10BDF0000698002802D00A20A082E8E7142009272C
:10BE0000A08271193A0020002DF3C7FF0BB0F0BDDE
:10BE1000694910B5087331F333FA10BD10B52EF32C
:10BE200011FA6D48644980388079097B084301D153
:10BE3000FFF7C3FE10BD70B51C00CB7E002B18D1E0
:10BE40008B7E002B15D0694B5D7818236B43684DB2
:10BE50005B190B25ED015B191B6A0125CA61002BDB
:10BE6000CD7604D05B8A032B01D8072300E015238D
:10BE70008B8523002FF31EFF70BD70B50D00046885
:10BE8000E07E002816D029002000FFF78EFC002855
:10BE900004D0A18DE0694018281A0BD420002DF39E
:10BEA000EDFE0020E076608A41193520025D200019
:10BEB0002DF373FF70BD494949780840704703006E
:10BEC000454800B5407AFFF7F6FF002806D0998A6A
:10BED0000720072900D20800988200BD4548008845
:10BEE000FAE73548407B002800D001207047F7B5BD
:10BEF00004001600807E002500285AD13E480078B4
:10BF0000012856D94020005D002852D1208A18F31C
:10BF10007AFB002815D1314F208A0122797882409E
:10BF200011420ED1294A0199126890473979884205
:10BF300007D3618A01E005042D0C4819B042FAD3F9
:10BF400037E0608A4100B14233D82C492C4A097845
:10BF5000127811432CD1207E617E00264018E18AA0
:10BF60004008002901D1A18D00E0A18A401E0818D7
:10BF700003041B0CFFF7B5FF002802D05B1C1B0459
:10BF80001B0C608A984200D203000B48407BFFF7ED
:10BF900092FF002801D00A2606E00F488078FFF7BC
:10BFA0008AFF002800D00826608A9919814200D9AA
:10BFB00005002800FEBD0000BC5C00B03CEE00B0F7
:10BFC000B4B4000450EA000440EA00041384EE9282
:10BFD000010000008CB800A000020000BDC3CBE946
:10BFE0001CF7000420F7000458D3000450D20004CA
:10BFF00078D5000410F80004DAEA0004DBEA000453
:10C000002CEB000470CA000472EC0004D0EA0004B7
:10C01000D8EA0004D7EA0004FFB583B00C0005009D
:10C020001F00888980088000FF49C97A0843A081E1
:10C0300020002EF3DEFCA28D082100913B002100A0
:10C040002800FA4D01922D68059AA8470290E07EDB
:10C0500000286BD1208AE1698200F5488150208A4E
:10C0600018F3DBFAF34A012600280AD01178208A57
:10C070000B00C340DB0704D1330083400B43137034
:10C0800005E0218A3000884011788143117020003A
:10C09000FFF71FFF2268059920002EF3BDFEE6483A
:10C0A00018234079E549584340180B21C90140182D
:10C0B000026A059920002EF3AFFEA18A3000012903
:10C0C00000D90800DE49A0820978012907D9618AD0
:10C0D000062904D8A18D884200D30800A08225003B
:10C0E00040352879042804D123F3ACFF002800D080
:10C0F000A6826878012809D1E08A002804D0A08AA5
:10C10000A18D884200D9AE7000206870A8780128FF
:10C1100005D1207E617E40184008B84202D32878BD
:10C12000002802D00320E07600E0E676029807B00F
:10C13000F0BDF7B582B00D00272204992800FFF763
:10C14000E0FE0499BF4B41181B6800222800984765
:10C15000E861012628004030019048207043B7492B
:10C160004418270040373879042801D0022864D1C8
:10C17000A54262D00199097981425ED1B24A21007B
:10C18000126828009047002857D0298A228AA84B95
:10C190008E4694468900920059589A580120891A6F
:10C1A000002900DC0020A97E00231A00002903D00A
:10C1B000A98F012900D10122A37E0021002B03D0E9
:10C1C000A38F012B00D10121002907D0994B614693
:10C1D0001B78CB40D90701D000280BD00FD5A47D08
:10C1E0000100000088BA00A000020000492B75542D
:10C1F000002A01D1002807D1934A71461278CA401B
:10C20000D1070AD1002808D0E969934B491C1B6863
:10C21000002228009847E8611EE020002DF342FD2F
:10C220000020E076A18FA1858D498B4B0988A182E2
:10C23000B87001207870E1691B68491C0022200059
:10C240009847E06101003A7920002DF3BAFD761C91
:10C250003604360C082E8AD30020E876A98F804A4F
:10C26000A9851288AA82019A0124907001984470CD
:10C270007C486A8A40889200904200D31000AA7ECF
:10C280000004000C002A09D1298A8A006D498958C6
:10C29000049A511A81421DD800241BE02A8A1C23CB
:10C2A0005A43714BD21892780C235A436F4B1B6838
:10C2B000D2189288824201D9012400E00024012989
:10C2C00008D1FF22049991322800FFF773F8002863
:10C2D00000D001240422002C00D10222E9692800A8
:10C2E0002DF36FFD05B0F0BDF8B515001E00482315
:10C2F0004343574C069A1C19009233002A0031F32D
:10C30000BFFE2089802108432081B1E4FEB50D00E5
:10C310001F00482343434E4C1600099A08991C19E4
:10C32000019200913B003200290031F31FFF208968
:10C3300080210843208151E6FEB50D001F004823EF
:10C340004343434C1600099A08991C190192009125
:10C350003B003200290032F395F9208980210843FF
:10C3600020813BE6F8B515001E0048234343384CB6
:10C37000069A1C19009233002A0032F3B5F920897D
:10C3800080210843208173E4FFB500209FB0002185
:10C390000A000C900B900A90099007A806C023F39E
:10C3A000F7FE049020981C230068109022982E49D4
:10C3B00080881C902298FF22408945082298807925
:10C3C00012901C985843401800791390082105A832
:10C3D0003DF364ED00210A000B000C0015A81EC0FF
:10C3E000012064214143049A89180A7BDA5AD2C198
:10C3F0000100000084BC00A00002000050D3AB2468
:10C40000012A13D14A7B012A10D11C9A904202D1F1
:10C410002299098A07E03422525C002A06D0042AB5
:10C4200004D04031C989420015AB9952401C000626
:10C43000000E0828DFD31348007D01284AD1114E91
:10C440001C23F08A0D49584340180079317E1BE0C7
:10C45000C0BD0004F8F7000438D30004C6EA0004A5
:10C460002CEB000470CA0004D0EA000458F8000461
:10C470005CF8000472EC000430D20004B4B4000490
:10C4800098EA0004A0BD00044C08717E4908002809
:10C490000B9104D12DF373FB11900A9003E00AAACB
:10C4A00011A92DF399FBB07E21F3AAFA012802D13C
:10C4B0000B990A9804E00A980121490648400B9913
:10C4C0003DF328EE601AA14201DD0B994018119945
:10C4D0000818099010980F900D9001201B902806C5
:10C4E000000E1E900F9A0E92501B0F9007A81092EC
:10C4F000FF4B1E991B689847002401260E9910983F
:10C50000884205D00F9B421AC31A9A4200DA0F9153
:10C51000641C2404240C0B2C0E900FD1F548807859
:10C52000002808D0F44A0021126807A89047002884
:10C5300001D0012000E000201B9013E1012C11D15B
:10C54000EE4B187D01280DD19A8B09990B986F46F7
:10C5500007C70EA9EA4FD88A3F68139A2B00B8473D
:10C5600001282BD0E74920000968884700283DD0E2
:10C57000139800280AD01C206043E3494018007932
:10C580001399884202D11298F8282FD1DF49200050
:10C590000968884764216143049A6F468B1801003B
:10C5A00098699A8B0006000E07C72B00D44F139A88
:10C5B0003F6820000EA9B847012817D1CD486B4627
:10C5C0008678187F401C1877D1480168002908D167
:10C5D00001E0012000E000206B46997F4018987729
:10C5E000BBE01C9888470028F5D0F2E722988088A5
:10C5F000A042F5D064206043049947185F1DB8F34A
:10C600000100000080BE00A000020000A43B1599BC
:10C610003420C05D0028EDD00428EBD01C986423A2
:10C62000584304994018BC491D900968008C8847FC
:10C630000028139805D0002805D01298F828D9D1E1
:10C640001DE000281BD11C206043B449401800792C
:10C65000002814D11D981D99007B497B7A7B4018D6
:10C66000229940088989401E4018397B00048918A6
:10C670004A084A21C95B000C521E511817E01D9848
:10C680001D99007B497B7A7B4018397B40088918CB
:10C69000139A4908002A02D0801C0004000C1C22B6
:10C6A00062439E4BD2181279002A02D0891C0904D9
:10C6B000090C1C9A15AB52009A5A10180004000C71
:10C6C0001A906000185A401800049549000C1990FF
:10C6D0000968200088474037BA88AA4221D3219AA6
:10C6E0001099891A00E049198142FCDB00E0491BDE
:10C6F0008142FCDC1A9A8A18531E834203DB82496A
:10C70000101A8E782AE0199A49198218521E8A4204
:10C710002DDB091A7C4A1A98967808181EE0801AB0
:10C7200002E0109B2199591A8142F8DB00E01018B1
:10C730008142FCDC1A9BCB185F1E874203DB7249E7
:10C74000181A8E780AE0801A199A8218521E8A42A4
:10C750000DDB6D4A081A1A99967840180E996B46A7
:10C76000081A800180090E90187F401C1877012E4E
:10C7700000D1CDE60B2C3BD11398002838D16B4665
:10C78000987F002834D11C992298490015AA515A43
:10C790008089642341181C98049A58436B4680187A
:10C7A000027B407B101840081A8E401E5E4B081812
:10C7B00000041E68000C29000EABB047002817D0FB
:10C7C00001216B461B91197F491C19779A7F012122
:10C7D000022800D0002150186B4698770E991098C7
:10C7E000884205D00F9B421AC01A824200DA0F918C
:10C7F0004E4A05A9126807A890471B98012811D135
:10C800000D98401B06D40F99884200DAF8080E7D77
:10C81000010000007CC000A000020000416C489EA6
:10C8200074E600201B900AE00D9A0F999142F7DD03
:10C83000012189064018F0E71B98002817D10B2C1E
:10C8400018D00023012015AE4100725A002A02D0F0
:10C85000521E01237252401C0006000E0828F3D31A
:10C86000002B04D001201B900D980F904EE61B98D2
:10C870000128D5D029488078002813D0284D0021E0
:10C880002A6807A89047002815D02A6814A905A887
:10C89000904700280FD010AB187C00280BD10698C9
:10C8A000109007E0274B02201B6810AA0CA998479C
:10C8B000012800D10B241F98048020981099016052
:10C8C00023B0F0BD70B50400080016002DF3CFFAB8
:10C8D000050030002DF3CBFA1B4E2D1A0122482003
:10C8E000504380194168002936D02E21095C002967
:10C8F00032D0817EA1422FD1016A691A0906091638
:10C900002AD00562C3695B18C36144231B5C022BF8
:10C9100001D0042B20D119E034FC000420E90004EC
:10C9200038FC0004A0BD000458FC000468FC0004AE
:10C93000B4B4000448F7000490E600049CF300043B
:10C9400030FC0004ACF3000470CA0004036B5B18F5
:10C950000363436B59184163521C1206120E0B2AD3
:10C96000BDD370BD10B530F362FBFF490B68198869
:10C9700000290BD1CA00D21894886404640C9480F6
:10C98000491C0906090E0E29F4D310BDF749497D4B
:10C99000C900C9188A885204520C8A8010BDF8B5A3
:10C9A0000C00C97E00291CD12500403529790729B2
:10C9B00017D1EF4EB178002913D0B169891A10D47C
:10C9C0000127BF02B9420CDA20002DF389F9B169C1
:10C9D0002A79C91C20002DF312FA0120E0760020EC
:10C9E000B1E421002EF3E2FFADE4F8B58446E14D59
:10C9F000DE4CCF7E2E782034002F06D1607A0028BE
:10CA000001D0082000E010208885DB4F387801280D
:10CA100004D1A078002801D0012028705073D6FEE0
:10CA20000100000078C200A000020000B584F623D7
:10CA300060462EF39BFE3978012903D1A1780029A5
:10CA400000D02E7089E470B50400CE4D1000002691
:10CA50002335002909D0FCF7CAFE002801D10126A0
:10CA600007E0218A0020485503E0208A415D491CE7
:10CA700041552000FCF7B4FEC249002804D0207EB6
:10CA8000627EC978801811E0208A1C235843C04A6E
:10CA90000C2380188078BF4A584312688018808819
:10CAA000142807D2207E627E097980184843C00589
:10CAB000000E00E02D20218A495D814200D9012627
:10CAC000300070BDF8B50600B34800250068408FFF
:10CAD000AC4C0006070F318AA0783EF315F8002809
:10CAE0000CD0308AAD49085C052807D1A4483A002B
:10CAF0006038C17D3000FFF7A6FF05000021002D42
:10CB000000D161792800617127E470B505009C4C63
:10CB10004823603CA08AA2495843461829003000A7
:10CB2000FFF7D0FF002803D00020E0750120B0857A
:10CB3000280030F367FE70BD10B530F367F99048F8
:10CB400060388079022812D18E4A907800280ED061
:10CB50008A48006883881721548AC9028B430C4095
:10CB6000234383805079002801D0401E507110BDAE
:10CB7000F8B50E000468E17E00293ED0A78DE56976
:10CB800031002EF3A9FE81480078012803D08548A2
:10CB90000078012831D1E819301A2ED420002DF365
:10CBA000A9F881481823407A7D49584340180B2141
:10CBB000C9014018056A7948298A405C012806D1D4
:10CBC0006F482030C0783DF39FFF00280ED1002D24
:10CBD0000CD0287E697E4018A97E4008002901D12A
:10CBE000361803E0430018188619761C4420A785E0
:10CBF000025D310020002DF30CF9FBE670B55F4DAE
:10CC00002A681488C27E032A0BD1827E002A08D1AA
:10CC1000664A1278002A04D162040123520CDB0315
:10CC2000D41830F325FD2868048070BD22126E737D
:10CC30000100000074C400A000020000AC7C285376
:10CC4000F8B504001C23808856495843401845799C
:10CC500000202CF330FE28216943405C01281FD1BD
:10CC6000E088A66857493018877809686801401835
:10CC7000C18A008B081A544940183DF374EA2D20EC
:10CC80000001401A0004000CB84209D24F48C069A4
:10CC9000002805D04E4A3100126828009047B3E6BC
:10CCA00020002CF3DDFBAFE631B582B00298002402
:10CCB0000168FF39F7391CD0464A89181FD1858889
:10CCC000280016F315FF0078C00718D04249280045
:10CCD00009688847002812D00820FAF2F7FA3F497D
:10CCE0000190016085803E48016801A8FAF2FDFAD2
:10CCF00005E0FFF7A5FF012402A8FAF2EAFA2000F6
:10CD00003EBD70B505000C0004D13448290009303F
:10CD10002BF347FC2100280028F338F91E4A012193
:10CD2000107AA9408843107270BD3EB504000D0012
:10CD300008F31FFD882161436B460818017D29A077
:10CD400023C30022284B110020001EF35DFC3EBDD2
:10CD500038B504001020FAF2B9FAFF2143310090EF
:10CD60000160011D200023F390FE19F368FB1F49A9
:10CD70003DF3CCEA0A00E1001D48091949010818F1
:10CD80000400FF30401C426120000099653031E012
:10CD900028EA000430D20004BC5C00B0D5EA0004EC
:10CDA000D7EA0004B4B4000498EA000484EA00045A
:10CDB00024EB000470CA0004D8EA00042CEB000441
:10CDC000C5EA00046CEA0004D202000008D700049F
:10CDD00008F7000464F5FFFF14F60004BB0C000024
:10CDE00000AA3400696200007F1F000040420F006B
:10CDF000E0BD0004CA6004220C313DF38AE80099CA
:10CE00002000553004220C313DF382E8FF480168D0
:10CE10006846FAF26AFA38BD10B52FF36CFFFC4889
:10CE20000078012812D1FB4800680188090909012E
:10CE3000491C0180F84B9978002907D0ECE22DDDE0
:10CE40000100000070C600A000020000589496EE99
:10CE5000818817225B8AD202914313401943818053
:10CE6000F3493220087210BDF14910B589790229C1
:10CE700002D1EF492039886130F3A9FB10BDF8B524
:10CE800006000F0008F37FFC05003900300005F3B1
:10CE90007BF9040001281AD13068572817D1E54AD8
:10CEA0003900126830009047012810D13888882353
:10CEB00058434019C08D002800D10B200EF34FF9C4
:10CEC000002804D0DC49300009688847002420008D
:10CED000A4E5F1B584B00326049805680AF314FCB0
:10CEE000070008F350FCE979020001204B082B2BC6
:10CEF00000D100200190C807C00F0290A8888823A5
:10CF0000039058438418E08D002802D008380604A6
:10CF1000360C5D20C05D012805D01E207043C0196D
:10CF2000C07801284FD1217D029881424BD0A87D45
:10CF3000002803D0C14803992BF33DFB01982B2215
:10CF4000002801D0BD4A6732A1780D2001290DD1FA
:10CF50000199002901D1297A00E0697A1E237343DF
:10CF6000DB199B798B4208D00A2006E0217D00293D
:10CF70000BD16178012900D123200306029903987F
:10CF80001B161EF323FA05B0F0BD012174200155D4
:10CF900004980068206704990020086060780128E0
:10CFA000F1D11E2171433720C9198978012904D193
:10CFB00001993620002900D03920A14B0399002285
:10CFC00011F3EEFFDFE704980DF36EFDDBE710B51C
:10CFD00004F322FA95490020887310BD10B50400AF
:10CFE00018F3FAF9200027F3B7FB10BD70B50B1D3D
:10CFF0004A88D204920D9A189278D20725D0914B84
:10D00000122242431C68A35A5B071ED58E4D14237F
:10D0100043432D685B19DD88002D16D11D89002D35
:10D0200013D15D89002D10D1A55AAE077F4D07D4CD
:10D03000A35A02263343A352AA8A521CAA8204E0AE
:10D040000122DA80EA8A521CEA8217F3C9EDD8ED90
:10D05000010000006CC800A0000200009F8D94B386
:10D0600094FE70BD38B500247D4A0168891808D146
:10D070008088082805D200221100130000921BF3BB
:10D080003FFC200038BDF8B504000D00160000205C
:10D0900016F342FD070032002900200027F334FE7A
:10D0A000032D15D12000FDF7F1FF002810D0382006
:10D0B0006043C019006A00280AD01C216143694AF4
:10D0C000012089188978654A1423594312685052FF
:10D0D000AEE4F7B598B00500002016F31DFD1C2145
:10D0E000694304905F48081817900679E8005E4984
:10D0F00040194001441827008037F87C002806D1E9
:10D100001A9A1999280024F3F8FE1BB0F0BD002EDE
:10D1100006D1002014900EA819F300FC0CA905E01C
:10D12000012014900CA819F3F9FB0EA9280023F391
:10D13000C0FC00206B461875B87B002800D0012089
:10D140006B46220058757D32484F2300169200929C
:10D150003F682D3320000CAA0EA9B847200060308C
:10D160001590408B1021081A07063F0E04D005A821
:10D170003900801C3CF3A6EF15981A22825E7800D5
:10D1800005A940181699801C3CF3D6EE210009A889
:10D1900098310822801C3CF3D0EE35486B4600786D
:10D1A0001875280023F3FBFC05AA0092149A0021AD
:10D1B000280001231BF3A4FB002E0DD11998102287
:10D1C00010A901AB07C32BA2009201220021280065
:10D1D00011231EF32DFA98E72800FDF757FF0028CA
:10D1E0000ED03821694304980818006A002807D037
:10D1F00017991A4A8978012014235943126850520A
:10D20000199811220106091628001EF3DEF87CE7A2
:10D210007CB50C001500A67E079A0699002E2DD12C
:10D220004426365D092E03D0062E01D0052E25D1C9
:10D23000012921E0F4E70004CBEA000428EA000415
:10D24000BC5C00B0D0D10004A0F90004CCF900040B
:10D25000180C0000317F31005CEA00048AC576E1D9
:10D260000100000068CA00A0000200006B652A0EE1
:10D2700060EA000407F4FFFFB4B40004E0BD00045A
:10D2800050FD000454E90004696D000000D1022142
:10D29000019200912A0021002DF346FC7CBD38B597
:10D2A00004002AF301F8A188012088405F49097A27
:10D2B00008420DD00820FAF227F8FF2188310090AB
:10D2C0000160A18881805A4801686846FAF22BF80B
:10D2D00038BD70B504000068564A016800258918F9
:10D2E00008D1FFF7DCFF20680125002802D02000CC
:10D2F000FAF20DF8280070BD10B526F30DFE4B496B
:10D300000020C87210BD08212030417370474A497F
:10D3100038B505000968884700282DD0434CE07ACD
:10D32000002829D1E8004549401940014018807C77
:10D330000025002803D1607A401C60720AE0A07AC0
:10D34000401C0006000E0328A07203D1607A401C26
:10D350006072A572607A03280ED10420F9F2D4FF1E
:10D3600037490090016065720120A572E07235486E
:10D3700001686846F9F2D7FF38BD10B5040024F300
:10D3800027FA2000FFF7C3FF10BD10B5040024F3F7
:10D3900077FA2000FFF7BBFF10BD10B5234904004A
:10D3A0000120097AA040084288B01FD004A823F3C6
:10D3B000D4FB200008F31AFCE000204B00194001C8
:10D3C000C01840308078102204A901AB07C31EA208
:10D3D000009201220021200041231EF333F91B4A51
:10D3E000072112682000904708B010BD200028F3E4
:10D3F00061F8F9E7FFB581B01E00070002980A281E
:10D400000CD10A4D0124287ABC40044206D003986E
:10D4100010213CF362EE287AA0432872039A029905
:10D420003300380028F3E5FBC1E50000BC5C00B028
:10D43000F4E700045DF0FFFF94F60004E0BD000493
:10D44000A90F0000D0A63400696D000090F600041A
:10D45000012B10B50BD0042B07D127483DF337F82B
:10D46000002220212548F6F2A1FA0020C98443C3F6
:10D470000100000064CC00A000020000729DF47E58
:10D4800010BD24483DF32DF800220121F4E74B297B
:10D4900010B504D11E4800224021F6F291FA002076
:10D4A00010BD70B51C4D6C68A00706D51848002249
:10D4B0000421F6F285FA02206860E00706D01448DD
:10D4C00000220221F6F27CFA01206860286B01211B
:10D4D000090608432863002070BD10B50F4C1048A2
:10D4E000216881600021016141618161C1610D4953
:10D4F00001620D4941620D498162F9F2F5FD002199
:10D500000BA0F9F23CFE606010BD0000642101B088
:10D51000782101B0502101B000F003A9805D00B076
:10D52000B4EF00B049CC000073CC000087CC000001
:10D53000626C656D6278000013B50C00FF490098BD
:10D54000CA7E032A02D0897E012904D11C380090AA
:10D550003CF312FF1CBDFA4A0168914210D1407998
:10D5600013280DD1F54A3F23203A108F1B020100EA
:10D570008004800E401E80069943800C0143118771
:10D58000F5F744FB21006846F9F2D7FE1CBD10B543
:10D5900004000022EB480A21D2433CF317FF002885
:10D5A00016D001890022081882710E21C27104234D
:10D5B0000172437201238372230AC4720373E04B26
:10D5C00042730360417102710A22C280FFF7B4FF07
:10D5D00010BDDD480022082110B5F6F2F1F910BDAA
:10D5E000DA487047142170B54143D44D1423203DCF
:10D5F0004919096958430A891F23521814682A00D7
:10D60000801800691B030289298F1218D0880F2601
:10D610000005000D98435379FF3CDB06DB0B1843F4
:10D620001F235B04984313797606DB069B0A184395
:10D6300007239B059843CB07DB091843C000012350
:10D64000C0085B07C018653CB0430832002C05D009
:10D65000BF4BE31805D101239B0601E001235B06C4
:10D66000C0188B089B008907A86000D15B1CB949D2
:10D670002B870A62086100F0A1FA70BDDD97EB1AF2
:10D680000100000060CE00A00002000086754AC3C1
:10D69000AF49002230B41000F02520390C8F14233C
:10D6A00043435B189B69002B05D0401C0004001409
:10D6B0000228F4DB04E0022802DAAC430C870EE017
:10D6C0000820C441400620181824E04104060B003D
:10D6D000240F072C088702D9A843012218870120AC
:10D6E000801A0C8F00040014A204920E22E014236E
:10D6F00043435B189B69002B19D0002809D1102ADD
:10D7000015D20E22D44101229206A2181223DA4128
:10D710000A870A8F0C239A4383071B0F1A430A8731
:10D720008B4905220004CA7630BC000C64E7401E19
:10D73000000400140028DADA30BC7047030570B525
:10D740000120834C1B0D00068343203C208F0907DA
:10D75000C507ED092B43DB000325DB086D075B19CB
:10D760000F256D06AB43C9080B438108890080076C
:10D77000A36000D1491C7C4821870262036100F04C
:10D7800027FA70BDF8B5724CA07E2500203D002818
:10D7900010D0E07E03280CD00320E0760220A07693
:10D7A000288F724900228843288703211000FFF741
:10D7B000C5FFF8BD28686E4F0126002819D1402109
:10D7C0006548002200913CF30BFE00280FD0417BFE
:10D7D00031434173876101890A18101D28600620B2
:10D7E000E0760098121D0121FFF7A8FF0120002814
:10D7F000DFD1686800281AD100225E4811003CF38E
:10D80000EFFD002811D01421C180417B31434173C9
:10D81000242187610181243006216860E1760200BD
:10D820000221C801FFF78AFF01200028C1D1E07E54
:10D830000428BED1A8680028BBD1FFF729FFF8BD96
:10D84000F8B50024484FBD6941482038C5607E6A5C
:10D850000100098F01239B038C466A0F9943022A1A
:10D8600013D0032A07D162461A43EB001B0F082B83
:10D8700000D00A0002877D6100F0AAF93448C07E1A
:10D88000042801D1FFF77EFFF8BDEA00DA66D9224D
:10D89000010000005CD000A000020000F86EED73F3
:10D8A000130F3CF360ED0504040A0A04100002683B
:10D8B000B24208D10022026004E04268B24202D1C2
:10D8C00000224260012401877D6100F08BF9002C69
:10D8D000DED0300000F0A1F90028D9D0A902C90E8D
:10D8E000FFF73EFED4E7410F70B5032919D11D495A
:10D8F000C400CA7E230F012A14D00425022A1DD099
:10D90000032A0ED10A00927E0024032B1AD0042B86
:10D9100007D1032A05D18C76CD7600F04FF9FFF7B9
:10D920003BFF70BD052BFCD10220C876F8F706FB43
:10D9300016494000085A0022062112E0200FF0D1BB
:10D94000CD76ECE7074B203B9D688542E9D1022A62
:10D95000E7D1032088769C6000F099F90022042129
:10D96000100015E004F000B00C14000068C800B00E
:10D97000782101B0B7CD000059EDFFFF00F003A9F9
:10D98000F03F0000C5CD000080C800B000000004DA
:10D99000FFF7DEFE70BD70B5060014204843D34A81
:10D9A0008518103524E0D1492031CB7E3CF3DAECE8
:10D9B00008050808050D080814053CF3F1FC17E0FC
:10D9C000010028003CF3A1FD12E0010028003CF317
:10D9D0009CFDFFF7E1FE0BE00189091808314A7947
:10D9E000097914020C433CF3DBFC2000FFF7E3FD54
:10D9F00030003CF361FD0028D5D170BDBB4810B5A7
:10DA00002030C07E042801D1FFF7C6FE012010BDE2
:10DA1000B64A10B52032D37E002B07D0937E002B60
:10DA200006D101239376FFF7E9FF01E000F0C6F885
:10DA3000012010BDAD4810B52030C07E002803D0B5
:10DA4000072801D0FFF706FF012010BD70B50120A7
:10DA5000A64CA74D2034E37EA44E3CF384EC071E75
:10DA60000505051E09121E00E869FFF73CFF14E0DA
:10DA7000E969B2688A4204D1308F0007800F00F054
:10DA8000BAF8E969002808D0B068884205D10420B6
:10DA9000E0760020B060FFF77FFE0120C7B2830C64
:10DAA0000100000058D200A0000200000C8653CEF6
:10DAB00070BD9548012110B5FFF777FF012010BD1B
:10DAC0009248002110B5FFF770FF012010BDFEB590
:10DAD0000020471E8E4E01908E4801227F2101AB0F
:10DAE0000097F5F2FBFE00240EE0E1007258891960
:10DAF0004D68284204D0002A02D000210800904737
:10DB00000198A843641C019001980028EDD1E3E737
:10DB10007B4870B52030C07E01242200042800D14B
:10DB20000022774D00212000002A06D114224A430A
:10DB300052199269002A00D10020491C09060200EE
:10DB4000090E0229EFD3002A16D1714E083E317812
:10DB500000290AD07068F4F756FD7D21C90088427B
:10DB600001D2012000E000203070002802D1288F6F
:10DB7000400403D5002C01D0012100E00021200049
:10DB8000002900D0002070BD70B500255C4C203409
:10DB9000E576F4F7CFFA5B480123E376016B0322C5
:10DBA0001202914301635C498A680824A2438A6097
:10DBB000426B1A4342638A6822438A6057498163F1
:10DBC0005048403041689A0411434160856070BDFF
:10DBD000534810B5046800225248D24310213CF348
:10DBE00013FC002807D001890818FF216331016068
:10DBF0002100FFF7BFFC10BD10B5F4F700FD44494C
:10DC0000083948600120087010BD142358433C496E
:10DC100010B5401810300024002806D03CF356FC04
:10DC2000002802D03CF3C6FB0124200010BD34497B
:10DC300010B5CA683C4CD1000B0F010008393CF309
:10DC40009CEB0509041422092E00001FFF216431FA
:10DC5000016010BD0179001F046041711102890F3C
:10DC600001711105090DC18010BD437802781B02B6
:10DC70001A438378C078000203432B48401C086095
:10DC80008A80CB8009E0037810020C60800F4B7112
:10DC900008711005000D001DC880080010BD00208F
:10DCA00010BD70B50025164C20680028D9D03CB0B6
:10DCB0000100000054D400A000020000157E8DBEBB
:10DCC00003D020383CF380FB25606068002803D037
:10DCD00024383CF379FB656000242006000EFFF732
:10DCE0009EFF0028F9D1641C2404240C022CF4D3D8
:10DCF00001E03CF369FB09483CF3F2FB0028F8D152
:10DD000001E03CF361FB06483CF3EAFB0028F8D154
:10DD100070BD0000E4EF00B000F003A9502101B095
:10DD2000642101B0905D00B0782101B080210080B5
:10DD30001E1E0000E4A6340068C800B00C140000E9
:10DD4000F8B50500FF4C607A1AF32DFD060014208B
:10DD5000F9F20CFBFC4900900160FC4909898180C3
:10DD60008572217A8173068261894182F84801684F
:10DD70006846F9F20AFBF8BDF8B5C021F54C2068F9
:10DD8000020060325181EF4E0123317BDB0200291A
:10DD9000818B01D0994300E019438183EE493378A8
:10DDA0000968DD0900D1CB81B378DD0900D14B8250
:10DDB000EA497379FF27E54D09787F1C002B0FD1C5
:10DDC000838B3B438383B079F37940180002591861
:10DDD000084310816020A871216800208884F8BD64
:10DDE000828BBA438283C183D649DD480A22006808
:10DDF00015313CF3DEE85020EDE7DA49D34810B5A1
:10DE00000968083086B08847D04C1C2120894143DE
:10DE1000D5480818817861714178E17000792071E6
:10DE20000001C121C9010843D049096808800120C7
:10DE30002AF30CFC01A818F3ADFD01A903A818F3FF
:10DE40002AFD2079CA490C23584309680C2240183E
:10DE50004C3003A918F37AFBC64A207913680021D5
:10DE6000400119521368C3185980126880188181C3
:10DE70000A21818006B010BD70B5F8F79CFEB54C44
:10DE80002068418CCD2211404184F9F253FBBA48FD
:10DE90000068818C090B09038184F9F257FB206823
:10DEA0000021FF30E1304181FFF7A7FFFFF764FF5A
:10DEB00000F0ADF9A3480079FFF742FF633197788E
:10DEC0000100000050D600A000020000E1963303DC
:10DED000A34D01246C7000F082F900F025F92C703C
:10DEE00070BD1CB59E4AD268019200900021FF20AF
:10DEF0001923A7A2FBF27BFC1CBD70B52BF3AAFE75
:10DF0000A4480022006842710123C370A24C100093
:10DF10002568C1006B52256849194A80401C0E28AB
:10DF2000F6DB2BF39FFE70BD70B58D4C607800253D
:10DF300000281FD06570FFF7E0FFF9F205FB934E54
:10DF40003068418FFF22913291434187F9F2FCFA08
:10DF50006079316840000A5AC0239A430A52F9F2A4
:10DF6000FFFAF9F2FDFA00F08DF9FF20FFF7F2FE5B
:10DF7000F8F72DFE257070BDF3B50C0081B0784F19
:10DF80007878002804D02079FF2801D0FFF7CCFF53
:10DF900021797148FF29017109D17878002804D0CE
:10DFA000FFF7C2FF0120FFF79CFF0020FEBD217894
:10DFB000017061784170A1788170E178C170217938
:10DFC000017161794171A1798171E179C171217A20
:10DFD00001720091657A4572E17AA67A09020E43D0
:10DFE0004681217B0173019912290CD3A27B617BAD
:10DFF00012021143E27B237C12041B061A431143D5
:10E000000161617C02E00021016104210175524837
:10E01000019915301C2905D321000A2212313BF346
:10E02000D2EF03E0FF220A213BF3C4EF002E07D01A
:10E030005A496800085A864202D800980E2801D929
:10E040001220FEBDE806C00FB870FFF71FFFACE757
:10E05000F8B5534D2868C48F008C002801D01CF3FC
:10E06000C5FF3F4FE00629D52868468FF0050BD540
:10E07000F868401CF86038480069002804D0F96846
:10E08000884201D80220387030060DD53878022831
:10E090000AD1FFF732FF3D480068418FFF228132ED
:10E0A0009143418703203870F00607D5387803285C
:10E0B00004D1FFF739FF0020FFF713FFA00611D5A9
:10E0C00029684020405A80050CD07879D99D954424
:10E0D000010000004CD800A000020000268F315E35
:10E0E0004200895A002907D00A06920F04D0324A0A
:10E0F0000906126809169047600601D52868C08C89
:10E10000E00508D52968002042005218528E401CB4
:10E110000328F9DB088F200607D529680020420074
:10E120005218128D401C0528F9DBA00501D528687E
:10E13000C08B600501D52868408CF8BDF8B52BF37D
:10E1400093FD1948002100684171084B197AC1708C
:10E150000849FF278A79002015022E000A79133614
:10E1600011353F1D114C4979920327E020F000B092
:10E17000940C0000C85D00B0FCA9340084EA0004DF
:10E180008CEA00041FE90004A8EA0004E8FB00048C
:10E19000B4B4000480EA000488EA000478EA0004C9
:10E1A00034EA00046262770020EA000428EA0004EE
:10E1B00080A9340038EA0004ECF400040A43120495
:10E1C000120C0FE0002802D121680E8002E02368C3
:10E1D000C1005D522368C100CB185A802368C9185A
:10E1E0008F80401C4049097A8142EBDC2BF344FDCF
:10E1F000F8BD10B53D4C0120617988403C49096863
:10E200006031C883F9F2AAF90020E060F9F2A6F9BA
:10E210006079384C400021680A5AC0231A430A52D8
:10E22000F9F2A8F92068418FFF229132114341870A
:10E23000F9F2A0F910BD304810B5026813882B4CD4
:10E240000121607981400B431380A2782B4B002A77
:10E250001A68148801D18C4300E00C4314801968BB
:10E260000A8823490968FF3181310A821E4A142134
:10E2700051560C220C2900DA0A001321C9438A42A4
:10E2800000DD1100490029310906090E442900D397
:10E29000432113F072ED10BD10B5144C1848E1780D
:10E2A00018F34FF86179174818F34BF820890106E5
:10E2B0001548090E18F345F8218900201C235943FD
:10E2C000124A50540C480068028863790121994031
:10E2D0008A4302800948006802888A4359E93EA4BB
:10E2E0000100000048DA00A000020000D2678FE3BE
:10E2F000028002888A43028010BD000020F000B036
:10E30000C85D00B084EA000434EA000430EA000486
:10E310001CEA000488E8000484E8000480E80004A3
:10E32000B4B40004020010B5937811203CF34CE81B
:10E33000081B05080E0B1114171B10001C4A10E0D7
:10E3400010001C4A0DE010001B4A0AE010001B4A96
:10E3500007E010001A4A04E010001A4A01E0100019
:10E36000194A1268904710BD70B506001078140065
:10E37000E02886B004D12000FFF7D4FF050000E0BC
:10E3800011250021481EFBF25DFB2279E178A0787F
:10E3900003AB07C33300627821780191FF21029219
:10E3A00021310E2009A20095FBF235FA06B070BDAE
:10E3B0000CF9000410F90004FCF8000408F900044A
:10E3C00000F90004F8F8000404F9000452686262DD
:10E3D0006262626200000000F8B50D000021009149
:10E3E000382116004143FA4A8C180021F9F75BFEE8
:10E3F00000282AD0607DC11C8A07411C80000019BA
:10E4000083698907920F890F002B0AD1876A002F31
:10E4100007D1920012199769002F02D1926A002A3F
:10E4200001D001220092002D08D0002E06D02A68CB
:10E43000D2182A603268806A101830600022880082
:10E44000001982618262A27561750098F8BDF8B505
:10E4500038235843DE4B8E7AC418C87A4B7A0002B0
:10E460000643087A1B0218438446E07C257C042876
:10E4700001D3002D75D108795700022805D0032853
:10E4800031D006287BD1002055E0002102206174A4
:10E49000009008256046112806D0132804D01928BA
:10E4A0006FD101250095A174207C002804D138216A
:10E4B00020003BF338EE0FE000208100625A002A72
:10E4C00005D109194988002901D1207504E0401CB3
:10E4D0000006000E0428F0D3207D81000819C653E1
:10E4E000257400984AE0207D800003198F5A2BBBC9
:10E4F0000100000044DC00A000020000CB9F51930B
:10E500000120002A00D000204000185AB04240D11B
:10E510000222012D05D12274012262740022A2740C
:10E5200004E0082D02D1092020746274087B0028C1
:10E5300005D1487B002802D1E07C401CE074217D9D
:10E5400060468A001119C85323E081000B19D95B7A
:10E55000B14211D10121002A00D000214900595AAD
:10E56000614509D18200111900220A804A80E17CAC
:10E57000491EE17405E016E0401C0006000E042868
:10E58000E3D3002805D1082D05D0092D03D0207430
:10E590006074002D08D0207C002805D1F5F768FEB6
:10E5A0000020F5F75CFEF8BD607C0128FBD1F5F793
:10E5B0005FFEF8BDF8B5002406008A4F2500002153
:10E5C0002800F9F77AFD00281AD0002E03D1641C28
:10E5D0002406240E14E0012E08D138206843C01907
:10E5E000007C0128F3D00228F1D009E0022E07D1E7
:10E5F00038206843C019007C0828E8D00928E6D0F4
:10E600006D1C2D042D0C082DD9D32000F8BD002041
:10E61000D0E71CB5002074490190009004000870F8
:10E6200020006A4601A9FFF7E1FE002801D000F0B2
:10E6300003F9641C2404240C082CF1D300990198DC
:10E64000F5F728FE1CBDFFB583B0050008285CD295
:10E6500038236B43634892071C18677CA07C0290A8
:10E6600048780E780002CB78064388781B0218435E
:10E67000920F012A49D0069A012803D0280000F001
:10E68000E9F802E02800FFF7ECFE607C2A00310088
:10E69000FBF702F806980028607D05D0800000197D
:10E6A000816A8919816204E08000001981698919F1
:10E6B000816100F0C1F8607CB84208D1002824D004
:10E6C000012822D16B46A17C1A7A91421DD00128E3
:10E6D00001D1012600E000260127022800D00027F2
:10E6E0000C20F8F26BFE4149019001608580867133
:10E6F000A17C0172C7713E48016801A8137BA2A6E4
:10E700000100000040DE00A0000200003F77EF2E75
:10E71000F8F26DFEA17C607C2A00FBF734F807B0AC
:10E72000F0BD70B5040008281CD2002211002000A2
:10E73000FFF766FEFFF775FF00280CD12F4D2878F4
:10E74000002808D03048002129F3E9FF002001000B
:10E750002870F5F7A9FD3820604327494018382173
:10E760003BF3F4EC70BDF0B500263821414387B08F
:10E77000214A05968A18162104960296019600925F
:10E78000515635003700002901D00E0051E000211C
:10E79000F9F79DFC00284CD00024009AA0008218B4
:10E7A000906901231900002800D00021C9190F0623
:10E7B000916A3F0E0029069100D000230199049A26
:10E7C00059180906090E80180191059B002159412D
:10E7D0000490029A06980591801800214D41641C0E
:10E7E0002406240E042C0290D7D3022F0ED30198B6
:10E7F00002280BD300261AE040F000B0D85D00B02C
:10E80000120D000000AA3400F3130000029A0498CD
:10E8100005992B00121A8B4101D2012607E0029ABA
:10E8200004980599801AA94101D20026F643009860
:10E830008675300073E70100382359432C4A0120C4
:10E840008918497C022900D000207047294810B55A
:10E850000178002907D1012101707D20264900227D
:10E86000C00029F349FF10BDF7B53823009858437D
:10E870001F4BC518C8788B7800020343287C0128F9
:10E8800007D0022805D0082801D0092803D1022486
:10E8900002E0012400E000240120002A00D0002032
:10E8A0004600A85B984206D1012C6C7402D101206D
:10E8B000F5F7E8FCFEBD012081004919895B99420A
:10E8C0000FD1012C6C74F5D10220002A00D1012057
:10E8D000A874FAF773FFA97C009A2000FAF753FF97
:10E8E000FEBD401C0006000E0428E5D3FEBD00005E
:10E8F00040F000B0D85D00B0F31300002E4810B512
:10E90000006800224B21F8F2E0FC10BD71192FCEF7
:10E91000010000003CE000A00002000037A81EF348
:10E92000FFB581B006000D003C292CD82F00093717
:10E930003806000E30F312FC040024D0208924494C
:10E94000001901600021017122492A000968417102
:10E950001F49C78008307839016086808571039926
:10E96000C01D3BF362EB194800220068210001231F
:10E970003BF3DEFD0498002803D100210120FEF2C4
:10E98000E6F805B0F0BDB30512219B0DB20A0420D4
:10E99000FBF206F8F5E7FFB581B0050016001F0091
:10E9A00030F3DCFB0400ECD02089FF210019653135
:10E9B000016007714671C58002992A0008303BF357
:10E9C00034EB200030F3D0FBDBE70000845D00B0C7
:10E9D0000A140000E4A63400F8B5002406008038CC
:10E9E000864B87490004000C1A5C0D88854F52192C
:10E9F0000A801C5411E0A0003D58A8880005000DB5
:10EA0000B04207D11C3D2000FAF2F7FB28003BF38F
:10EA100017FD02E0641C2406240E7B480078844223
:10EA2000E9D3F8BD10B5C178827809020A432438C9
:10EA30001C21431801817549C16103211971744971
:10EA400009685971111D418401007248042300684E
:10EA50003BF36EFD10BD70B504000D000020F8F70B
:10EA600013FB052D19D1E188A088091D0A046A4904
:10EA700000050978000D120C002912D00100803920
:10EA80003F290ED85E4B1988491E19805B4908182A
:10EA900080380178491C017003E0E088001F0204FF
:10EAA000120C5E48210000681C392B003BF340FD2E
:10EAB00070BD594930B40978002903D050490988FC
:10EAC000002903D05649096830BC08474E4A4D4CCE
:10EAD00011788B00491CE050117030BC704770B544
:10EAE000474C2588FFF778FF4E4A20881388411B42
:10EAF000C918401A1180208070BD10B580242000F4
:10EB0000641C2404240CFFF767FFBF2CF7D910BD49
:10EB10001CB5454A1178002912D0917895F6A8DDE8
:10EB20000100000038E200A000020000C340A04E37
:10EB3000D2786B461A7058700A0A9970DA700A0C0B
:10EB40001A71090E59713E4C0300062120006A46D5
:10EB5000FFF7F0FE1CBD0006001610B513F042E9E9
:10EB60000020FFF7DFFF10BD020035480A21801C9E
:10EB7000012310B5FFF7DEFE10BD10B52F4C6070FD
:10EB8000A170E27001206360207010BD00B589B0F3
:10EB900000906B462B481971006800230206120E84
:10EBA00024206946FFF701FF09B000BDF0B504005D
:10EBB000241D6179257909020D432349234B0E78E1
:10EBC000216800200222994221D130207043204B3D
:10EBD0000021C6180F0048004018A31830181B79F0
:10EBE000521C12048370120C01238B402B4205D05F
:10EBF00005230370114BDB78437002E00770477008
:10EC00008770491C0906090E1029E4D30120F0BDC4
:10EC1000A09D0004A8E50004E09D00049CE500041C
:10EC20000B140000E0A63400845D00B09BE50004F6
:10EC3000880E0004B0E50004AAE50004DC5D00B025
:10EC400087FC0000E4A63400CD5B00B05321000037
:10EC500000F200B0010000220C48D243083110B588
:10EC60003BF322FC10BD10B5040000681C383BF3D8
:10EC7000F1FB0020206010BD0100054810B50068C0
:10EC8000002201233BF35EFC10BD000068C800B009
:10EC9000845D00B010B52A4C2848208004F096FF0F
:10ECA00060602648401C208105F015F82100C860EE
:10ECB00010BD31B50098002819D0214D00240098CE
:10ECC000E1006A5A83889A420ED149194B68002B99
:10ECD0000AD081790022C01D9847002804D06846D8
:10ECE000F8F28DFB012038BD641C022CE7D3002014
:10ECF00038BDFFB581B00C0007000498114D4618CF
:10ED000030000F30F8F278FB0028009014D0056036
:10ED100007724672039922000A303BF390E900988B
:10ED2000049A00190A990A303BF388E9009B15BE42
:10ED30000100000034E400A000020000DAB87E3ECA
:10ED4000064801686846F8F270FB012005B0F0BD86
:10ED500080FE000060F200B09C130000E0A63400CA
:10ED600030492F48086031482F49416031493048C7
:10ED700008603249304808603249314808603349F8
:10ED800031480860334932480860344932480860E5
:10ED900034493348086035493348086035483449B8
:10EDA00001603549364A416034491160364A354977
:10EDB00011603649C160364901613649374A4161BF
:10EDC00035491160374A36491160384A3649116071
:10EDD000384A37491160394A37491160394A384948
:10EDE00011603A4A38491160394981603A493948D5
:10EDF00008603A483A4908603B493A4808603C494B
:10EE00003A4808603C493B4808603D493B48086037
:10EE10003D493C4808603E493C4808607047000056
:10EE20009C5E00B078ED000450F500B070DC00048A
:10EE30002134010000EF00041934010004EF000444
:10EE4000813D010008EF00040F3E01000CEF0004BB
:10EE5000793F010010EF00048B3F010034EF000404
:10EE60003140010030EF0004CF3F010014EF0004F7
:10EE7000233A0100E45D00B04B3A01003B3B010046
:10EE8000F4EF0004793A0100BCEF0004613801009E
:10EE90009D3801003B3D0100DB380100DCEF000440
:10EEA000B1360100A0EF0004094101008C5E00B002
:10EEB00077410100985E00B0905E00B068ED0004FC
:10EEC000AD41010074EF00042544010070EF00041F
:10EED00043430100785E00B06CED00047C5E00B03E
:10EEE00070ED00048144010020F00004854401001D
:10EEF00058F00004A34401005CF00004EF45010059
:10EF000060F00004014101002CF000045D470100A5
:10EF100050F00004374936480860384936480860E0
:10EF2000384937480860394937480860394938480E
:10EF300008603A49384808603A493948DA2D521B86
:10EF40000100000030E600A0000200002E50C08347
:10EF500008603B49394808603B493A4808603C49E9
:10EF60003A4808603C493B4808603D493B480860D6
:10EF70003D493C4808603E493C4808603E493D48A0
:10EF800008603F493D4808603F493E4808604049A5
:10EF90003E48086040493F48086041493F48086092
:10EFA0004149404808604249404808604249414858
:10EFB0000860434941480860434942480860444961
:10EFC000424808604449434808604549434808604E
:10EFD0004549444808604649444808604649454810
:10EFE000086047494548086047494648086048491D
:10EFF000464808604849474808604949474808600A
:10F0000070470000B0F900B008F20004885F00B05B
:10F010000CF200049406000410F20004B006000490
:10F0200014F20004AB7001009CF100047B48010065
:10F03000B0F10004E7480100B4F10004D7BA0100C0
:10F040001CF20004B1BB010020F20004B5BA0100BB
:10F0500018F20004BBB9010054F10004ABB8010080
:10F0600050F2000405B301006CF20004F9BC010089
:10F070002CF20004E1BD010094F2000415BE010071
:10F0800098F20004A5BD01009CF200041DB7010028
:10F0900064F20004655B0100F0F20004AB5B010068
:10F0A000F4F200043B63010014F300046763010001
:10F0B0001CF30004756501002CF30004D765010002
:10F0C000F8F200046F66010024F3000491A001002F
:10F0D0004CF300043BA1010068F3000491A101007E
:10F0E0006CF30004AFA1010074F30004C3A101009C
:10F0F00060F30004934600B084F0000475AD010095
:10F1000088F00004C5AC01008CF00004B5C7010014
:10F1100078F3000417C001007CF3000435B001004F
:10F1200080F3000410B50FF080F9012000F0F5F82D
:10F1300010BD7F4A10B551880B00034209D08143AE
:10F140007C485180014202D148084000F1E0046A45
:10F15000010000002CE800A000020000E949C2DE26
:10F1600050800BF078FE10BD0120ECE7022010B5B6
:10F1700000F0DDF810BD0220E5E7042010B500F036
:10F18000D6F810BD0420DEE701204002DBE70820AE
:10F1900010B500F0CCF810BD0820D4E7102010B551
:10F1A00000F0C5F810BD1020CDE7202010B500F00C
:10F1B000BEF810BD402010B500F0B9F810BD6020B9
:10F1C000C1E7802010B500F0B2F810BD8020BAE78A
:10F1D0000120800210B500F0AAF810BD01208002C5
:10F1E000B1E7FFB581B01600994200D919000D00B2
:10F1F00054480021554F0C00818013E0305D0028F9
:10F200000DD0019821000BF0F3F881007A5C824266
:10F2100005D14C4AC9199088498808439080641CDC
:10F220002406240EAC42E9D30BF015FE05B0F0BD68
:10F23000444908707047434800787047414A00B518
:10F240005288002103003BF306E90A06080A0D0F65
:10F25000060D1113211402210BE0042109E0012104
:10F26000490206E0082104E0102102E0202100E02C
:10F2700040211000084000D00120114000D00121A1
:10F28000002803D0002901D0012000BD002000BDCE
:10F290002C4841880020CA0705D02B4A114202D0D1
:10F2A000002900D00120704770B50025FFF7F0FF5E
:10F2B000002812D00024012120000BF020F9092899
:10F2C00005D0FFF7BBFF002801D0012504E0641C36
:10F2D0002406240E0A2CEED3280070BD19480B21F9
:10F2E0004088C901084000D0012070471548408877
:10F2F000C005C00F7047134840884005C00F7047D5
:10F300001349012010B588711248007806280DD1E4
:10F310000C484188090609D50078012806D10E4914
:10F32000096888470D4980200968884710BD054A4B
:10F3300010B5518803008B4303D0014351800BF07B
:10F340008AFD10BDFC5D00B07E02000004030004D5
:10F35000455F00B0365F00B0D4F20004DB3E140C11
:10F360000100000028EA00A0000200001DA17C634B
:10F37000D8F20004FF480021FF2201704270817022
:10F38000C170017141714173012181737047FA4865
:10F3900010B5006800248047F6498878002808D016
:10F3A000072809D14879042806D10EF08CF90028E5
:10F3B00002D001240EF020FAF048006880472000B7
:10F3C00010BDED4870B50068804702200CF0CDFA02
:10F3D000EB48EA4D0078062806D1EA480078002874
:10F3E00002D02868804770BD0BF0E0FAE14C00289D
:10F3F00005D10EF041FA002801D1042000E00320DD
:10F4000060712868804760790428ECD10BF0C4FA59
:10F41000002802D0DC480068804706F009FB00287D
:10F4200001D006F0CBF9D9496078096888470EF019
:10F43000C1F90720A07007F0E9FF70BD10B50BF00F
:10F44000ABFA002802D0D0480068804706F0F0FAF6
:10F45000002801D006F0B2F9CC49C64C09686078A2
:10F460008847042060710EF0A5F90720A07010BD38
:10F4700070B5C04DA878002828D000242C7068787A
:10F48000FF2808D0C24909688847002803D0BF492F
:10F490006878096888470BF07FFABE4E002805D0CF
:10F4A0000BF072FAB1680120887401E0B0688474CE
:10F4B00006F0BEFA002801D006F080F9A8780928E5
:10F4C00005D100200EF046F9AC706C7170BD0120C2
:10F4D000F8E770B5002806D0002901D0AE4C04E052
:10F4E000AD4CA41E01E0AC4CA41C022501200EF082
:10F4F0008CF9002809D0A94B2A001B6801002000C4
:10F50000984701200EF0EDF90120002806D1FFF701
:10F51000AFFF022101200CF051F970BDA14B9548BD
:10F5200005211C68C90140789D4A0023A04770BD91
:10F5300070B500288F4C42D1A0789A4D012810D187
:10F540000EF0CAF802210028A17006D060782C685D
:10F550002021934A0023A04770BDFFF789FF0221B5
:10F5600025E002280ED10320A070012079A6B188E1
:10F570000100000024EC00A0000200000459A213C6
:10F580006071607805212C68C9018A4A0023A04770
:10F5900001200EF0C2F870BD032803D0042801D06A
:10F5A000072812D12078401C0006000E0328207086
:10F5B0000BD8E078012800D000200121FFF793FF4D
:10F5C00070BD01200CF004F970BDFFF75BFF032153
:10F5D000F7E70128F8D16F4801786F48062902D172
:10F5E00001780029F0D1007AFF2804D06D4909681C
:10F5F00088470028E8D1A0780528E5D102200CF042
:10F60000BEF9042060710720A0700EF0DDF80BF049
:10F61000CDF9002802D061480068804706F012FA50
:10F62000002801D006F0D4F807F0FAFE70BD10B53E
:10F630000EF0DEF8544800210170012141715E4B4B
:10F6400005211C68C90140785A4A0023A04710BD13
:10F6500070B505004C4C6078FF2804D15749002054
:10F6600009688847607028000DF0F8FF002801D075
:10F670000EF001F870BD10B5434CA078082810D1E9
:10F680000920A0700EF032F800280CD04A4B6078A8
:10F690001C6820214A4A0023A04701200EF03DF8B3
:10F6A00010BD092801D1FFF7EDFEA16801208847B0
:10F6B00010BD70B50600344C0D00A078002803D0B2
:10F6C0000120A847002070BD3848001D805DFFF76D
:10F6D000BFFF002802D10EF047F8F1E70820A07024
:10F6E00000202070A560344B267360781C682021B0
:10F6F000334A0023A047012070BD10B5224C0022E0
:10F70000227062732271E1700121A173A1702749F7
:10F71000091D085CFFF79CFF002804D101200EF0B2
:10F7200023F8002010BD244B60781C682021214A5A
:10F730000023A047012010BDF8B50125124EB07876
:10F74000072803D0002101200CF042F80520B070FA
:10F75000307900283BD001F090FD040037D0E088DC
:10F76000022834D9A188891EA1801649801EE08014
:10F7700009682000884707000CF0E9FD10F666BC18
:10F780000100000020EE00A000020000F0B11CAE5D
:10F79000002826D02100380020E000007CF200B0D4
:10F7A000CCF20004D0F20004365F00B0455F00B038
:10F7B00064F3000438F300043CF3000440F600B0A6
:10F7C0002E030004D0F10004E9EB000030F3000444
:10F7D00034F300041BED0000C4F1000406F018F837
:10F7E00009E00BF0BEF8002804D0002030700220A1
:10F7F000707100E000252800F8BDF1B582B0012647
:10F800000298C588002D01D10020FEBDA5490298AF
:10F81000096888470400A4480178032906D9FFF73E
:10F820003BFE032101200BF0DDFFEDE783789F49CC
:10F830009F4FDB1E3AF32CEE07054A61F8A8F8E566
:10F84000F8009948096840788847032D01D0042DB5
:10F850002FD1600903282CD1E7200440612C28D146
:10F86000904C029821688847924D297A884205D1A8
:10F87000216802988847697A884205D08A48002121
:10F8800001710120387402E0874901200871864C1B
:10F89000E078012807D10021FFF72FFE002020701B
:10F8A0000420A0700DE000280BD1FFF74FFF0600E9
:10F8B00007E07D48C078012800D000200121FFF733
:10F8C0001CFE79480178491C017084E00968070032
:10F8D00040788847012D01D0022D06D16009032808
:10F8E00003D1E7200440602C72D038780121401CFD
:10F8F00038700800FFF701FE75E0096805004078E0
:10F900008847A87B002806D00020A873387C0028F0
:10F9100001D10CF049FD6009022805D102982100AF
:10F9200006F007F8060026E0E00924D062480190BE
:10F93000077C06F091F8002801D005F053FF06205F
:10F940005E4AA8701268029821009047002801D1F1
:10F9500000260EE0002F0CD001980078002808D077
:10F96000574800688047002803D15649022009689B
:10F9700088470520A870554B7D211C68890268784E
:10F98000514A0123A04726E0474809681A318ABC3A
:10F99000010000001CF000A0000200008EAABB1EA7
:10F9A00040788847032D2AD16009032827D1E72012
:10F9B0000440612C23D1404C029821688847424D75
:10F9C000297A884205D1216802988847697A884255
:10F9D00005D03A48002101710120387402E037490E
:10F9E00001200871FFF7BCFE0600002E05D1FFF7CD
:10F9F0005DFD022101200BF0FFFE3000FEBD2F4C0B
:10FA0000E078012800D000200121FFF780FD207858
:10FA1000401C2070F1E70968070040788847032DF3
:10FA200001D0042D0BD16009032808D1E720044040
:10FA3000612C04D100240A20B87001E006E0012402
:10FA4000FFF734FDB96820008847D6E70026CEE7E7
:10FA500070B50500194CA07805282CD1184960789C
:10FA600009688847002D03D01E480068804717E0CA
:10FA70006079032814D1042060710720A0700DF074
:10FA8000B7FE0AF0A7FF002802D017480068804799
:10FA900005F0ECFF002801D005F0AEFE07F0D4FC25
:10FAA000A078052807D10E4B60787D211C6889025B
:10FAB0000A4A0123A04770BDC4F100047CF200B0E3
:10FAC00038F3000470E0000490ED0004CCDF000483
:10FAD00054F3000448F3000444F20004E9EB00008E
:10FAE00030F3000470F3000464F3000470B50D00FB
:10FAF0004178040000782A000BF022FD002803D092
:10FB0000FF4920784855012070BDFD4A10B5115CB1
:10FB1000052908D0FB4C8900091949680023DB43FB
:10FB20004B600521115410BD0522F548110010B598
:10FB30003AF3C2EAF24900208860C87488734874B6
:10FB400010BDF8B5040015000220F8F731FDEC48AF
:10FB5000005D052815D08100EA4808184068416812
:10FB6000A1420ED14078E84EE84F01280AD1E84979
:10FB7000280009688847002804D03A68012120003D
:10FB80009047F8BD316828008847F6E710B50DF0BA
:10FB9000BCFB002809D00022C2706122B96D861416
:10FBA0000100000018F200A0000200007A4205A344
:10FBB000012102700A2242708170D649886010BD0E
:10FBC00070B5D44CA068002809D08178002501299F
:10FBD00002D80DF0A0FB01E00DF0ABFBA56070BDFD
:10FBE00000280BD0022809D0052807D0CA4A810076
:10FBF000891849684978022900D101207047FFB56A
:10FC000081B006000D0000283BD0052E39D0300011
:10FC1000FFF7E6FF0400052833D0039930000BF00E
:10FC200080FC00282DD0BB4EB268002A29D09078E5
:10FC3000401DF62806D3FFF7C3FFFFF7B1FFB268F8
:10FC4000002A1ED0D31C111DD678002005E04F7865
:10FC5000891C7918401C0006000E8642F7D8761CD5
:10FC60000120002D1E7000D0002008700320487075
:10FC7000891C0C7003984870049888709078401D17
:10FC8000907005B0F0BDFFB581B00D000700160003
:10FC90000028F6D0052FF4D03800FFF7A1FF0400AC
:10FCA0000528EED0310038000BF03BFC0028E8D0EE
:10FCB00006200DF036FB0028E3D00122C11C002DE8
:10FCC000C27000D000224A7003228A70C91C0C70D6
:10FCD0004E70049A8A70612101700A2141700621D8
:10FCE00081700DF026FBCCE7FEB5052500280CD071
:10FCF000894901280CD0022807D0052805D08200A8
:10FD000051184968497A002900D105002800FEBD34
:10FD1000814800248068C668307A0028F6D001281F
:10FD200001D1346817E0804B00211F68BA206A4671
:10FD300001ABB847307A009A00210AE08B00F358F3
:10FD40001778DB681B78BB4202D18800345802E088
:10FD5000491C8842F2D8002CD8D060780228D5D12E
:10FD60006D480321027808E08B001B185B68A342F2
:10FD700002D10D062D0EC9E7491C8A42F4D8C5E709
:10FD8000052810B508D0002806D0634B8200D21891
:10FD90005268527A002A01D0002010BD0BF092FA6E
:10FDA00010BD5C48052210B50021C27327782A7F58
:10FDB0000100000014F400A00002000063BADBD3CD
:10FDC00001740273417312F06CE810BDF7B50E00B8
:10FDD000FFF794FF0500052801D10920FEBD01248D
:10FDE000F00709D0029A0021280012F05EE8040012
:10FDF000FFF7C2FA002C40D04B4FB0071DD5387B1F
:10FE0000052801D0A84202D1F87C002801D00024A6
:10FE100033E03D7302980BF0D2FE797B0843787390
:10FE2000029A0121280012F040E8B97B0400014346
:10FE300001D0012000E00020B873002C1DD0700715
:10FE40001BD5F87B052801D0A842E0D1F87C00281A
:10FE5000DDD1FD7302980BF0B2FE397C0843387493
:10FE6000029A0221280012F020E8797C0400014364
:10FE700001D0012000E0002078740020002CADD1DA
:10FE80000320FEBDF7B50E00FFF738FF050005287B
:10FE900001D10920FEBD0124F00709D0029A0021FA
:10FEA000280012F006E80400FFF766FA002C4DD097
:10FEB0001D4FB0071DD5387B052801D0A84202D1BF
:10FEC000F87C002801D0002440E03D7302980BF03C
:10FED00088FE797B08437873029A0121280011F08B
:10FEE000E8EFB97B0400014301D0012000E00020CD
:10FEF000B873002C2AD0700728D5F87B052801D0CC
:10FF0000A842E0D1F87C0028DDD1FD7302980BF007
:10FF100068FE397C08433874029A0221280011F0E7
:10FF2000C8EF797C04000BE08CF200B040F600B022
:10FF3000BCF100047CF3000468F20004ECF100045E
:10FF4000014301D0012000E0002078740020002C43
:10FF5000A0D10320FEBDFFB581B00E001D00FFF74C
:10FF6000CDFE0700052801D1092094E60124F00701
:10FF70000AD0039A2B000021380011F09EEF0400F4
:10FF8000FFF7FAF9002C13D0B00706D5039A2B001F
:10FF90000121380011F090EF0400002C08D0700708
:10FFA00006D5039A2B000221380011F086EF0400D9
:10FFB0000020002CD9D103206DE6FFB5BD0497BC0D
:10FFC0000100000010F600A0000200009752656ECC
:10FFD00081B01E00FF494978002921D000281FD098
:10FFE00005281DD0FFF710FE0500052818D0F01CCD
:10FFF00007063F0E38000DF0A8F9040010D0E57098
:020000021000EC
:1000000002992171667103993200A01D3AF37AE8D2
:1000100061202070092060702000A7700DF09DF90C
:1000200043E6FFB585B004000E00002702970F706D
:10003000089811F050EF050075D00798002808D0F7
:1000400001283BD002286ED1E87C002835D0002062
:1000500099E028780028F9D00020019029E0019843
:100060002818417805291DD00021217003216170D5
:100070004078FFF7C9FDA07008980BF08AFDE0708A
:100080000198207102987F1C401C0006000E02900F
:10009000307861783F064018801C307060783F0EE1
:1000A000A41C04190198401C0006000E04280190AD
:1000B0006DD2297802988142D1D868E06879002809
:1000C00065D00020019029E0019828188179052940
:1000D0001DD001212170032161708079FFF794FD0B
:1000E000A07008980BF055FDE070019820710298FF
:1000F0007F1C401C0006000E0290307861783F069D
:100100004018801C307060783F0EA41C04190198C0
:10011000401C0006000E0928019038D26879029927
:100120008842D1D833E035E0019812235843401972
:100130000490203003904079052820D002202070C0
:1001400003980079801C607003984079FFF75CFD8C
:10015000A07008980BF01DFDE070039804990279D7
:100160001431201D39F3CEEF307861787F1C4018B0
:10017000801C307060783F063F0EA41C0419019863
:10018000401C0006000E0190E97C8142CCD838006A
:1001900009B0F0BD0020FBE7FEB5050000208E4948
:1001A00000900968F62088472B00002269460190DC
:1001B000FFF737FF01266127002802901BD06B460E
:1001C0001878801C0006000E0DF0BFF8A3F7D39539
:1001D000010000000CF800A000020000504B673343
:1001E0000400C01C0670029941706B461A78019990
:1001F000801C39F392EF022127706B4661701978E9
:100200002000891CA1700DF0B2F801982B0001228A
:100210006946FFF710FF002802901BD06B46187844
:10022000801C0006000E0DF09AF80400C01C067039
:10023000029941706B461A780199801C39F36CEF72
:10024000022127706B46617019782000891CA1700B
:100250000DF08DF801982B0002226946FFF7EBFEA6
:1002600005001AD06B461878801C0006000E0DF0B1
:1002700076F80400C01C067045706B461A78019928
:10028000801C39F34AEF022127706B4661701978A0
:100290002000891CA1700DF06AF855490198096881
:1002A0008847FEBD002010B5FFF780FF0120FFF753
:1002B0007DFF0220FFF77AFF02200DF050F80022A8
:1002C000C2706121027101700221417081700DF0D4
:1002D0004EF810BD022010B50DF041F80022C2709A
:1002E00061210271017005214170022181700DF0C0
:1002F0003EF810BD022010B50DF031F80122027158
:1003000003226121C27001700621417002218170B7
:100310000DF02DF810BDF3B581B001250F002800B8
:100320000DF01DF84F2101700021417001210400E2
:10033000C61C012F817000D2002501980078FFF7BC
:10034000F1FC2C498000401840684078032800D018
:10035000002511F0CEED00280DD1002D0BD002208C
:1003600011F0CAED002806D00020307020000CF0FB
:10037000FEFF0020FEBD0320F7E7F8B507000229C5
:100380003FD3891E0D0638782D0EFFF7CBFC0228CF
:1003900037D1BC1C002651E02078002833D001283A
:1003A0002FD1A01C0B2D2CD30B3D01782D062D0E2B
:1003B000022926D14178042923D182784179120675
:1003C0001143C278037912041B021A431143801DA2
:1003D0000278032A15D14278012A12D392AB53ED49
:1003E0000100000008FA00A000020000A4A3D98EBA
:1003F0006B1C9A420FD80904090C07E084E0000442
:10040000D8F10004DCF1000440F600B0801C04F0D8
:10041000EDFE002818D10320F8BD062DFBD360782F
:100420000428F8D1A178607909060843E178227997
:10043000090412021143AD1F08432D0600042D0EBE
:10044000000C04F0F1FEE4E76078A41C0419761CAB
:100450007878B042AAD80020F8BD10B5FFF797FF12
:1004600004000BD101200CF084FF4F220270022205
:10047000427001228270C4700CF083FF200010BD16
:10048000F3B581B00CF073FF0500C41C029801267F
:10049000032703285AD30298401E0006000E02903C
:1004A00001980078FFF748FC02284FD10198407866
:1004B000002823D0012849D101980299C01C08299D
:1004C00044D30178022941D1417804293ED1817871
:1004D000427909060A43C178007909040002014300
:1004E0000A43009204F0ABFE009AF12182422DD221
:1004F000009A801AF12814D90E0014E004F09FFE2F
:100500000299022922D3002204216270A170010EF7
:10051000E170010C2171010A6171A071072622703E
:1005200015E00604360C01206070B01CA070E77066
:100530002671009932000904090C601D04F066FE62
:100540000020761D3604360C207000E027702478D9
:100550004F2028706F702800AE700CF012FF200042
:10056000FEBDF7B5901C15000606360E30000CF0E7
:1005700000FF009A04000027C01C3900002A00D1A7
:1005800003210170457001992A00801C39F3CEEDDA
:100590006F20207067702000A6700CF0F2FEFEBD88
:1005A00070B50400FC4D0026297B012800D0E97BB2
:1005B000052914D011F0AEEC11F0B0EC200011F0D0
:1005C000B2EC00280BD0A87C002800D00124012028
:1005D000012C00D10020002111F0A8EC0600300011
:1005E00070BDF8B500240327EB4D2600F784C37CCB
:1005F0000100000004FC00A000020000BD5B07FE3B
:10060000287D00280BD0012821D002282BD00328D8
:1006100045D1012011F098EC042028753DE0687C5C
:10062000002807D00220FFF7C5FF00280CD00120CA
:1006300028750AE0A87B002806D00120FFF7BAFF42
:10064000002801D02F7500E001246E741EE0012007
:1006500011F07AEC0121080011F072EC002817D09B
:1006600002202875F8BD012011F06EECA87B00284F
:1006700008D00120FFF79EFF002801D02F7504E06D
:10068000012402E004202875EE74AE73002C06D01D
:10069000042028756F756E74AE73EE7402E0287DC9
:1006A0000428DFD1002101200AF061FCF8BD10B55B
:1006B000BE4CA07B002807D1607C002804D100211B
:1006C00001200AF054FC10BDB94800688047E07C66
:1006D000B849002804D00868804703206075EEE719
:1006E000627C0120002A00D0A074E0740868804772
:1006F00000202075FFF77FFF10BD7CE7AB4901208C
:10070000C97C002900D000207047F3B583B00500F4
:100710000026049C641C022815D100202070A649E4
:1007200001206070097BA170E41C207002206070C1
:10073000A2480226017AA170407AE070241D0021AF
:10074000282001AA02E00021272001AA9C4B1F6853
:100750006B46B847022020700820607002000199A3
:10076000A01C39F3EEEC6078761CA41C3606041944
:10077000360E022D01AA02D100212D2001E0002118
:100780002B208F4B1F686B46B84703206B462070A9
:10079000187860701A780199A01C39F3D2EC60784F
:1007A000A41C0419761C3006000E022D02902AD1DA
:1007B00004202070834E262262703168A01C39F319
:1007C000C0EC6078029FA41C041905214C22217002
:1007D000627031687F1C2631A01C39F3B2EC61785D
:1007E000A01C0C18062113222170627031687F1C36
:1007F000A431A01C39F3A4EC6178A01C908DBA56EA
:100800000100000000FE00A00002000049B3B9434F
:100810000C187F1C3806000E029007202070002064
:100820000600A71C6070062070436C494118887848
:10083000A84207D160780622C01939F38CEC6078A1
:10084000801D6070761C3606360E042EEBD314E045
:100850000621714361480918487800280AD0887831
:10086000A84207D160780622C01939F374EC607889
:10087000801D6070761C3606360E2C2EE8D360780C
:10088000049AC1190298401C10700498081A0004B8
:10089000000C05B0F0BDF7B582B0002417000129A7
:1008A0007ED302780229019200D3441C491E080617
:1008B000000E039001987AE062780399901C8842B8
:1008C0006FD80398801A801E0006000E03902378CC
:1008D00039F32EEE0862050B161C20272C623C48CB
:1008E000A1780172E178417256E013002820022FAE
:1008F00000D027203A4DA21C2D680021A8474BE0CC
:1009000013002D20022FF5D02B20F3E73248A11C35
:10091000006803E03048A11C0068263039F31AEC67
:100920003AE02D48A11C0068A430F7E7A61C380067
:100930000BF08FFF29490025062068434018827874
:10094000BA4205D1727842706078B61D801F60701F
:100950006D1C2D062D0E042DEED318E006216943E3
:100960001E480818417800290ED13178891CA94207
:100970000AD1B178B94207D10622310039F3EAEB46
:100980006078B61D801F60706D1C2D062D0E2C2DFD
:1009900002D260780028E1D16078A41C041901E03B
:1009A00007E025E00198401E0006000E0190002897
:1009B00082D10C4A012F17D10021252016E000001A
:1009C0008CF200B0CCF20004D0F200047CF200B053
:1009D00090ED0004ECF1000408F20004ECED0004DA
:1009E000F0F10004F8F1000400212620126890477D
:1009F0004FE70000FF4810B5016B4908490001634B
:100A0000FC48403001694908490001610BCDDAB961
:100A100001000000FCFF00A0000200008D66666877
:100A2000F94880300168490849000160F7480068CA
:100A3000804755204006026902218A430261C16055
:100A4000F3480068804710BDEF4A0121803203005F
:100A500000B539F378ED09060B0A111506110611D8
:100A60000A00E94A106B0843106300BDE6484030B5
:100A700002690A43026100BD10680843106000BDAE
:100A800090690843906100BDDF4B002A10B505D185
:100A9000002903D05A681C0622435A60002902D05C
:100AA0000121490701E00121C9070843586010BD31
:100AB000F8B5D54B9A6B2024A243C5070124002D1D
:100AC00001D0224301E0520852009A63CE4B4033DA
:100AD0001A6A0225AA43860701D5224301E052087B
:100AE00052001A62C84B80331A6AAA43FF256D1C54
:100AF000AA43050701D5224301E0520852001A62B9
:100B00009A68450701D5224301E0520852009A60D5
:100B10005526BE4DBE4F7606002807D1286880476F
:100B20003069400840003061F4600EE000070ED0EC
:100B3000002904D0002201210A20FFF7A5FF286820
:100B40008047F46030692043306138688047F8BDE1
:100B5000AD48416802061143416070477047552215
:100B60005206516B202399434001014318208143D1
:100B700051637047F8B506000020FFF7F0FFA54865
:100B8000C06A01214905084349008843A149C86258
:100B90005522520611681020014311609D4A9E495A
:100BA000D1639E4AFF21083111609B49891F9162E0
:100BB000954CE36801210B43E360002E02D1536A98
:100BC00003435362904D80352C6B914F84438F4883
:100BD000002E06D100680C4380472C63386880479C
:100BE000F8BD060000688047286B20210843286371
:100BF00038680C438047306880472C6338688047EA
:100C0000FFF7A6FFF8BD70B506000C00FFF7FCFE6D
:100C10007D4D8035002C04D000210800F13384C5BF
:100C200001000000F80101A000020000BF0D01D783
:100C3000FFF748FF09E07A4800688047286B2021C9
:100C400008432863774800688047286B40084000C5
:100C50002863002C08D077480078032804D10420AA
:100C600002F07AFC01F041FB6C48C1684908490078
:100C7000C160002E05D055214906086802221043A4
:100C8000086070BD10B511F082E9002802D0012182
:100C900008000CE011F05EE9032806D101210800EC
:100CA000FFF7BBFF11F076E910BD01210020FFF72F
:100CB000B4FF10BD552040060168022211430160B7
:100CC000704770B50C000025030039F346EC090AA3
:100CD0001D2521250A0A06062500002C1CD1564C8C
:100CE0001AE0002C18D15548407803280AD005DCBA
:100CF000002807D001280FD1514C0DE0082801D061
:100D00000A2809D14F4C07E0002C05D14E4C03E0D6
:100D1000002C01D1092464054C488078002801D1B9
:100D20004B4824184B48844200D90400002A03D0C1
:100D30000125280001F073FB60004008E907084323
:100D40003649886044490120087070BD33484349E2
:100D500041614349C161FF210A31016181617047ED
:100D60002F4810B5006880475520400601680122D1
:100D700092029143016081680322114381600169FD
:100D8000FF22521C914301610021816125480068C6
:100D9000804710BD264870B5403041680126314378
:100DA00041604168B1434160552464062068304386
:100DB0002060C046C046C046C046C046C046206807
:100DC000102108432060FFF7CBFF2068082108436B
:100DD000206000210800FFF775FE134D403528699B
:100DE000310208432861FFF7B1FF002020613F2056
:100DF000E0610D488030C168F82291431831C1602C
:100E000018484671184800688047E96840208143C7
:100E1000E960296901432961034927E0400000AAEC
:100E2000CCF20004D0F20004400100AAAAF9B37B7E
:100E300001000000F40301A0000200009F69625459
:100E400003060000000800AA2D5E00B0FF0F00009E
:100E500080ED000410350600D4090000D00800041D
:100E600083ED0004AC080000FFFFFF0F045E00B03C
:100E7000001000AA001200AA001F00AABCF0000483
:100E80004039086A072212069043AA0480180862B3
:100E9000D0132860FF48016B3F2252069143EA04B9
:100EA0008918016370BD70B50500FA4CE06805D182
:100EB000F9480078032801D101F021FA55204006B5
:100EC0000168082291430160416B202291434163F4
:100ED000F348F249D2000160F24B2B214905D96356
:100EE000F1498162EB48403081681F231B0299431E
:100EF00005235B02C9188160A06B80218843A06331
:100F0000002D05D1A0691043A06120691043206124
:100F100070BD0021080010B5FFF7DEFDFFF788FD6A
:100F2000FFF71EFF552040060168082211430160AB
:100F3000D94900204870087010BD10B50400002188
:100F400055204006C0694200D20D8002400F02D0F9
:100F5000521C1204120C002A06D0D44822600168E8
:100F6000D34839F316E90121002902D1002020607D
:100F700010BDCF4810BDF7B50D00C64FB869FF21B1
:100F8000491C0843B861386908433861C948009969
:100F90002A0039F3FEE8022055267606F060C6489E
:100FA000006880473069022420433061C3480068EC
:100FB0008047C3480678FEF7CAF9002804D1029991
:100FC00000223000FFF787FE3300B24EFF210902F6
:100FD00028020122803639F3CAEA09063463404AFE
:100FE000064006406300AB4B1E6BB54F00237F7875
:100FF000002F04D101231B061E43102302E001270A
:101000003F06BE438E430643F0208643AD48164359
:10101000264386439F4806630099097850290ED0DD
:1010200020210B4313439B4A80218B43403291681C
:101030001F242402A1430524640209197A49C39E8E
:1010400001000000F00501A000020000521D611A1D
:10105000916083632EE0944A403213698B430343CB
:1010600023431361106A40084000106222E0336895
:10107000E027BB43A0338B43034313432343336035
:1010800018E0B7698F43074327431743402087433E
:101090009248007801280CD0B06940084000B06147
:1010A000FFF774FDF06A0022000100090121FFF73B
:1010B00009FDB761002000E0401CA842FCD3FEBD42
:1010C0007948C0684006800F072800D9082070477B
:1010D000FFB5022055241D00640681B0E0607B4806
:1010E0000068804720690226304320617848006804
:1010F00080476D4FB869F1010843B861386908430A
:101100003861FEF72EF904006D4800210838012DE2
:1011100002D0022D02D100E001210170002C03D089
:101120006F480078042826D1002D1FD00021080028
:10113000FFF7DCFC022D19D1B86869070843B860D5
:10114000002001F080F9202055214906C8605F4841
:1011500000688047552040060069202188435521BA
:10116000490608615A480068804704E003990298DC
:101170000022FFF7BAFD01984B49029B0002403163
:1011800039F3FEE909063FB45F70065F065FB400FD
:101190003B6B5048427801200006002A01D10343EE
:1011A00000E08343FF2000028343019821220006D0
:1011B000000C03434848E0308343334301201F269B
:1011C00003433602002C09D1FFF77AFF002805D12E
:1011D0008868A122B0430126360303E08868B04343
:1011E00005267602801988603A484078002801D1A7
:1011F00010200243BA633B6308694008400008615D
:1012000018E02949403109690122FF2311431B02DB
:10121000994301433143012C05D1234B4033186AD4
:10122000104330431862204840300161386B400859
:10123000400038631C48803001684908490001605B
:1012400054E0A0220243012002431748DD54E78EF8
:1012500001000000EC0701A000020000DFA1A55280
:101260003243803002600869400840000861386BF2
:1012700040084000386343E0104F8037B969019B54
:101280004022002B01D1114300E09143FF221202C2
:101290009143014303200143B8690E004008400018
:1012A000B861FFF77DFCF86A002200010009012106
:1012B000FFF712FC012C22D1386A1DE0400000AA81
:1012C0002D5E00B010830000000800AA400100AAB3
:1012D000FD0500000C5E00B0A4F200B0001000AAF2
:1012E000CCF20004D0F2000480ED00040C00800079
:1012F000365F00B0A4F500B0032108433862BE6138
:10130000002D0DD0029804280AD0002C03D0FB48F1
:101310000078042804D1002201210A20FFF7DCFB19
:1013200005B0F0BD7FB50028F54D2CD001AA02A96B
:1013300003A86B4604F00BFD6B46187A002803D017
:10134000FF21FD31880002E00121490288006B463F
:101350001A7B0400002A02D189008000A4004A0000
:10136000852312185B01D2186B461B79022B04D11E
:10137000602359430818001982182C6804210020A2
:101380000123A0477FBD0022042110002C68022306
:10139000F7E755204006C069DA494000C00D888053
:1013A000C88008007047D74900201031C880080065
:1013B0007047D5488169FF22521C114381617047F3
:1013C00055204006C0690006C00F704770B5012661
:1013D000360303207500000355246406E060CB4803
:1013E000006880472069304328432061C84800686E
:1013F000804770BDC54810B500688047552040063D
:10140000016903221203914301611100C160C048C8
:101410000068804710BD70B50500BC480068804773
:10142000B64C2034A078012802D0022806D101E071
:10143000FFF7B6FB00210800FFF70DFCFFF7C6FF22
:101440000320A070B34900222800FFF758FC202099
:1014500055214906C86008692022104318E5125B2F
:1014600001000000E80901A00002000061ECDDFAC3
:101470000861FFF7AFFFA94A00280ED00B690120D1
:1014800003430B61072D14D0082D04D1A34B8033E7
:101490009968014399600420A07090680121490770
:1014A000084390609A490020C8719E4800688047B0
:1014B00070BD916B01439163EDE7984800B5016BF6
:1014C000490849000163016B0122114301631B209C
:1014D00000220121C001FFF709FB00BD00B5FFF7A5
:1014E00005FB00BD0022110000B5FFF7FFFA00BDAB
:1014F0008A4810B580680401240905F028F80028FE
:1015000001D08A48807A00280AD001280ED002280B
:1015100018D0032810D101200004854900190AE0E1
:1015200001208349C0040019383104E001208049BA
:101530008004001918314418002211002000FFF720
:10154000D5FA10BD01207A49400400190831F2E7AC
:1015500010B5724A04000800116B49084900116374
:101560006E4A403211694908490011616B4A803264
:101570001168490849001160916949084900916161
:10158000FFF794FAFFF716FB002201212000FFF776
:10159000ADFA10BD70B50D0060490400C031886A15
:1015A000644AC008C000C01C1040FF22D20080184E
:1015B0000322120490430A02801888620020FFF779
:1015C0000BFB002D04D001F036F88007400D041904
:1015D000102055256D06E86051480068804728694D
:1015E000102108432861012211002000FFF77EFA34
:1015F00002F096F8514BE1091C681F314E4A002356
:10160000A0474F490120087046480068804770BDD8
:10161000002810B505D141488169FF22521C1143B1
:1016200081613F4800688047552464062069102185
:10163000884320613B4800688047E0694009C00753
:1016400004D0E06920210843E061012010BDF7B516
:1016500084B0002407001B20019006982500260076
:1016600004280394029403D005993800D822572601
:1016700001000000E40B01A0000200004188BE79D7
:1016800000F0D8FD2A490322069BFC20120380317A
:1016900038F394EF090680CFDCFA06DC06DC47005D
:1016A000002F61D0012F63D0022F66D0032F02D10B
:1016B000294C2A4D2A4E1E4A4032D3681B0F1B0765
:1016C0002343D3601A4BDD6316605568AD0AAD0243
:1016D000FF3531355560059A002A53D0012A54D080
:1016E000022A54D0032A00D1164C5A6B120F12074B
:1016F00022435A634A6B8243FF2000028243012047
:10170000C0031018032210434863886B154A104029
:10171000032212068018800BBF228003D20080189B
:101720008863D4E0A4F500B05CF100040C5E00B066
:10173000400000AACCF20004D0F20004FC3F0000FC
:1017400067DF00045C0400000780FFFFBF2C01007E
:1017500030F30004305E00B0441A00000A121A028E
:10176000131B2428FFFF00C0F84CF94DF94EA2E7E7
:10177000F64CF94DF94E1B3C9DE7F44CF84DF94EF3
:101780002B3C98E78324E400AFE7F74CADE7F64C39
:10179000103CAAE7002F33D0012F36D0022F39D0CA
:1017A000032F03D1F14BF24DF24E03934B6B834366
:1017B000FF20C83300028343981803221043486374
:1017C000886BED4A1040052252058018800B80037B
:1017D000A0308863E949039808624D628E62086B05
:1017E000E74A000F0007801808630598002816D004
:1017F000012816D0022818D0032818D0029812E029
:10180000E04BE14DE14E0393D0E7E14BE14DE24E79
:101810000393CBE7E14BE24DE24E0393C6E7E24888
:1018200000E0E2480290486151E0E148FAE7E1480F
:10183000F8E74B6B8343FF20C833000283439818BB
:101840000222104340084000486340E01F230193F8
:10185000A7231B014B6067239B01CB600B614B6B84
:101860008343FF20C83300028343981803221043A8
:101870004863886BC04A104005225205EFCDD9DA83
:1018800001000000E00D01A0000200008CFCBD374B
:101890008018800B8003A0304CE7FFE7086A202205
:1018A0001023042F01D1904306E0052F01D190436E
:1018B00007E0062F02D11043984303E0072F01D120
:1018C000104318430862C869020F832012074001C1
:1018D0001018C861C86A020F21201207C001101831
:1018E000C862AB498031C869B84A1040019A1204F5
:1018F0001043C86107B0F0BDB54B10B501241C7092
:1019000058709970DA7010BDB14A1378002B04D169
:101910000822027000200A70704753780370907894
:10192000087001207047F3B503009948C030C16BBF
:10193000012500222D05032714006E107F0538F3C2
:1019400048EE0906150A151D061506150A00019A26
:10195000002A0BD103E0002A06D0002C02D1A943B3
:10196000314305E0002A05D1002C0AD02943B143B8
:10197000B94306E0002C04D0002A02D0A943B143A9
:101980003943C163FCBDF7B582B000260298370029
:10199000340035000928019602D00398092802D1A5
:1019A0000020029003900399029800F04DFC7848C3
:1019B000049B403038F30CEE09064B36CAD206CAF7
:1019C00006CA36006D4A6D4B02986C49103A183BB6
:1019D000002828D001282BD002282DD0032802D19E
:1019E0007C4C7D4D1E006A48C7683F0F3F07374358
:1019F000C760674F403FFC6305604468A40AA402C7
:101A0000FF34313444600398002819D001281AD0DB
:101A100002281AD0032800D11E00786B000F00079F
:101A2000304378639AE4554E4E4C4F4D1736DAE703
:101A30006A4C6B4D0E00D6E76A4C6B4D1600D2E730
:101A40004E4E5B3EE9E70E00E7E71600E5E70023B0
:101A5000029E180019001A00002E59D0012E5BD0EA
:101A6000022E61D0032E06D10223604F604D614CDF
:101A7000180019001A00604E3E40BF01BF0DFB1850
:101A80001B041E43E30A6405640DDB023D4A1B2E62
:101A900001000000DC0F01A0000200005E302B5EA0
:101AA000241A23435A4C5B4F1C401B03DB0D5B1A6B
:101AB000DB021C4323006400640DA41A3B40240590
:101AC0002343EC0A6D056D0DE402281804435048C9
:101AD00020402403E40D6118C902084304004000BB
:101AE000400D304980183C40000504430E624B62B3
:101AF0008C628869FF22120490430B22D204801862
:101B00008861086B444A000F000780180863039837
:101B100000281BD001281BD002281DD003281DD06F
:101B2000019817E03D4F3E4C3E4D02E03E4F3F4C8A
:101B30003F4D1023180019001A00A6E704231800CF
:101B400019003C4F3C4C3D4D1A009EE7204800E0F8
:101B50002048019048610BE41F48FAE71F48F8E766
:101B60003521C90141601521C901C160016163E7E7
:101B700066E00000771A000066A6E60299D917D938
:101B80002E4E6E024F6F9088162636022737484831
:101B90007404000000070300090890000C20C00036
:101BA000FFFF00C0800000AA8C150000003F11005C
:101BB0004F78F00459C89005001F090027387002BB
:101BC0002D68D002000F050013183001173870017E
:101BD000000508508002042840010214A000010AF8
:101BE000FFFF00F0065E00B00A151E02141D281843
:101BF00031517102507090601929390228384830EB
:101C000000076000C000020C9880C009FFFF00FCC4
